:020000040000FA
:1000000088EF47F0FFFFFFFF08D0FFFFFFFFFFFF74
:10001000FFFFFFFFFFFFFFFF00D0E0CF02F1010174
:10002000D8CF01F1E8CF00F181509EB0A2EC38F0BA
:10003000F2B489EC38F0A1B29EEC38F09EBA48ECEC
:1000400038F0F2B277EC38F0F0B07DEC38F000C167
:10005000E8FF01C1D8FF02C1E0FF1000FFFFFFFF72
:10006000FFFFFFFFFFFFFFFFFFFFFFFFFFFFFFFFA0
:10007000FFFFFFFFFFFFFFFFFFFFFFFFFFFFFFFF90
:10008000FFFFFFFFFFFFFFFFFFFFFFFFFFFFFFFF80
:10009000FFFFFFFFFFFFFFFFFFFFFFFFFFFFFFFF70
:1000A000FFFFFFFFFFFFFFFFFFFFFFFFFFFFFFFF60
:1000B000FFFFFFFFFFFFFFFFFFFFFFFFFFFFFFFF50
:1000C000FFFFFFFFFFFFFFFFFFFFFFFFFFFFFFFF40
:1000D000FFFFFFFFFFFFFFFFFFFFFFFFFFFFFFFF30
:1000E000FFFFFFFFFFFFFFFFFFFFFFFFFFFFFFFF20
:1000F000FFFFFFFFFFFFFFFFFFFFFFFFFFFFFFFF10
:10010000001210180606080A0A0C0606080A060A53
:1001100006060808060E06060A0A08140C0A060A4D
:1001200008060606101010101010101010101010F5
:1001300010101010101010101010101010101010BF
:10014000101010101014161416120C140E1414148F
:100150000E180A0608080A060C0A08080808060607
:10016000040A0C120A0A0A060A0E140808061214D7
:10017000040E140806100E0C0606080606060606EF
:10018000080804040A16161614080A080806060ABF
:100190000808040A0E140A0C0A141010101010108B
:1001A000101010101010101010101010101010104F
:1001B000101010101010101010101410120E08084B
:1001C00006141414141414141414141414141414FD
:1001D00014141414141414141414141414141414DF
:1001E0001414141414141414141414140A0A0A08F9
:1001F0000808080E0614100A100C06060606060863
:10020000020E0E080808060606060A0A0408040E6E
:100210001412140E0A0E0C100E0A0A0A0E0C10000C
:10022000FFFFFFFFFFFFFFFFFFFFFFFFFFFFFFFFDE
:10023000FFFFFFFFFFFFFFFFFFFFFFFFFFFFFFFFCE
:10024000FFFFFFFFFFFFFFFFFFFFFFFFFFFFFFFFBE
:10025000FFFFFFFFFFFFFFFFFFFFFFFFFFFFFFFFAE
:10026000FFFFFFFFFFFFFFFFFFFFFFFFFFFFFFFF9E
:10027000FFFFFFFFFFFFFFFFFFFFFFFFFFFFFFFF8E
:10028000FFFFFFFFFFFFFFFFFFFFFFFFFFFFFFFF7E
:10029000FFFFFFFFFFFFFFFFFFFFFFFFFFFFFFFF6E
:1002A000FFFFFFFFFFFFFFFFFFFFFFFFFFFFFFFF5E
:1002B000FFFFFFFFFFFFFFFFFFFFFFFFFFFFFFFF4E
:1002C000FFFFFFFFFFFFFFFFFFFFFFFFFFFFFFFF3E
:1002D000FFFFFFFFFFFFFFFFFFFFFFFFFFFFFFFF2E
:1002E000FFFFFFFFFFFFFFFFFFFFFFFFFFFFFFFF1E
:1002F000FFFFFFFFFFFFFFFFFFFFFFFFFFFFFFFF0E
:100300000000010F0019010F0002010F4102010F4F
:100310004102010F1423010F1441010F1423010F97
:10032000145F010F147D010F14B9010F7302010F47
:100330000018010F0000010F3202010F0A1E010F09
:100340000A37010F0A50010F0A69010F0A82010FD3
:100350001423010F2041010F205F010F209B010F8B
:100360000600010F3702010F0E02010F2802010FD4
:100370003202010F1423010F6400010F6419010FF1
:10038000644B010F6464010F0000010F2823010F6B
:100390002823010F2823010F2823010F2823010FF1
:1003A0002823010F2823010F2823010F2823010FE1
:1003B0002823010F2823010F2823010F2823010FD1
:1003C0002823010F2823010F2823010F2823010FC1
:1003D0002823010F2823010F2823010F2823010FB1
:1003E0002823010F2823010F2823010F2823010FA1
:1003F0002823010F2823010F2823010F2823010F91
:100400002823010F2823010F2823010F0023010FA8
:100410000041010F005F010F007D010F009B010FE4
:1004200000B9010F00D7010F0023010F0041010F98
:10043000005F010F007D010F009B010F00B9010F4C
:1004400000D7010F6696010F0000010F6CD8010F55
:100450006CD8010F6400010F0000010F0000010FB4
:100460000000010F0000010F0000010F0000010F4C
:100470000000010F0000010F0000010F0000010F3C
:100480000000010F2802010F1423010F147D010F3A
:10049000557D010F557D010F557D020F557D010FD3
:1004A0000000010F0A02010F0000010F0000010F00
:1004B0001423010F1441010F0E02010F0000010F60
:1004C000145F010F0A02010F0009010F557D020F91
:1004D0000012010F001B010F0024010F002D010F5E
:1004E0000036010F6432010F6419010F6432010FED
:1004F000644B010F6464010F6400010F6419010F64
:100500001441010F4141010F4141010F6432010FBC
:100510000A00010F0A19010F0A32010F0A4B010FDD
:100520006432010F557D010F6978010F693C010F9D
:100530004102010F149B010F2A48010F3C02010FD9
:100540003460010F3478010F644B010F0000010F7C
:100550000008010F0227010F0230010F557D010F26
:100560001441010F2823010F2823010F2823010F15
:100570002823010F2823010F2823010F2823010F0F
:100580002823010F2823010F2823010F2823010FFF
:100590002823010F2823010F2823010F2823010FEF
:1005A0002823010F2823010F2823010F2823010FDF
:1005B0002823010F2823010F2823010F2823010FCF
:1005C0002823010F2823010F2823010F2823010FBF
:1005D0002823010F2823010F2823010F2823010FAF
:1005E0002823010F0D02010F000000000201010F7E
:1005F0000230010F0000010F0000010F0000010F89
:100600000023010F0041010F005F010F007D010F6A
:10061000009B010F00B9010F00D7010F0023010F4C
:100620000041010F005F010F007D010F009B010FD2
:1006300000B9010F00D7010F0023010F0041010F86
:10064000005F010F007D010F009B010F00B9010F3A
:1006500000D7010F0023010F0041010F005F010FC0
:10066000007D010F009B010F00B9010F00D7010FA2
:100670000023010F0041010F005F010F007D010FFA
:10068000009B010F00B9010F00D7010F0023010FDC
:100690000041010F005F010F007D010F009B010F62
:1006A00000B9010F00D7010F0A02010F557D010F9C
:1006B000020C010F6419010F6400010F6400010FA7
:1006C0006419010F6400010F020C010F6464010F33
:1006D0001441010F021E010F147D010F1E02010FB4
:1006E0001423010F6419010F6432010F644B010FD1
:1006F0006464010F6400010F6432010F0000000FF9
:100700001423010F2802010F6923010F6923010F30
:100710006923010F0101010F41A8010F0730010BEF
:100720007887010F0227010F00D8010F0A08010F77
:100730000A10010F0000010F1802010F0023010F22
:100740000041010F007D010F009B010F145F010F9D
:100750001441010F145F010F147D010F149B010F51
:100760006432010F6400010F5A36010F145F010F4C
:10077000147D010F149B010FFFFFFFFFFFFFFFFF21
:10078000FFFFFFFFFFFFFFFFFFFFFFFFFFFFFFFF79
:10079000FFFFFFFFFFFFFFFFFFFFFFFFFFFFFFFF69
:1007A000FFFFFFFFFFFFFFFFFFFFFFFFFFFFFFFF59
:1007B0004275696C64696E67204D443220486173EC
:1007C000687D506C6561736520576169742E2E2EAB
:1007D0007D7D4865696E72696368735765696B6191
:1007E0006D70204F535443327D7D4D656E753F7D56
:1007F0004D656E753A7D4C6F67626F6F6B7D4761BB
:10080000732053657475707D5365742054696D65EC
:100810007D7D5265736574204D656E757D7D536574
:100820007475707D457869747D7D576169742E2E6D
:100830007D7D4D443220486173683A7D4465736123
:10084000747D496E746572666163657D537461720F
:10085000747D446174617D7D4865616465727D7DF0
:1008600050726F66696C657D446F6E652E7D436165
:100870006E63656C2052657365747D7D54696D652A
:100880003A7D446174653A7D53657420486F757292
:10089000737D52657365742E2E2E7D7D4C6F67625D
:1008A0006F6F6B7D437573746F6D2046756E6374E7
:1008B000696F6E7320497D7D5265736574204D6547
:1008C0006E757D7D5365742054696D653A7D4D6FFD
:1008D00072657D7D4465636F706C616E7D7D47617F
:1008E000736C6973747D4D6F72657D7D4578697435
:1008F0007D7D4E6F466C797D5374617274204469BE
:100900007665205B636D5D7D456E64204469766528
:100910002020205B636D5D7D456E642044656C61C5
:10092000792020205B735D7D506F776572204F6664
:10093000662020205B735D7D5072652D6D656E7540
:10094000202020205B735D7D76656C6F6369747910
:100950005B6D2F6D696E5D7D57616B652D757020C8
:10096000205B6D4261725D7D6D61782E537572669C
:100970002E5B6D4261725D7D474620646973706CC9
:10098000617920205B255D7D6D696E2E204F3220C0
:100990004469732E5B255D7D44697665206D656EC7
:1009A000757320205B735D7D53617475726174652E
:1009B000207820205B255D7D4465736174757261CC
:1009C000746520785B255D7D4E6F466C79205261A1
:1009D00074696F205B255D7D474620616C61726D97
:1009E000203120205B255D7D474620616C61726D62
:1009F000203220205B255D7D4465636F204F666655
:100A00007365745B646D5D7D70704F32206C6F77C1
:100A1000205B634261725D7D70704F322068696750
:100A2000685B634261725D7D73686F772070704FA1
:100A3000325B634261725D7D73616D706C696E677C
:100A4000207261746520207D44697669736F72201D
:100A500054656D702020207D44697669736F722023
:100A60004465636F6461747D44697669736F722055
:100A70004E6F74557365307D44697669736F72206B
:100A800070704F322020207D44697669736F722028
:100A9000446562756720207D44697669736F7220B2
:100AA0004E6F74557365327D73686F7720434E5374
:100AB000202020205B255D7D4C6F67626F6F6B206F
:100AC0006F6666736574207D4C6173742044656342
:100AD0006F2061745B6D5D7D456E642041706E6F4B
:100AE00065205B6D696E5D7D53686F77205662612E
:100AF0007474205B3D315D7D546869732070726F42
:100B00006772616D2069737D64697374726962755F
:100B100074656420696E207468657D7D686F70659A
:100B200020746861742069742077696C6C20626538
:100B30007D7D75736566756C2C20627574205749D0
:100B400054484F55547D414E592057415252414EC1
:100B500054593B20776974686F75747D6576656E4E
:100B60002074686520696D706C6965647D7D77614E
:100B70007272616E7479206F667D4D4552434841B3
:100B80004E544142494C495459206F727D7D46492B
:100B9000544E45535320464F5220417D50415254AC
:100BA0004943554C415220505552504F53452E7D8C
:100BB0005365652074686520474E552047656E650E
:100BC00072616C7D5075626C6963204C6963656EFF
:100BD000736520666F727D7D6D6F726520646574CC
:100BE00061696C733A7D7777772E6865696E726993
:100BF0006368737765696B616D702E64657D4465AC
:100C0000636F73746F707D7D6D2F6D696E7D4E6F38
:100C10002053746F707D4465636F73756D7D446997
:100C2000766574696D657D7D44657074687D46691F
:100C3000727374204761733F7D7D44656661756C96
:100C4000743A7D7D4D696E757465737D4D6F6E74FC
:100C50006820207D446179202020207D59656172C3
:100C60002020207D536574207D7D47617323207D86
:100C70005965737D43757272656E743A7D7D5365F7
:100C8000747570204D656E753A7D437573746F6D24
:100C90002046756E6374696F6E73497D4465636F3A
:100CA000747970653A7D5A482D4C3136204F437D1A
:100CB0004761756765202020207D47617567657DE8
:100CC0005A482D4C31362043437D41637469766523
:100CD000204761733F207D7D4761732053657475A4
:100CE00070202D204761736C6973747D4465707446
:100CF00068202B7D4465707468202D7D4261636B94
:100D00007D7D436F6E73742E2070704F322053655B
:100D10007475707D436F6E7374616E742070704F64
:100D2000322053657475707D5350237D4261747415
:100D300065727920496E666F7D7D4261747465725B
:100D40007920496E666F726D6174696F6E7D43794B
:100D5000636C65733A7D41706E6F657D4C61737431
:100D600020436F6D706C6574653A7D7D4C6F77655F
:100D700073742056626174743A7D4C6F7765737436
:100D80002061743A7D7D546D696E3A7D546D617851
:100D90003A7D536574204761737D4F32202B7D7DF2
:100DA0004F32202D7D7D4865202B7D7D4865202D8F
:100DB0007D7D457869747D7D44656C6574657D7D58
:100DC00044656275673A7D7D4F4E207D4F46467D76
:100DD00044656C2E20616C6C7D7D556E6578706508
:100DE000637465642072657365742066726F6D7DCF
:100DF000446976656D6F64652120506C656173652B
:100E00002068656C707D616E64207265706F7274AD
:100E100020746865204465627567207D496E666F41
:100E2000726D6174696F6E2062656C6F77217D7D74
:100E30004261696C6F75747D41706E6F6520202012
:100E4000207D44657363656E747D5375726661635E
:100E5000657D517569743F7D4D6F72657D7D436F12
:100E60006E6669726D3A7D7D4D656E7520323A7D94
:100E700043616E63656C7D7D4F4B217D53746F7054
:100E80007761742E7D7D4E4F54205553454421216A
:100E90002121217D4E4F54205553454421212121AC
:100EA000212121212121217D4E6F742075736564DC
:100EB000217D4E6F7420757365642121217D4C3135
:100EC000362D4746204F437D437573746F6D204622
:100ED000756E6374696F6E7349497D7D4746204C1A
:100EE0006F772020202020205B255D7D474620480D
:100EF00069676820202020205B255D7D436F6C6F33
:100F000072202342617474657279207D6E6F742043
:100F100075736564202020202020207D6E6F742052
:100F200075736564202020202020207D6E6F742042
:100F300075736564202020202020207D53686F7702
:100F400020736563732E205B3D315D7D6E6F742071
:100F500075736564202020202020207D6E6F742012
:100F600075736564202020202020207D4176722E1C
:100F7000204465707468205B3D315D7D6E6F742028
:100F800075736564202020202020207D6E6F7420E2
:100F900075736564202020202020207D6E6F7420D2
:100FA00075736564202020202020207D6E6F7420C2
:100FB00075736564202020202020207D6E6F7420B2
:100FC00075736564202020202020207D6E6F7420A2
:100FD00075736564202020202020207D6E6F742092
:100FE00075736564202020202020207D6E6F742082
:100FF00075736564202020202020207D6E6F742072
:1010000075736564202020202020207D6E6F742061
:1010100075736564202020202020207D6E6F742051
:1010200075736564202020202020207D6E6F742041
:1010300075736564202020202020207D6E6F742031
:1010400075736564202020202020207D6E6F742021
:1010500075736564202020202020207D6E6F742011
:1010600075736564202020202020207D6E6F742001
:1010700075736564202020202020207D6E6F7420F1
:1010800075736564202020202020207D6E6F7420E1
:1010900075736564202020202020207D6E6F7420D1
:1010A00075736564202020202020207D6E6F7420C1
:1010B00075736564202020202020207D6E6F7420B1
:1010C00075736564202020202020207D6E6F7420A1
:1010D00075736564202020202020207D4375737463
:1010E0006F6D2046756E6374696F6E732049497D1C
:1010F0004E6F742055736564212121212121217DAA
:101100004E6F7420557365642121212121212121F5
:10111000217D4E4F54205553454421212121217DCD
:1011200070704F32202B7D7D70704F32202D7D7D71
:1011300044696C2E7D7D4465636F747970653A20D7
:101140005A482D4C3136204F437D466F72204F70E8
:10115000656E20436972637569742020207D44693F
:10116000766572732E20537570706F7274732035AC
:10117000207D5472696D69782047617365732E20F4
:1011800020202020207D436F6E6669677572652080
:10119000796F757220676173207D696E2047617376
:1011A0007365747570206D656E752E20207D4368A3
:1011B00065636B204346313120262043463132207F
:1011C000217D4465636F747970653A204761756766
:1011D00065202020207D4469766574696D652077DF
:1011E000696C6C20626520696E7D4D696E757465F1
:1011F000733A5365636F6E64732E2020207D4F53C6
:101200005443322077696C6C206E6F74202020204C
:10121000207D636F6D70757465204465636F2C204D
:101220004E6F466C797D74696D6520616E642044F3
:10123000657361742E2D2020207D74696D65206199
:101240007420616C6C21202020202020207D4465AA
:10125000636F747970653A5A482D4C313620434398
:10126000207D466F72202853656D692D29436C6F70
:1012700073656420207D43697263756974207265AB
:101280006272656174686572737D436F6E666967CB
:10129000757265207468652033202020207D536599
:1012A00074506F696E747320696E2070704F322DA8
:1012B000207D5365747570206D656E752E20352008
:1012C0006261696C2D7D6F75742061726520617635
:1012D00061696C61626C652E207D4465636F747911
:1012E00070653A2041706E6F65202020207D4F533D
:1012F0005443322077696C6C20646973706C617937
:10130000207D656163682064657363656E74207316
:10131000657061722D7D6174656C7920696E204DF8
:10132000696E3A5365632E20207D57696C6C20747A
:10133000656D706F72616C6C79207365747D73611B
:101340006D706C657261746520746F2031207365F7
:10135000637D4E6F204465636F2063616C63756CC1
:101360006174696F6E7D4465636F747970653A204E
:101370004C31362D4746204F437D4465636F6D7079
:1013800072657373696F6E2063616C2D207D637568
:101390006C6174696F6E7320776974682074686516
:1013A000207D47462D4D6574686F64202847465F51
:1013B0006C6F2F47467D5F6869292E2043686563FF
:1013C0006B20434633322026207D43463333212091
:1013D0004F70656E2043697263756974207D77690B
:1013E000746820446565702053746F70732E2020DC
:1013F000207D4465636F747970653A204C31362DD9
:1014000047462043437D4465636F6D707265737317
:10141000696F6E2063616C2D207D63756C617469EA
:101420006F6E73207769746820746865207D474605
:101430002D4D6574686F64202847465F6C6F2F4799
:10144000467D5F6869292E20436865636B204346AB
:1014500033322026207D4346333321436C6F73653E
:101460006420436972637569747D77697468204488
:101470006565702053746F70732E2020207D446545
:10148000636F6D6F6465206368616E6765642120BA
:10149000207D4C31362D47462043437D4E6F7420CE
:1014A000666F756E647D536574506F696E747D7D73
:1014B0004E6F204465636F7D4772617068737D7DF8
:1014C000446973706C61797D4E6F206465636F7DD4
:1014D000536561726368206D6F64756C657D4578D6
:1014E00069747D7D52657365742043462C47617332
:1014F0002026204465636F7D44697361626C6520BA
:101500006D6F64756C657D7D53696D756C61746F0D
:10151000727D4F5354432053696D756C61746F72C3
:101520007D7D537461727420446976657D7D2B20C6
:10153000316D7D7D2D20316D7D7D2B31306D7D7D3B
:101540002D31306D7D7D457869747D7D6E6F7420A1
:101550007573657D787D4461746520666F726D6119
:10156000743A7D7D5365747570204D656E752032BB
:101570003A7D4D4D444459597D7D44444D4D595912
:101580007D7D59594D4D44447D7D4F535443207DBD
:101590004261696C7D7D41697220207D41697220C4
:1015A000207D43616C6962726174657D4D61782054
:1015B00044657074687D6E6F747D666F756E6421AE
:1015C0007D7D6D563A7D4E6577204346206164648B
:1015D0006564217D4E657720437573746F6D467524
:1015E0006E6374696F6E737D776572652061646484
:1015F00065642120436865636B7D43462049206113
:101600006E64204346204949204D656E757D666FA6
:10161000722044657461696C73217D7D53616C69CE
:101620006E6974793A7D426F74746F6D2054696D80
:10163000653A7D7D4D61782E2044657074683A7DF1
:1016400043616C63756C617465204465636F7D7D77
:1016500053686F77204465636F706C616E7D4C6575
:101660006164205469737D7D4C65616420546973A5
:101670007D7D53746F7077617463687D52657365A7
:1016800074204C6F67626F6F6B7D5265626F6F7411
:10169000204F5354437D5265736574204465636FD6
:1016A000646174617D7D2C8B01D81200278D05D873
:1016B000279D12002C8B01D812000B6F800EA66E96
:1016C000F86A020EF76EFC0EF66E0BC14CF1000EBE
:1016D0002CBB010E4D6F040E4E6F4F6BF0EC0BF0F8
:1016E0004851F6264951F7220900F55027BD02D08E
:1016F000E8CF7DF00900F55027BD02D0E8CF7CF09F
:101700000900F5500108E8CF7EF00900F5CF1BF184
:101710000D6B0E6BF66AF86A010EF76E01D02C9B0A
:101720000900F5500D27000E0E230B2FF9D72CBB07
:10173000F6D7F86AB00E0D25F66E070E0E21F76E7D
:1017400027AD20EE60F009007D0EF56201D00AD0D1
:10175000F550DE6E09007D0EF56201D003D0F55024
:10176000DE6EF1D727AD26EC0EF0120032C14CF13F
:1017700033C14DF13C0E4E6F4F6B4FD848C133F122
:101780004CC132F11200D89046334533472FFBD776
:101790001200D8904B334A3349334833472FF9D797
:1017A00012004951FF08496F4851D890FF08486F0F
:1017B00012001F975451525D506F55515359516F3C
:1017C000D8A812001F8750C154F151C155F1526978
:1017D00053695451525D506F55515359516F120016
:1017E0004A6B4B6B4C514E03F350486FF450496FAA
:1017F0004C514F03F3504927F4504A234D514E03A7
:10180000F3504927F4504A23D8B04B2B4D514F0386
:10181000F3504A27F4504B231200486B496B4E514A
:101820004F11D8B4FF0C010E476F4FBF05D0472BA7
:10183000D8904E374F37F9D7D890483749374E515F
:101840004C5F4F51D8A04F294D5FD8B005D04E51B5
:101850004C274F514D2301D048814707D8B412007F
:10186000D8904F334E33E8D7200E476F4B514D6F12
:101870004A514C6F4951536F4851526F4B6B4A6BF1
:10188000496B486B556B546BD890523753374C3774
:101890004D37543755374F51555DD8A452EF0CF0A2
:1018A0004E51545DD8A05CEF0CF04E51545FD8A05F
:1018B00055074F51555FD880483749374A374B371E
:1018C000472F44EF0CF01200D89075337433762F05
:1018D000FBD71200D8907A33793378337733762F69
:1018E000F9D712007851FF08786F7751D890FF0828
:1018F000776F12002A978351815D7F6F84518259DF
:10190000806FD8A812002A877FC183F180C184F13B
:10191000816982698351815D7F6F84518259806FB3
:101920001200796B7A6B7B517D03F350776FF45023
:10193000786F7B517E03F3507827F45079237C51E4
:101940007D03F3507827F4507923D8B07A2B7C515B
:101950007E03F3507927F4507A2312000A6FBAEF0E
:101960000CF000000000000000000000000000007B
:101970000000000000000000000000000000000067
:101980000000000000000000000000000000000057
:101990000000000000000000000000000000000047
:1019A0000000000000000000000000000A2FB1EF5E
:1019B0000CF01200096FE6EF0CF0000000000000D0
:1019C0000000000000000000000000000000000017
:1019D0000000000000000000000000000000000007
:1019E00000000000000000000000000000000000F7
:1019F00000000000000000000000000000000000E7
:101A0000000000000000630EAEEC0CF0092FDDEFCB
:101A10000CF01200630E3261326F32C134F1356B5B
:101A20001F950A0E3A6F366B67D8010E3A6F366B08
:101A30001F8562D8120032C134F1356B1F85F1D792
:101A400032C134F1356B1F95640E3A6F366B54D842
:101A5000E8D7259F376F1F8B372B372F1F9B238B83
:101A6000372B372F239B32C134F133C135F11F950A
:101A7000100E3A6F270E366F1FAD3ED8E80E3A6F44
:101A8000030E366F23BB07D025BF03D01F85372D2C
:101A90001F9523B91F851FAD2FD81F9D640E3A6F68
:101AA000366B27B924D023BB09D025BF03D01F85AF
:101AB000372D1F9523B91F8523BB1F851DD80A0EFF
:101AC0003A6F366B23BB09D025BF03D01F85372D56
:101AD0001F9523B91F8523BB1F8529B708D00CD8B4
:101AE000010E3A6F366B1F8524A506D824952799D9
:101AF000386B382B23991200396B3651355DD8A0DD
:101B00000ED004E13A51345DD8A009D03651355F8A
:101B10003A51345FD8A03507392B1F85EED7382FBF
:101B20001200382B300E39251FB504D01FBF04D04A
:101B3000200E01D0258FDE6E372F12002E0EDE6EA6
:101B400023891200A96E31D0A96E2BD02B91010EE2
:101B5000AA6E690E03D02691AA6A640EAD6E238F19
:101B6000040EA96E9D9A9E9A0FEC4AF049D8AECF0A
:101B7000A8FF01EC4AF026BF11D017D803EC4AF0B9
:101B8000A8CFADFF37D8A93EF1D711EC4AF09E9A05
:101B90009D8AAA6A269F239FF0EF47F0FF0EAD6E45
:101BA000F4D7A69EA69CA6801200A69EA69CA684FC
:101BB000F29E550EA76EAA0EA76EA682F28EA6B250
:101BC000FED7A6941200948C948E240EAC6E900EC8
:101BD000AB6E080EB86EB06A220EAF6EAE6A9E6A29
:101BE0009D8A1200AC6AAB6A9D9A949C949E829CDA
:101BF000829E1200ABAE12000000ACA2FBD7120016
:101C00009E9A269F436B446B9EBA12000000000010
:101C1000000000009EBA120000000000000000005A
:101C20009EBA120000000000000000009EBA1200E0
:101C300000000000000000009EBA1200442FE4D70C
:101C4000432FE1D7AB98AB88268F1200DE6A7BC0AA
:101C5000FAF17AC0F9F134EC5AF00101FAC17BF0E3
:101C6000F9C17AF01200106F10C17DF0210E2FD94A
:101C7000D8901035000ED8B0010E2ED9D89010355E
:101C80002BD912000F6F0FC17CF0200E20D9000E4F
:101C900023D90F5121D91200220E19D984807AC07C
:101CA00083FF809480847BC083FF80948084210E96
:101CB0000ED9D8901035000ED8B0010E0DD9D8909D
:101CC0001037102909D9200E02D9000E05D90F515D
:101CD00003D9220EFCD884807AC083FF809480844C
:101CE0007BC083FF809480841200220EF0D8848011
:101CF0007AC083FF809480847BC083FF809480843B
:101D00001200836A80968194809A8494809484924D
:101D10001200F45128EC10F0F5C11CF11C51B2DF97
:101D2000F75133EC0EF0E1DF1C2B1C51F663F6D7B4
:101D30001C51A8DFF75133EC0EF0D7DFF5C11CF1D1
:101D40001C51A0DFF85133EC0EF0CFDF1C2B1C51DF
:101D5000F663F6D71C5196DFF85133EC0EF0C5DF71
:101D6000F7C11CF11C517FDFF5518CDF95DF1C2B77
:101D70001C51F863F7D7F7C11CF11C5174DFF65101
:101D800081DF8ADF1C2B1C51F863F7D7FF0E28EC8C
:101D900010F01200F45128EC10F0350E98D8F7C16D
:101DA0001CF1D8901C35000ED8B0010E95D8D890F3
:101DB0001C3592D8360E8BD8F8C11CF1D8901C3542
:101DC000000ED8B0010E88D8D8901C3585D8370EB3
:101DD0007ED8F5C11CF11C517FD8F6C11CF11C51F5
:101DE0007BD8200E74D8000E77D8F5C11CF11C5199
:101DF00073D8210E6CD8F7C11CF1D8901C35000E99
:101E0000D8B0010E69D8D8901C3566D8220E5FD89C
:101E1000F5C11CF1F6C11DF11C511D5F1D2BF7C151
:101E20001CF1F8C11EF11C511E5F1E2B84801EC1C7
:101E30001CF17AC083FF809480847BC083FF8094F0
:101E400080847AC083FF809480847BC083FF8094E9
:101E500080841C2FEED71D2FEAD7000E38D8FF0E36
:101E600028EC10F01200350E32D8000E35D8000ED6
:101E700033D8360E2CD8010E2FD83F0E2DD8370E62
:101E800026D8000E29D8EF0E27D8200E20D8000E15
:101E900023D8000E21D8210E1AD8000E1DD8000E0E
:101EA0001BD8220E14D88480836A0A0E1E6F1E0E61
:101EB0001D6F1C6B80948084809480841C2FFAD7C3
:101EC0001D2FF7D71E2FF3D7000E01D812008490D4
:101ED000836E8094808412008480836E80948084DA
:101EE00012008096200EDAEC0CF081840000809ABB
:101EF000000084820A0EDAEC0CF0848400008492E4
:101F0000020EAEEC0CF084820A0EDAEC0CF0240E19
:101F1000DEDF020EDCDF000EDFDF000EDDDF030E92
:101F2000D6DF000ED9DF300ED7DF180ED0DF000E5F
:101F3000D3DF280ED1DFF80ECADF000ECDDF0F0E83
:101F4000CBDFF90EC4DF000EC7DF0F0EC5DF100EAA
:101F5000BEDF000EC1DF000EBFDF0CD884DF80863D
:101F6000200EDAEC0CF0050EB2DF000EB5DF010E2C
:101F7000B3DF1200700EABDF1F0EAEDF000EACDF62
:101F8000710EA5DF230EA8DF800EA6DF720E9FDF85
:101F90002A0EA2DF800EA0DF730E99DF150E9CDFE4
:101FA000110E9ADF740E93DF1C0E96DF110E94DF74
:101FB000750E8DDF1B0E90DF150E8EDF760E87DF20
:101FC0001A0E8ADF150E88DF770E81DF1C0E84DF84
:101FD000180E82DF780E7BDF210E7EDF150E7CDF90
:101FE0001200700E74DF140E77DF000E75DF710EB5
:101FF0006EDF170E71DF000E6FDF720E68DF150ED9
:102000006BDF800E69DF730E62DF150E65DF110E68
:1020100063DF740E5CDF140E5FDF0B0E5DDF750E89
:1020200056DF1B0E59DF150E57DF760E50DF130EED
:1020300053DF0E0E51DF770E4ADF1C0E4DDF180EF8
:102040004BDF780E44DF150E47DF0E0E45DF120022
:102050002E6F2EC12FF1030E2F17000E2F4F500E93
:102060002F4FA00E2F4FF80E306F2EC12FF11C0EE8
:102070002F172F432F43000E2F4F040E2F4F080E04
:102080002F4F0C0E2F4F100E2F4F140E2F4F200ED0
:102090002F4F3F0E316F31333033313330333133E3
:1020A00030332EC12FF12E6B31332E3331332E339B
:1020B00031332E33E00E2F172F432F432F432F435F
:1020C0002F43000E2F4F040E2F4F080E2F4F0C0ED4
:1020D0002F4F100E2F4F140E2F4F200E2F4F3F0E4D
:1020E000316F31332E3331332E3331332E3331339D
:1020F0002E3331332E332EC17AF030C17BF01200F3
:10210000E46F1F0EE46505D0010EAA6E200EE45F99
:1021100001D0AA6AE451040DF350820FA96ED1ECEC
:102120000DF0A850AA6A1200E46F1F0EE46505D0F6
:10213000010EAA6E200EE45F01D0AA6AE451040DDC
:10214000F350820FA96ED1EC0DF0A8CF32F1A92A7D
:10215000D1EC0DF0A8CF33F1AA6A12009A0EE36F0A
:102160002A8D010EAA6E04D0240EE36F2A9DAA6A5E
:102170001F8F33EC0FF0010EBA6F21992197209930
:10218000AA6BA56B229D229F23EC2AF0010EE8CFBB
:102190007FF02AAD04D0BA0E5DEC0BF003D01B0E1D
:1021A0005DEC0BF0000EE8CF7FF0B86B219121932E
:1021B000140EE8CF7DF0230EE8CF7CF020EE60F027
:1021C000AAC132F1000E2ABD200E322732C1DCF145
:1021D000386B382B376B1BEC0DF03A0EDE6E200E91
:1021E000DE6E26EC0EF0E351AA255DEC0BF01F0E1F
:1021F000DC5DD8B411D0260EDC5DD8B40DD0270E2E
:10220000DC5DD8B409D0280EDC5DD8B405D0290E29
:10221000DC5DD8B401D003D0010EDC6F01D0DC6BE3
:10222000140EE8CF7DF0410EE8CF7CF020EE60F098
:102230002B0EDE6E2F0EDE6E2D0EDE6E3A0EDE6E75
:10224000200EDE6E2B0E22BD2D0EDE6E26EC0EF065
:10225000140EE8CF7DF05F0EE8CF7CF020EE60F04A
:10226000310EDE6E2F0EDE6E310EDE6E300EDE6E45
:102270003A0EDE6E200EDE6E310EDE6E300E22BFA6
:10228000DE6E200EDE6E26EC0EF0140EE8CF7DF032
:102290007D0EE8CF7CF020EE60F0590E56EC0BF08E
:1022A000A551800FA96ED1EC0DF0A8CF32F1A55148
:1022B000810FA96ED1EC0DF0A8CF33F1339F386BAD
:1022C000382B376B375129EC0DF0280EDE6E310EAE
:1022D000A8AE380EDC67310EDE6E350EA8BEDE6E9F
:1022E000420EDE6E290EDE6E200EDE6E200EDE6EDB
:1022F000200EDE6E26EC0EF0140EE8CF7DF09B0E65
:10230000E8CF7CF020EE60F0610E56EC0BF0A551AA
:10231000820FA96ED1EC0DF0A8CF32F1A551830F39
:10232000A96ED1EC0DF0A8CF33F1386B382B376B99
:10233000375129EC0DF0200EDE6E200EDE6E200EE1
:10234000DE6E26EC0EF00B0E5DEC0BF0F9EC12F0ED
:102350002CEC1DF031EC2FF021B30FD021B11AD0AD
:1023600020B3F0EF47F020B152EC3BF020B1D3ECBA
:1023700040F0209120B91CD0EDD7BA2B070EBA63DC
:1023800002D0010EBA6FB86B2CEC1DF0F9EC12F014
:102390002193E0D7AA6A010E2ABDAA6EBA4F0FD0C8
:1023A000BA4F17D0BA4F19D0BA4F1BD0BA4F39D045
:1023B000020E2AAD010EBA6FAA6AAAEF13F0AA2B79
:1023C000AABBAA6BAA51040DF3CFA5F1010EBA6FF7
:1023D000ECD6227D020EBA6FE8D6227F030EBA6FCA
:1023E000E4D6A551800FA96ED1EC0DF0A8CF32F143
:1023F000A551810FA96ED1EC0DF0A8CF33F1339F19
:10240000A551820FA96E32C1A8FFD5EC0DF0A551E0
:10241000830FA96E33C1A8FFD5EC0DF0040EBA6F7F
:10242000C4D6A551820FA96ED1EC0DF0A8CF32F120
:10243000A551830FA96ED1EC0DF0A8CF33F1A551B2
:10244000810FA96ED1EC0DF0A8CFA6F1010EDC63CF
:1024500005D032673269322B336B16D022AD0BD0E8
:10246000010E22BF0A0E325F000EA6BF335B7F0E45
:1024700033BF336F09D0010E22BF0A0E3227000E80
:10248000A6BF332333BF336BA551820FA96E32C170
:10249000A8FFD5EC0DF0A551830FA96E33C1A8FF9D
:1024A000D5EC0DF0050EBA6F80D6E46F1F0EE46513
:1024B00005D0010EAA6E200EE45F01D0AA6AE45195
:1024C000040DF350800FA96ED1EC0DF0A8CF32F1BE
:1024D000A92AD1EC0DF0A8CF33F1AA6A1200CF4F90
:1024E00014D0CF4F19D01200CF4F0FD0CF4F14D0F0
:1024F000CF4F19D0CF4F1ED0CF4F23D0CF4F28D0A2
:10250000CF4F2FD0CF4F34D012000B0E3DD8BFECA1
:1025100012F0020ECF6F12000C0E49D8BFEC12F071
:10252000030ECF6F1200110E2FD8BFEC12F0040E65
:10253000CF6F1200120E3BD8BFEC12F0050ECF6F1A
:102540001200130E34D8BFEC12F0060ECF6F12003B
:10255000060ECF6F1D0E3ED8BFEC12F0070ECF6FE8
:102560001200200E24D8BFEC12F0080ECF6F12001C
:10257000210E1DD8BFEC12F0010ECF6F1200326F8A
:102580003267120077EF28F0396F94EC10F032C107
:1025900052F133C153F1395155EC12F032C154F1BB
:1025A00033C155F1D9EC0BF01FA7FF0C000C396FAC
:1025B00094EC10F032C154F133C155F1395155EC5E
:1025C00012F032C152F133C153F1D9EC0BF01FA715
:1025D000FF0C000C396F94EC10F032C154F133C190
:1025E00055F1CFC152F1536BD9EC0BF01FA7FF0C83
:1025F000000C280E2BA3C80EE56F050EDAEC0CF0CC
:1026000081B008D0E52FF9D781B006D02B8324877D
:102610002499120081A2F1D7249724992B930DECD1
:102620004AF012002B97010EBA6F1F9F33EC0FF088
:10263000B86B209921912193208F2187CDEC1DF03B
:102640002CEC1DF0249724993FEC13F021B124D0F9
:1026500020AFF0EF47F020B152EC3BF020B1D3ECCB
:1026600040F020B190EC3AF020B176EC45F02091AA
:1026700020B9F0EF47F020B3F0EF47F0E5D724A9F9
:1026800008D02183BA2B060EBA6518D0010EBA6F96
:1026900015D024B721811200BA4FE8EF2BF0BA4FC2
:1026A000A9EF33F0BA4F09EF15F0BA4FA7EF13F0C7
:1026B000BA4F64EF13F0BA4FF0EF47F0B86B21B7A1
:1026C0002CEC1DF024991200010EBA6F1F9F33EC01
:1026D0000FF0B86B209921912193208F21871EEC58
:1026E0001EF02CEC1DF0249724993FEC13F0050EFE
:1026F000BA6304D0060EBA6F2CEC1DF021B115D0D0
:1027000020AF90D720B152EC3BF020B1D3EC40F099
:1027100020B190EC3AF020B176EC45F0209120B950
:1027200081D720B3F0EF47F0E0D7BA4FACEF16F007
:10273000BA4F69EF31F0BA4F8BEF32F0BA4FF4EF86
:1027400048F0BA4FF4EF48F0050EBA6F6ED72B97EA
:10275000010EBA6F1F9F33EC0FF0EBEC1DF0B86B5E
:10276000209921912193208F2187F4EC13F098EC8C
:1027700014F02CEC1DF0249724993FEC13F021B1B8
:1027800017D020AFF0EF47F020B152EC3BF020B172
:10279000D3EC40F020B190EC3AF020B176EC45F06B
:1027A000209120B9F0EF47F020B3F0EF47F0E5D7E4
:1027B000BA4FB4EF10F0BA4FAEEF10F0BA4FA4D04A
:1027C000BA4F03D0BA4F5CD036D02B87220EA4EC80
:1027D0000DF0A82A060EA86201D0A86AD5EC0DF06B
:1027E000040EBA6F2499BBD7220EA4EC0DF0A86694
:1027F00004D0650E5DEC0BF01200A82E04D0660E1E
:102800005DEC0BF01200A82E04D0680E5DEC0BF00E
:102810001200A82E04D08A0E5DEC0BF01200A82E38
:1028200004D0980E5DEC0BF01200A82E1200EC0EF6
:102830005DEC0BF012002BA7F0EF47F033EC0FF03C
:1028400023EC2AF0010EE8CF7FF0EB0E5DEC0BF0ED
:10285000000EE8CF7FF0220EA4EC0DF0070EA802C8
:10286000F350C10FBA6F070E396FBA515DEC0BF020
:10287000BA2B392FFAD71E0E9DEC48F0F0EF47F037
:10288000010EBA6F1F9F33EC0FF009EC1EF0B86B0E
:10289000209921912193208F2187FAEC14F0D4EC18
:1028A00014F02CEC1DF0249724993FEC13F0030E48
:1028B000BA6304D0060EBA6F2CEC1DF021B117D00C
:1028C00020AFF0EF47F020B152EC3BF020B1D3EC59
:1028D00040F020B190EC3AF020B176EC45F0209138
:1028E00020B9A7EF13F020B3F0EF47F0DED7BA4FCF
:1028F0004CD0BA4F6CD0BA4F2AD7BA4F28D7BA4F5C
:1029000026D7050EBA6F26D71A0EA4EC0DF0A82A0A
:10291000630EA8640AD0690EA86007D01A0EA2EC54
:102920000DF0030EBA6F24991AD7640EA86EF6D76D
:102930001A0EA4EC0DF0630EA86421D8690EA860ED
:102940001ED85F0EE8CF7CF0530EE8CF7DF0000E6E
:10295000E8CF7EF020EE60F0A8CF32F1336B1F8F0E
:10296000030E29EC0DF01F9F6B0EDE6E670EDE6E00
:102970002F0EDE6E6C0EDE6E26EC0EF01200640E74
:10298000A86E1A0EA2EC0DF012005B0EA4EC0DF076
:10299000A82A020EA86401D0A86A5B0EA2EC0DF072
:1029A000010EBA6F249973D75B0EA4EC0DF0A866E4
:1029B00004D0030E5AEC0BF01200A82E04D0040E23
:1029C0005AEC0BF01200050E5AEC0BF01200270E19
:1029D000A4EC0DF0A82A010EA86401D0A86A270E65
:1029E000A2EC0DF02A85010EA8622A95020EBA6F9C
:1029F00024994DD7270EA4EC0DF0A86603D0830EC2
:102A00005DEC0BF0A806A866FED6820E5DEC0BF01E
:102A10001200010EBA6F33EC0FF039EC1EF0B86BF8
:102A2000209921912193208F218739EC1EF02CECE5
:102A30001DF0249724993FEC13F021B116D020AF5C
:102A4000F1D520B152EC3BF020B1D3EC40F020B1F5
:102A500090EC3AF020B176EC45F0209120B912EFDD
:102A600013F020B3F0EF47F0E6D7BA4F08D0BA4FD3
:102A70003AD0BA4F16D0BA4F05D0BA4F20D0030E75
:102A8000BA6FD3D5B7EC20F0BA6FBA6701D0F7D7D9
:102A900081EC0EF0000E9B6E7E0ED36EFF0000EFF9
:102AA00000F0B7EC20F0BA6FBA6701D0E8D733EC8A
:102AB0000FF0190E5DEC0BF085EC16F0E0D7B7ECDB
:102AC00020F0BA6FBA6701D0DAD733EC0FF0190EE5
:102AD0005DEC0BF08DC100F58EC101F520EC80F0AE
:102AE0000101F0EF47F0B7EC20F0BA6FBA6701D000
:102AF000C6D733EC0FF0190E5DEC0BF08DC100F56D
:102B00008EC101F520EC80F00101AA6A030EA96EC6
:102B1000336B150EE2D8150EE0D8150EDED8150E63
:102B2000DCD8150EDAD8150ED8D8010EA86E210EF5
:102B3000A2EC0DF0A86A220EA2EC0DF0A86A230EFA
:102B4000A2EC0DF0000EA86A270EA2EC0DF0A86A08
:102B50005A0EA2EC0DF0A86A5B0EA2EC0DF0640E0A
:102B60001A0EA2EC0DF01F0EA86E1B0EA2EC0DF0BB
:102B7000A86A1C0EA2EC0DF0A86A1D0EA2EC0DF0C6
:102B8000A86A1E0EA2EC0DF0A86A1F0EA2EC0DF0B2
:102B9000A86A200EA2EC0DF0640EA86E240EA2EC22
:102BA0000DF0250EA2EC0DF0260EA2EC0DF0010E9C
:102BB000CC6FCD6B7F0EA96E336B640E8ED81E0E5C
:102BC0008CD8F00E8AD8780E88D8050E86D8070ED5
:102BD00084D8040E336F338F880E7FD8040E336F82
:102BE000338F4C0E7AD8140E78D8140E76D81E0E69
:102BF00074D86E0E72D85A0E70D83C0E6ED8640E11
:102C00006CD8780E6AD80A0E68D8130E66D8A00E53
:102C100064D8960E62D80A0E60D8060E5ED8060EEC
:102C20005CD8000E5AD8000E58D80C0E56D8000E9C
:102C300054D8140E52D8336B338F000E4ED8030E77
:102C40004CD80A0E4AD8000E48D8010EAA6E7F0E44
:102C5000A96E336B1E0E41D85A0E3FD8DF0E3DD8F9
:102C60008C0E3BD8780E39D8000E37D8000E35D8E8
:102C7000000E33D8000E31D8000E2FD8000E2DD8FC
:102C8000000E2BD8000E29D8000E27D8000E25D80C
:102C9000000E23D8000E21D8000E1FD8000E1DD81C
:102CA000000E1BD8000E19D8000E17D8000E15D82C
:102CB000000E13D8000E11D8000E0FD8000E0DD83C
:102CC000000E0BD8000E09D8000E07D8000E05D84C
:102CD000000E03D8AA6AF0EF47F0326FA92A32C17A
:102CE000A8FFD5EC0DF0A92A33C1A8FFD5EC0DF053
:102CF000A92A32C1A8FFD5EC0DF0A92A339F33C110
:102D0000A8FFD5EC0DF0336B1200BD6BBE6B020E4D
:102D1000366F376B400E3A6F23933B693B51E6ECBD
:102D20002AF03A2FFAD7C5849CEC2BF0070EDAEC88
:102D30000CF0372FEFD7362FECD72393BD6BBE6B3C
:102D4000FD0EDAEC2AF0FD0EDAEC2AF0FE0EDAECDB
:102D50002AF0BD6BBE6B120033EC0FF02195219968
:102D60002197B86B2191219320992291229322954A
:102D7000BB6B23EC2AF0010EE8CF7FF01D0E5DEC5B
:102D80000BF0000EE8CF7FF0160E5DEC0BF0170E87
:102D90005DEC0BF0E6EC16F0180E5DEC0BF02497F2
:102DA000249924B7ABEC17F024B977EC17F021B9CC
:102DB00042D020B152EC3BF020B1D3EC40F0209156
:102DC00020B991D020B3F0EF47F0EBD7460EE8CF13
:102DD0007DF0410EE8CF7CF020EE60F005C132F1CD
:102DE000386B382B376B1BEC0DF03A0EDE6E04C1DE
:102DF00032F1386B382B376B1BEC0DF0200EDE6E8A
:102E0000200EDE6E26EC0EF0460EE8CF7DF05F0E53
:102E1000E8CF7CF020EE60F007C1F1F106C1F2F1DD
:102E200008C1F3F131EC23F0200EDE6E200EDE6ED1
:102E300026EC0EF0120007C132F1324F1F0E324F56
:102E40001C0E324F1F0E324F1E0E324F1F0E324FCE
:102E50001E0E324F1F0E324F1F0E324F1E0E324FBC
:102E60001F0E324F1E0E324F1F0E066502D0010E8E
:102E7000066F200EE8CF7DF09B0EE8CF7CF0080EA9
:102E8000396FA5EC1CF0050E0A6F036B209120A191
:102E9000FED7209104EC17F0460EE8CF7DF0410EEE
:102EA000E8CF7CF020EE60F005C132F1386B382BB2
:102EB000376B1BEC0DF03A0EDE6E04C132F1386B4D
:102EC000382B376B1BEC0DF03A0EDE6E03C132F17E
:102ED000386B382B376B1BEC0DF0200EDE6E26ECBA
:102EE0000EF00A2FD4D7010EBA6F66EF13F022B19D
:102EF0002189BB2BBBC1BCF1BC4F2185BC4F2285B6
:102F0000BC4F2283BC4F2281200EE8CF7DF09B0E68
:102F1000E8CF7CF020EE60F05E0E56EC0BF0BBC10B
:102F2000BCF1BC2F04D05A0E56EC0BF00FD0BC2FC6
:102F300004D05B0E56EC0BF009D0BC2F04D05C0E15
:102F400056EC0BF003D05D0E56EC0BF026EC0EF0B9
:102F5000F9EC12F012002499036B22B120D022B3B5
:102F600010D022B515D021B506D0052B170E05655A
:102F70001CD0056B1AD0042B3B0E046516D0046BD5
:102F800014D0062B1F0E066510D0010E066F0DD053
:102F9000072B0C0E076509D0010E076F06D0082B12
:102FA000140E086502D0080E086FE6EC16F0F9EC76
:102FB00012F012007C6B080E7B6F6CC17DF16DC14D
:102FC0007EF191EC0CF0100E7727270E782372C15A
:102FD00081F173C182F177C183F178C184F17AEC18
:102FE0000CF07FC185F180C186F12AB71ED02395F0
:102FF00085C17BF186C17CF185C17DF186C17EF101
:1030000091EC0CF0110E766F6AEC0CF085C181F139
:1030100086C182F177C183F178C184F17AEC0CF03A
:103020007FC187F180C188F117D0238585C17BF1ED
:1030300086C17CF185C17DF186C17EF191EC0CF0F9
:103040000F0E766F6AEC0CF0855177278651782346
:1030500077C187F178C188F16AC181F16BC182F1D2
:10306000FA0E836F846B7AEC0CF07FC17BF180C128
:103070007CF185C17DF186C17EF191EC0CF077C1C8
:1030800074F178C175F10C0E766F64EC0CF074C1BC
:1030900077F175C178F12AA70DD064517727655172
:1030A0007823100E7727270E782377C189F178C10E
:1030B0008AF10FD064C181F165C182F177C183F1DA
:1030C00078C184F17AEC0CF07FC177F180C178F19E
:1030D000E8D766C168F167C169F1C80E6827000EBC
:1030E000692368C17BF169C17CF185C17DF186C12D
:1030F0007EF191EC0CF077C174F178C175F10D0E91
:10310000766F64EC0CF074C18BF175C18CF162C107
:1031100074F163C175F1010E766F64EC0CF07451BB
:103120008B2775518C23B80E8B270B0E8C2370C107
:1031300081F171C182F189C183F18AC184F17AEC94
:103140000CF07FC17BF180C17CF18BC17DF18CC122
:103150007EF191EC0CF00C0E766F6AEC0CF02AB755
:1031600072EC0CF0E80E7727030E782377C18DF10F
:1031700078C18EF125AD04D0C6C18DF1C7C18EF1E5
:103180006EC168F16FC169F1640E6827000E692392
:1031900068C17BF169C17CF187C17DF188C17EF195
:1031A00091EC0CF00B0E766F6AEC0CF0249D23B5BD
:1031B00009D0C80E7727000E782377C197F178C120
:1031C00098F11200C80E816F826B77C183F178C1CC
:1031D00084F17AEC0CF02AB7248D7FC197F180C17D
:1031E00098F11200D4D8A00E3D6F0C0E586F08D97C
:1031F0001200E3D857C171F156C170F11200C7D85F
:10320000900EF2D7DAD857C173F156C172F112009D
:10321000238F596B000EA96E010EAA6ED1EC0DF032
:10322000AA6AC80EA864A8CF59F1B1D80D0E586F7C
:10323000540E3D6FE5D8C1D857C15BF156C15AF164
:103240000D0E586F580E3D6FDBD8B7D857C15DF1E2
:1032500056C15CF10D0E586F640E3D6FD1D8ADD8DC
:1032600057C15FF156C15EF10D0E586F680E3D6F8C
:10327000C7D8A3D857C161F156C160F15BC163F1F2
:10328000D8906333D8906333D89063335AC162F1D6
:10329000D8805BA1D8906233D8805BA3D89062338A
:1032A000D8805BA5D89062335CC164F1D8805DA101
:1032B000D8906433D8805DA3D8906433D8805DA55E
:1032C000D8906433D8805DA7D8906433D8805DA946
:1032D000D8906433D8805DABD89064335DC165F11C
:1032E000D8805AA1D8906533D8805AA3D890653336
:1032F000D8805AA5D8906533D8906533D890653377
:10330000D89065335FC166F1D8805EAFD8906637DC
:10331000D8805EADD8906637676B5FBF67835FBD4F
:10332000678161C16AF1D88060AFD8906A376B6BF2
:1033300061BF6B815EC16CF16C9D5CB16C8D6C9FEB
:103340005CB36C8F6D6B5CB56D815CB76D835CB984
:103350006D855CBB6D876F6B60C16EF16E9F239F47
:10336000120080820000808E00000000000000003B
:1033700000000000809E120080920000808E0000FD
:1033800000000000000000000000809E1200E9DF45
:10339000F3DFE7DFF1DFE5DFEFDFE3DFEDDFE1DFE5
:1033A000EBDFDFDFE9DFDDDFE7DFDBDFE5DFE4DF0A
:1033B000E3DFE2DFE1DFE0DF1200080E586F10D834
:1033C0003DC157F1080E586F0BD83DC156F1808EA4
:1033D000000000000000000000000000809E1200BD
:1033E000808E000000000000000000000000809EB1
:1033F00080A8D89080B8D8803D37582FF1D71200D8
:10340000809E8082030E585F808E000000000000C6
:10341000000000000000809E00000000000000008E
:1034200000000000808E000000000000000000008E
:103430000000809E0000000000000000000000006E
:10344000808E000000000000000000000000809E50
:103450003DAF80923DBF8082D8903D37808E000086
:1034600000000000000000000000809E582FF0D7F0
:103470001200DB6FD9C1DAF1D8C1D9F1D7C1D8F1C7
:10348000D6C1D7F1D5C1D6F1DBC1D5F12AA512003D
:10349000C80EE8CF7CF0640EE8CF7DF0000EE8CFD8
:1034A0007EF0000EE8CF7FF0FF0E28EC10F020EE4B
:1034B00060F0D551DE6ED651DE6ED751DE6ED8513A
:1034C000DE6ED951DE6EDA51DE6E200EDE6E26EC37
:1034D0000EF0120005EC4AF015EC4AF071EC0FF01A
:1034E00033EC0FF0FF0E28EC10F0850E5DEC0BF0C6
:1034F000860E5DEC0BF0870E5DEC0BF0880E5DEC3C
:103500000BF0640EE8CF7CF00A0EE8CF7DF0000EE1
:10351000E8CF7EF0000EE8CF7FF0FF0E28EC10F031
:1035200020EE60F0D551DE6ED651DE6ED751DE6EE4
:10353000D851DE6ED951DE6EDA51DE6E2E0EDE6EA1
:10354000200EDE6E1FC132F1386B382B376B20EC4A
:103550000DF0200EDE6E20C132F1386B382B376B48
:1035600020EC0DF026EC0EF07D0EE8CF7CF00A0E7C
:10357000E8CF7DF0000EE8CF7EF0000EE8CF7FF0C0
:10358000FF0E28EC10F020EE60F021C132F1386B14
:10359000382B376B20EC0DF0200EDE6E22C132F19D
:1035A000386B382B376B20EC0DF0200EDE6E23C10C
:1035B00032F1386B382B376B20EC0DF0200EDE6EBD
:1035C00024C132F1386B382B376B20EC0DF0200E14
:1035D000DE6E25C132F1386B382B376B20EC0DF0E5
:1035E00026EC0EF0960EE8CF7CF00A0EE8CF7DF0C8
:1035F000000EE8CF7EF0000EE8CF7FF0FF0E28EC43
:1036000010F020EE60F026C132F1386B382B376BAA
:1036100020EC0DF0200EDE6E27C132F1386B382B16
:10362000376B20EC0DF0200EDE6E28C132F1386BC6
:10363000382B376B20EC0DF0200EDE6E29C132F1F5
:10364000386B382B376B20EC0DF0200EDE6E2AC164
:1036500032F1386B382B376B20EC0DF026EC0EF086
:1036600024A7FED703EC4AF01200E00E28EC10F07D
:103670000B0E5AEC0BF0560E5DEC0BF0570E5DEC9A
:103680000BF0FF0E28EC10F01200000EE8CFF4F162
:103690003C0EE8CFF5F1EF0EE8CFF6F15A0EE8CF89
:1036A000F7F19F0EE8CFF8F1CAEC0EF0A4EC1EF093
:1036B00010EC1FF01200E9DFE00E28EC10F0540EC1
:1036C0005DEC0BF0FF0E28EC10F0080E396F910E38
:1036D000E8CF7CF0000EE8CF7DF0A5EC1CF01200E6
:1036E0002BB512007A0E39EC1AF0B90EE8CF7CF047
:1036F000770EE8CF7DF0010EE8CF7EF0000EE8CF28
:103700007FF0FF0E28EC10F020EE60F022C532F1C1
:10371000386B382B376B20EC0DF0270EDE6E26EC65
:103720000EF0000EE8CF7EF01200AFDFE00E28ECC6
:1037300010F0550E5DEC0BF0FF0E28EC10F01200AF
:103740002BB5120020BF34D0790E39EC1AF0E00E00
:1037500028EC10F0520E5DEC0BF0FF0E28EC10F090
:10376000760EE8CF7CF05E0EE8CF7DF0010EE8CF5C
:103770007EF0000EE8CF7FF0FF0E28EC10F020EE78
:1037800060F02BC532F1386B382B376B0AEC0DF03B
:103790006D0EDE6E24C532F1386B382B376B0AECB8
:1037A0000DF0270EDE6E26EC0EF0000EE8CF7EF058
:1037B0002BB51200780E39EC1AF0B90EE8CF7CF078
:1037C000770EE8CF7DF0010EE8CF7EF0000EE8CF57
:1037D0007FF0FF0E28EC10F020EE60F031C532F1E2
:1037E000C70E3261326F1F9F386B382B376B20EC5E
:1037F0000DF0270EDE6E26EC0EF032C532F1080E0B
:1038000080EC10F0326101D060D7770E39EC1AF0FD
:10381000910EE8CF7CF0000EE8CF7DF0000EE8CFEF
:103820007EF0FF0E28EC10F020EE60F0470EDE6E0A
:10383000460EDE6E3A0EDE6E32C532F1386B382B34
:10384000376B20EC0DF0250EDE6E200EDE6E26ECC2
:103850000EF01200410EE8CF7CF0690EE8CF7DF04B
:10386000000EE8CF7EF0FF0E28EC10F020EE60F0A6
:10387000EBC132F11F8F386B382B376B20EC0DF01A
:103880001F9F6D0EDE6E690EDE6E6E0EDE6E200EFA
:10389000DE6E26EC0EF05F0EE8CF7CF0640EE8CF13
:1038A0007DF0000EE8CF7EF0FF0E28EC10F020EE49
:1038B00060F0ECC132F11F8F386B382B376B20EC86
:1038C0000DF01F9F6D0EDE6E200EDE6E26EC0EF0EC
:1038D00012002BB51200760E39EC1AF05A0EE8CF12
:1038E0007CF0000EE8CF7DF0000EE8CF7EF0FF0EFA
:1038F00028EC10F020EE60F02D0E1FB72B0EDE6EC0
:1039000045C132F1386B382B376B0AEC0DF0530E92
:1039100056EC0BF026EC0EF02B891200080E396FD6
:103920005A0EE8CF7CF0000EE8CF7DF02B990DD039
:10393000060E396F020EE8CF7CF0730EE8CF7DF0F3
:1039400004D0010EE8CF7EF003D0000EE8CF7EF069
:1039500020EE60F0200EDE6E392FFCD726EC0EF044
:10396000000EE8CF7EF01200630E39EC1AF0320E32
:10397000E8CF7CF0000EE8CF7DF0000EE8CF7EF0BF
:10398000000EE8CF7FF0FF0E28EC10F020EE60F084
:1039900019C132F1326705D01AC132F1326701D054
:1039A00039D02DAF34D0B72F01D034D02D8F060EA3
:1039B000B76125D819C132F11AC133F1B6EC0BF059
:1039C000335132C133F1326F490EDE6E6E0EDE6E50
:1039D000740EDE6E3A0EDE6E386B382B376B1BECD6
:1039E0000DF03A0EDE6E33C132F1386B382B376B87
:1039F0001BEC0DF0200EDE6E26EC0EF012002D9F5B
:103A0000050EB76F12002D8F050EB76F1200B72F7E
:103A100001D0CCD72D9F060EB761F5DF05C132F17D
:103A2000386B382B376B1BEC0DF03A0EDE6E04C191
:103A300032F1386B382B376B1BEC0DF03A0EDE6E23
:103A400003C132F1386B382B376B1BEC0DF0200EB5
:103A5000DE6E26EC0EF01200230EE8CF7CF0000E96
:103A6000E8CF7DF0000EE8CF7EF0000EE8CF7FF0CB
:103A7000FF0E28EC10F020EE60F0B80EDE6E26ECA3
:103A80000EF0410EE8CF7CF0000EE8CF7DF0000E86
:103A9000E8CF7EF0000EE8CF7FF0FF0E28EC10F0AC
:103AA00020EE60F0B80EDE6E26EC0EF05F0EE8CF72
:103AB0007CF0000EE8CF7DF0000EE8CF7EF0000E27
:103AC000E8CF7FF0FF0E28EC10F020EE60F0B80E8B
:103AD000DE6E26EC0EF07D0EE8CF7CF0000EE8CF17
:103AE0007DF0000EE8CF7EF0000EE8CF7FF0FF0EF5
:103AF00028EC10F020EE60F0B80EDE6E26EC0EF032
:103B00009B0EE8CF7CF0000EE8CF7DF0000EE8CFF2
:103B10007EF0000EE8CF7FF0FF0E28EC10F020EED4
:103B200060F0B80EDE6E26EC0EF0B90EE8CF7CF039
:103B3000000EE8CF7DF0000EE8CF7EF0000EE8CF5B
:103B40007FF0FF0E28EC10F020EE60F0B80EDE6E75
:103B500026EC0EF0BAC139F1394F230E394F410E20
:103B6000394F5F0E394F7D0E394F9B0E394FB90ECD
:103B7000E8CF7CF0000EE8CF7DF0000EE8CF7EF0BD
:103B8000000EE8CF7FF0FF0E28EC10F020EE60F082
:103B9000B70EDE6E26EC0EF0120023EC2AF0010EBA
:103BA000E8CF7FF0050E5DEC0BF0000EE8CF7FF064
:103BB000060E5DEC0BF0070E5DEC0BF0090E5DECF4
:103BC0000BF00A0E5DEC0BF08E0E5DEC0BF00B0EA5
:103BD0005DEC0BF0120023EC2AF0010EE8CF7FF031
:103BE000620E5DEC0BF0000EE8CF7FF0630E5DEC33
:103BF0000BF0990E5DEC0BF0140E5AEC0BF0640E0A
:103C00005DEC0BF08E0E5DEC0BF00B0E5DEC0BF033
:103C1000120023EC2AF0010EE8CF7FF0020E5AECDE
:103C20000BF0000EE8CF7FF0010E5AEC0BF0810E86
:103C30005DEC0BF00B0E5DEC0BF0120023EC2AF0A8
:103C4000010EE8CF7FF0900E5DEC0BF0000EE8CF98
:103C50007FF0080E5DEC0BF06E0E5DEC0BF0710E5C
:103C60005DEC0BF0F70E5DEC0BF00B0E5DEC0BF06A
:103C7000120023EC2AF0010EE8CF7FF01C0E5DEC61
:103C80000BF0000EE8CF7FF0150E5DEC0BF0F50E9B
:103C90005DEC0BF01C0E5AEC0BF01D0E5AEC0BF009
:103CA0001E0E5AEC0BF00B0E5DEC0BF0120023EC29
:103CB0002AF0010EE8CF7FF0F80E5DEC0BF0000E5D
:103CC000E8CF7FF0F90E5DEC0BF0150E5AEC0BF01F
:103CD000160E5AEC0BF0170E5AEC0BF0180E5AECAD
:103CE0000BF00B0E5DEC0BF01200650E39EC1AF0C8
:103CF00097C199F198C19AF1640EE8CF7CF0000E5B
:103D0000E8CF7DF0000EE8CF7EF0000EE8CF7FF028
:103D1000FF0E28EC10F020EE60F02D0E24BDDE6EBC
:103D200097C132F198C133F1030E386F1F8F020E25
:103D300029EC0DF01F9FB00EDE6E430EDE6E200EDE
:103D4000DE6E26EC0EF012002BB51200750E39EC6B
:103D50001AF097C199F198C19AF1D80EE8CF7CF08A
:103D6000410EE8CF7DF0000EE8CF7EF0000EE8CFE8
:103D70007FF0FF0E28EC10F020EE60F02D0E24BD39
:103D8000DE6E97C132F198C133F1030E386F1F8F89
:103D9000020E29EC0DF01F9FB00EDE6E200EDE6EBF
:103DA00026EC0EF01200740E39EC1AF0780EE8CF03
:103DB0007CF0000EE8CF7DF0000EE8CF7EF0FF0E25
:103DC00028EC10F020EE60F0700EDE6E700EDE6EED
:103DD0004F0EDE6E320EDE6E3A0EDE6E48C132F1EE
:103DE00049C133F12987010E29EC0DF02997200EE6
:103DF000DE6E26EC0EF012000A0E396F780EE8CF58
:103E00007CF0000EE8CF7DF0A5EC1CF01200C00E97
:103E1000E8CF7CF0410EE8CF7DF0050E396F95D5E7
:103E20002ABB12002BB51200730E39EC1AF0C00E2B
:103E3000E8CF7CF0410EE8CF7DF0000EE8CF7EF0B9
:103E4000000EE8CF7FF0FF0E28EC10F0640E10C5D6
:103E500032F1D880325511C532F1D8803257090E6F
:103E600080EC10F011C533F1326501D005D0336715
:103E700003D0050E396F69D5150E32630AD033674A
:103E800008D020EE60F0080E53EC0BF026EC0EF09C
:103E9000120020EE60F01F8F386B382B376B20EC50
:103EA0000DF02F0EDE6E11C532F1386B382B376BEB
:103EB00020EC0DF0200EDE6E1F9F26EC0EF012009F
:103EC000550EE8CF7DF0000EE8CF7EF0000EE8CF73
:103ED0007FF0AA6A220EA4EC0DF0A86622D07D0E17
:103EE000E8CF7CF0FF0E28EC10F020EE60F04F0ED3
:103EF000DE6E26EC0EF0550EE8CF7DF0000EE8CF1A
:103F00007EF0000EE8CF7FF0960EE8CF7CF0FF0E3B
:103F100028EC10F020EE60F0430EDE6E26EC0EF082
:103F20001200A806A86601D01200A806A8662BD029
:103F30007D0EE8CF7CF0FF0E28EC10F020EE60F054
:103F4000430EDE6E550EE8CF7DF0000EE8CF7EF01A
:103F5000000EE8CF7FF026EC0EF0960EE8CF7CF056
:103F6000FF0E28EC10F020EE60F0430EDE6E550ED2
:103F7000E8CF7DF0000EE8CF7EF0000EE8CF7FF0B6
:103F800026EC0EF01200A806A86601D01200A806C2
:103F9000A8662BD07D0EE8CF7CF020EE60F0470EB7
:103FA000DE6E550EE8CF7DF0000EE8CF7EF0000EFD
:103FB000E8CF7FF0FF0E28EC10F026EC0EF0960E06
:103FC000E8CF7CF020EE60F0460EDE6E550EE8CFB6
:103FD0007DF0000EE8CF7EF0000EE8CF7FF0FF0E00
:103FE00028EC10F026EC0EF012007D0EE8CF7CF0ED
:103FF00020EE60F0470EDE6E550EE8CF7DF0000E2D
:10400000E8CF7EF0000EE8CF7FF0FF0E28EC10F036
:1040100026EC0EF0960EE8CF7CF020EE60F0460E17
:10402000DE6E550EE8CF7DF0000EE8CF7EF0000E7C
:10403000E8CF7FF0FF0E28EC10F026EC0EF0120017
:10404000710E39EC1AF02ABB120028BF120029A108
:1040500024D0870EE8CF7CF05A0EE8CF7DF0000E1A
:10406000E8CF7EF0000EE8CF7FF0FF0E28EC10F0D6
:1040700020EE60F0240EA4EC0DF0A8CF32F1336BEB
:10408000030E29EC0DF0420EDE6E610EDE6E720E36
:10409000DE6E1F9F26EC0EF058D0820EE8CF7CF02B
:1040A000640EE8CF7DF0010EE8CF7EF0000EE8CF81
:1040B0007FF0FF0E28EC10F0210EA4EC0DF0A8CF3D
:1040C000D1F1D105040DF350070FA96ED1EC0DF01D
:1040D000A8CF11F5D105040DF350060FA96ED1EC50
:1040E0000DF0A8CFD0F111C50AF1D880640E0A55A1
:1040F000D880A856A8CF10F5640E10C532F1D8802C
:10410000325511C532F1D880325711C533F1150E31
:10411000326306D0336704D0090E5AEC0BF015D089
:1041200020EE60F01F8F386B382B376B20EC0DF0D2
:104130002F0EDE6E11C532F1386B382B376B20EC49
:104140000DF01F9F26EC0EF000D0000EE8CFF4F12A
:104150007A0EE8CFF5F1AF0EE8CFF6F1520EE8CFC8
:10416000F7F19F0EE8CFF8F189EC0EF01200000E87
:10417000E8CFF4F1440EE8CFF5F1920EE8CFF6F176
:10418000220EE8CFF7F1650EE8CFF8F1CAEC0EF099
:10419000FF0EE8CFF4F1460EE8CFF5F1900EE8CF30
:1041A000F6F1230EE8CFF7F1640EE8CFF8F189ECD1
:1041B0000EF08F0E5DEC0BF0910E5DEC0BF0920E9D
:1041C0005DEC0BF0010EBA6F000EE8CFF4F1600E5B
:1041D000E8CFF5F18F0EE8CFF6F1270EE8CFF7F133
:1041E000330EE8CFF8F1CAEC0EF0BAC139F1600E27
:1041F000394F600E394F780EE8CF7CF0270EE8CFAC
:104200007DF0000EE8CF7EF0000EE8CF7FF0FF0ECD
:1042100028EC10F020EE60F0B70EDE6E26EC0EF00B
:1042200020992191219324992497B86B640EDAEC9C
:104230000CF031EC2FF021B315D021B10ED020B10C
:1042400052EC3BF020B1D3EC40F0209120B903D0E8
:1042500020B301D0EED7000C010CBA4FFCD7BA4FF7
:10426000FBD7F9D7BA2B030EBA6302D0010EBA6F8F
:10427000ABD7720E39EC1AF090C133F18FC132F125
:10428000A2EC2AF0270E336171D02BBBDDEC21F0BC
:104290002B9B20EE60F0030E536FE80E526F33C17C
:1042A00055F132C154F1542B000E5523D9EC0BF0CB
:1042B0001FA780D8180EE8CF7CF0000EE8CF7DF065
:1042C000020EE8CF7EF0000EE8CF7FF0FF0E28EC64
:1042D00010F0000E536F630E526F33C155F132C1AF
:1042E00054F1D9EC0BF01FA70AD01F8F2987386B28
:1042F000382B376B375129EC0DF01F9F02D0300E51
:10430000DE6E26EC0EF02997010EE8CF7EF0320E1D
:10431000E8CF7CF0280EE8CF7DF0FF0E28EC10F0FF
:1043200090C133F18FC132F1A2EC2AF020EE60F09F
:104330002E0EDE6E000E536F090E526F33C155F113
:1043400032C154F1D9EC0BF01FA707D0040E386F1F
:104350002485000E29EC0DF002D0300EDE6E26EC26
:104360000EF02495000EE8CF7EF012002BABDDECB2
:1043700021F020EE60F0180EE8CF7CF0000EE8CFC0
:104380007DF0020EE8CF7EF0000EE8CF7FF0FF0E4A
:1043900028EC10F029871F8F386B382B376B37517B
:1043A00029EC0DF01F9F26EC0EF02997000EE8CFA8
:1043B0007EF01200200EDE6E1200000EE8CFF4F147
:1043C000180EE8CFF5F15A0EE8CFF6F1000EE8CF5F
:1043D000F7F15A0EE8CFF8F1CAEC0EF02B8B120071
:1043E000680E39EC1AF0960EE8CF7CF0000EE8CF9C
:1043F0007DF0000EE8CF7EF0000EE8CF7FF0FF0EDC
:1044000028EC10F020EE60F00E0E56EC0BF0200EB3
:10441000DE6E20C532F121C533F1B6EC0BF01F8FF3
:10442000325133C132F1336F386B382B376B20EC9C
:104430000DF03A0EDE6E33C132F1386B382B376B2C
:104440001BEC0DF01F9F26EC0EF01200670E39ECEE
:104450001AF07D0EE8CF7CF0000EE8CF7DF0000E64
:10446000E8CF7EF0000EE8CF7FF0FF0E28EC10F0D2
:1044700020EE60F0230E56EC0BF0200EDE6ECCC169
:1044800032F1CDC133F1B6EC0BF01F8F325133C195
:1044900032F1336F386B382B376B20EC0DF03A0E5E
:1044A000DE6E33C132F1320732BF326B386B382BDC
:1044B000376B1BEC0DF01F9F26EC0EF0120020BD99
:1044C0001200620E39EC1AF0190EE8CF7CF0000EE3
:1044D000E8CF7DF0000EE8CF7EF0000EE8CF7FF051
:1044E000FF0E28EC10F020EE60F08DC132F18EC18D
:1044F00033F11F8F386B382B376B375129EC0DF0A8
:104500001F9F6D0EDE6E620EDE6E610EDE6E720E2F
:10451000DE6E200EDE6E26EC0EF01200660E39EC1A
:104520001AF01F0E80EC10F0326F010E326324D0AF
:10453000AF0EE8CF7CF0000EE8CF7DF0000EE8CFA4
:104540007EF0000EE8CF7FF0FF0E28EC10F020EE9A
:1045500060F0C2C132F1C3C133F1010E386F24855E
:104560001F8F020E29EC0DF01F9F560EDE6E200EDF
:10457000DE6E26EC0EF01200FF0EE8CFF4F1AE0E68
:10458000E8CFF5F1C20EE8CFF6F1000EE8CFF7F173
:104590001F0EE8CFF8F189EC0EF0100E526F0E0EE0
:1045A000536FC2C154F1C3C155F1D9EC0BF01FB721
:1045B00044D0B80E546F0B0E556FC2C152F1C3C137
:1045C00053F1D9EC0BF01FB735D050C14CF151C1AC
:1045D0004DF1140E4E6F4F6B0DEC0CF048C10AF10B
:1045E000020E0A650A6FFF0EE8CFF4F1B50EE8CFB0
:1045F000F5F1BB0EE8CFF6F11F0EE8CFF7F1210E73
:10460000E8CFF8F189EC0EF0220E80EC10F0E8CF44
:10461000F4F1AF0EE8CFF5F1C10EE8CFF6F1010EDF
:10462000E8CFF7F10AC1F8F1CAEC0EF0FF0E28EC62
:1046300010F01200010E0A6FD6D71E0E0A6FFF0E81
:10464000E8CFF4F1B50EE8CFF5F1BB0EE8CFF6F107
:104650001F0EE8CFF7F1210EE8CFF8F1CAEC0EF00B
:10466000D3D75B0EA4EC0DF0A8660ED0F1C132F1E9
:104670001F8F386B382B376B1BEC0DF01F9F2F0EE5
:10468000DE6EF2C132F112D05B0EA4EC0DF0A82E5A
:104690001FD0F2C132F11F8F386B382B376B1BECF8
:1046A0000DF01F9F2F0EDE6EF1C132F11F8F386BA0
:1046B000382B376B1BEC0DF01F9F2F0EDE6EF3C1F6
:1046C00032F11F8F386B382B376B1BEC0DF012005B
:1046D000F3C132F11F8F386B382B376B1BEC0DF0A9
:1046E0001F9F2F0EDE6EF1C132F11F8F386B382BFA
:1046F000376B1BEC0DF01F9F2F0EDE6EF2C132F1F7
:104700001F8F386B382B376B1BEC0DF012005B0ED4
:10471000A4EC0DF0A86615D0F1C132F11F8F386BF3
:10472000382B376B1BEC0DF01F9F2F0EDE6EF2C186
:1047300032F11F8F386B382B376B1BEC0DF01F9F3E
:1047400012005B0EA4EC0DF0A82EE6D7F2C132F1F8
:104750001F8F386B382B376B1BEC0DF01F9F2F0E04
:10476000DE6EF1C132F11F8F386B382B376B1BECCB
:104770000DF01F9F1200640E39EC1AF04B0EE8CFBB
:104780007CF0000EE8CF7DF0000EE8CF7EF0000E4A
:10479000E8CF7FF0FF0E28EC10F020EE60F007C1AC
:1047A000F1F106C1F2F108C1F3F131EC23F026EC8E
:1047B0000EF01200000EE8CFF4F1000EE8CFF5F194
:1047C0001A0EE8CFF6F1410EE8CFF7F1640EE8CF0C
:1047D000F8F1CAEC0EF012002BB51200700E39EC95
:1047E0001AF0B80EE8CF7CF0000EE8CF7DF0010E95
:1047F000E8CF7EF0000EE8CF7FF0FF0E28EC10F03F
:1048000020EE60F091C132F192C133F1A2EC2AF0B6
:104810001F8F2485030E29EC0DF01F9F1F9D26EC92
:104820000EF0000EE8CF7EF0120020BF1200410E05
:1048300039EC1AF028BF99D02ABB97D0260E80EC0D
:1048400010F0326F010E326301D08FD0A5C132F16A
:10485000A6C133F11F9F20EE60F0386B382B376B09
:104860001F8D375129EC0DF0140EE8CF7CF0780E37
:10487000E8CF7DF0010EE8CF7EF0FF0E28EC10F0BF
:1048800026EC0EF0000EE8CF7EF0120020BF1200E2
:10489000E00E28EC10F08C0E5DEC0BF0FF0E28EC17
:1048A00010F0550EE8CF7CF05A0EE8CF7DF0010EE7
:1048B000E8CF7EF0FF0E28EC10F0E1C132F11F9F2F
:1048C00020EE60F0386B382B376B20EC0DF03A0E91
:1048D000DE6EE2C132F1386B382B376B1BEC0DF01A
:1048E00026EC0EF0000EE8CF7EF01200000EE8CFAE
:1048F000F4F13C0EE8CFF5F1770EE8CFF6F15A0E61
:10490000E8CFF7F19F0EE8CFF8F1CAEC0EF01200F5
:10491000E00E28EC10F08B0E5DEC0BF0FF0E28EC97
:1049200010F0910EE8CF7CF05A0EE8CF7DF0010E2A
:10493000E8CF7EF0FF0E28EC10F0DCC132F120EE63
:1049400060F0386B382B376B20EC0DF03A0EDE6ED2
:10495000DDC132F1386B382B376B1BEC0DF026ECD8
:104960000EF0000EE8CF7EF01200A5C132F1A6C114
:1049700033F11F9F1F8D20EE60F0386B382B376BA3
:104980001F8D375129EC0DF03A0EDE6EA7C132F1C2
:10499000386B382B376B1BEC0DF0140EE8CF7CF026
:1049A0005A0EE8CF7DF0010EE8CF7EF0FF0E28EC26
:1049B00010F026EC0EF01F9D000EE8CF7EF01200E6
:1049C000000EE8CFF4F1360EE8CFF5F1660EE8CF31
:1049D000F6F13E0EE8CFF7F19F0EE8CFF8F1CAEC02
:1049E0000EF0120020BF1200560E39EC1AF0E00E45
:1049F00028EC10F01B0E5AEC0BF0FF0E28EC10F018
:104A0000500EE8CF7CF06E0EE8CF7DF0000EE8CFC0
:104A10007EF0FF0E28EC10F020EE60F017C132F1AE
:104A200018C133F1020E325F000E335BB6EC0BF0AF
:104A300032C10AF133C132F1336B000E1F9F1F8D5B
:104A4000386B382B376B1F8D375129EC0DF03A0E30
:104A5000DE6E0AC132F1386B382B376B1BEC0DF070
:104A60001F9F26EC0EF0550E39EC1AF0500EE8CFD1
:104A70007CF03E0EE8CF7DF0000EE8CF7EF0FF0E1A
:104A800028EC10F020EE60F093C132F194C133F1C4
:104A9000A2EC2AF01F8F2485030E29EC0DF01F9F36
:104AA0006D0EDE6E200EDE6E26EC0EF01200610E34
:104AB00039EC1AF0000EE8CF7CF0000EE8CF7DF064
:104AC000000EE8CF7EF0000EE8CF7FF0FF0E28EC5E
:104AD00010F020EE60F0060E53EC0BF0AA6AA96A03
:104AE000D1EC0DF0A8CF32F1A92AD1EC0DF0A8CF6E
:104AF00033F11F8F386B382B376B375129EC0DF0A2
:104B0000200EDE6E560EDE6E010E326F1F8F386B7A
:104B1000382B376B20EC0DF02E0EDE6E330E326F1D
:104B20001F8F386B382B376B1BEC0DF01F9F26EC5B
:104B30000EF012006F0E39EC1AF0DAEC23F01F0EB3
:104B40005DEC0BF029B107D0200E5DEC0BF07A0E76
:104B50005DEC0BF006D0EE0E5DEC0BF0890E5DEC1B
:104B60000BF0210E5DEC0BF0220E5DEC0BF0120051
:104B70006F0E39EC1AF0F00E5DEC0BF0F10E5DECFF
:104B80000BF0190E5AEC0BF0930E5DEC0BF0F40EDB
:104B90005DEC0BF01200640EE8CF7DF0000EE8CF64
:104BA0007CF0000EE8CF7EF0FF0E28EC10F020EE37
:104BB00060F0530EDE6E650EDE6E6C0EDE6E180E4D
:104BC000A4EC0DF0A8CF32F11F9F386B382B376B58
:104BD0000AEC0DF02F0EDE6E190EA4EC0DF0A8CF2E
:104BE00032F1386B382B376B0AEC0DF026EC0EF0F7
:104BF0007B0E5DEC0BF07C0E5DEC0BF07D0E5DEC46
:104C00000BF07E0E5DEC0BF01200FE0E5DEC0BF077
:104C1000FA0E5DEC0BF0FB0E5DEC0BF0FC0E5DECA8
:104C20000BF0FD0E5DEC0BF01200FF0EE8CFF4F17F
:104C30007CC0F5F17CC0F6F1140EF6277A0EE8CFB1
:104C4000F7F1322732078A0E3261326F32C1F8F142
:104C5000CAEC0EF0000EE8CFF4F17CC0F5F17CC098
:104C6000F6F1140EF62732C1F7F1F72B8B0EE8CFD1
:104C7000F8F1CAEC0EF01200000EE8CFF4F133C1E7
:104C8000F5F17D0EE8CFF6F1640EE8CFF7F19F0E57
:104C9000E8CFF8F1CAEC0EF012006E0E39EC1AF003
:104CA0002BC532F1326706D0CDEC27F0EF0E5DEC6C
:104CB0000BF012001F8F640EE8CF7DF0000EE8CFDE
:104CC0007CF0336F42EC0EF020EE60F02BC532F139
:104CD0003251D8B43CEF26F0386B382B376B20ECD0
:104CE0000DF06D0EDE6E26EC0EF08C0EE8CF7DF032
:104CF000000EE8CF7CF020EE60F024C532F1386B76
:104D0000382B376B1BEC0DF0270EDE6E26EC0EF009
:104D100015EC26F0640EE8CF7DF0190EE8CF7CF09C
:104D2000336F42EC0EF020EE60F02CC532F13251C0
:104D3000D8B43CEF26F0386B382B376B20EC0DF0F5
:104D40006D0EDE6E26EC0EF08C0EE8CF7DF0190EA7
:104D5000E8CF7CF020EE60F025C532F1386B382BBF
:104D6000376B1BEC0DF0270EDE6E26EC0EF015EC0B
:104D700026F0640EE8CF7DF0320EE8CF7CF0336F82
:104D800042EC0EF020EE60F02DC532F13251D8B475
:104D90003CEF26F0386B382B376B20EC0DF06D0EA6
:104DA000DE6E26EC0EF08C0EE8CF7DF0320EE8CFF2
:104DB0007CF020EE60F026C532F1386B382B376B73
:104DC0001BEC0DF0270EDE6E26EC0EF015EC26F037
:104DD000640EE8CF7DF04B0EE8CF7CF0336F42ECF1
:104DE0000EF020EE60F02EC532F13251D8B43CEF17
:104DF00026F0386B382B376B20EC0DF06D0EDE6E25
:104E000026EC0EF08C0EE8CF7DF04B0EE8CF7CF058
:104E100020EE60F027C532F1386B382B376B1BEC76
:104E20000DF0270EDE6E26EC0EF015EC26F0640E6B
:104E3000E8CF7DF0640EE8CF7CF0336F42EC0EF0EB
:104E400020EE60F02FC532F13251D8B43CEF26F09D
:104E5000386B382B376B20EC0DF06D0EDE6E26ECC8
:104E60000EF08C0EE8CF7DF0640EE8CF7CF020EEE3
:104E700060F028C532F1386B382B376B1BEC0DF026
:104E8000270EDE6E26EC0EF015EC26F012006D0EED
:104E900039EC1AF0640EE8CF7DF0000EE8CF7EF01A
:104EA0001F8F020E0A6FE70E096F336B332B040E50
:104EB0000A27190E0927640EE8CF7DF009C17CF09E
:104EC00020EE60F0470EDE6E33C132F1386B382BC6
:104ED000376B20EC0DF03A0EDE6E0AC1A9FFD1EC63
:104EE0000DF0A8CF32F1386B382B376B20EC0DF07A
:104EF0002F0EDE6EA92AD1EC0DF0A8CF32F1386B5F
:104F0000382B376B20EC0DF01B0EA4EC0DF033C1E9
:104F100032F1A832322FFDD70F0ED8A00A0E1B6F28
:104F200026EC0EF00F0E1B6F050E3363BFD7120079
:104F3000640EE8CF7DF0000EE8CF7EF01F8F230EC9
:104F40000A6FE70E096FE66B0A2BE62B190E09278D
:104F500009C17CF0640EE8CF7DF020EE60F0530EC6
:104F6000DE6E500EDE6EE6C132F1386B382B376BD9
:104F700020EC0DF03A0EDE6E0AC1A9FFD1EC0DF067
:104F8000A8CF32F1336B030E29EC0DF026EC0EF0B6
:104F9000030EE663D9D71F9F1200000EE8CFF4F18D
:104FA000000EE8CFF5F17D0EE8CFF6F1520EE8CF16
:104FB000F7F19F0EE8CFF8F1CAEC0EF012006C0E7C
:104FC00039EC1AF0000EE8CF7CF0550EE8CF7DF0FA
:104FD000000EE8CF7EF0000EE8CF7FF0FF0E28EC49
:104FE00010F020EE60F0B80EDE6E26EC0EF0190E1A
:104FF000E8CF7CF0550EE8CF7DF0000EE8CF7EF0D4
:10500000000EE8CF7FF0FF0E28EC10F020EE60F0ED
:10501000B80EDE6E26EC0EF0320EE8CF7CF0550EA8
:10502000E8CF7DF0000EE8CF7EF0000EE8CF7FF0F5
:10503000FF0E28EC10F020EE60F0B80EDE6E26ECCD
:105040000EF04B0EE8CF7CF0550EE8CF7DF0000E51
:10505000E8CF7EF0000EE8CF7FF0FF0E28EC10F0D6
:1050600020EE60F0B80EDE6E26EC0EF0640EE8CF97
:105070007CF0550EE8CF7DF0000EE8CF7EF0000EFC
:10508000E8CF7FF0FF0E28EC10F020EE60F0B80EB5
:10509000DE6E26EC0EF0BAC139F1000E394F000E6B
:1050A000394F190E394F320E394F4B0E394F640EAE
:1050B000E8CF7CF0550EE8CF7DF0000EE8CF7EF013
:1050C000000EE8CF7FF0FF0E28EC10F020EE60F02D
:1050D000B70EDE6E26EC0EF012007F0E5DEC0BF0CC
:1050E000800E5DEC0BF0840E5DEC0BF01200000EF8
:1050F000E8CFF4F1380EE8CFF5F1580EE8CFF6F12D
:10510000450EE8CFF7F1730EE8CFF8F1CAEC0EF0D8
:10511000FF0EE8CFF4F13A0EE8CFF5F1560EE8CFE6
:10512000F6F1460EE8CFF7F1720EE8CFF8F189EC10
:105130000EF03C0EE8CF7CF0470EE8CF7DF0000E7D
:10514000E8CF7EF0010EE8CF7FF0E00E28EC10F003
:1051500020EE60F0430EDE6E460EDE6E39C132F197
:10516000386B382B376B20EC0DF0210EDE6E26EC01
:105170000EF0000EE8CF7FF0FF0E28EC10F01200CA
:10518000680E39EC1AF0690E39EC1AF0FF0EE8CF10
:10519000F4F1190EE8CFF5F1780EE8CFF6F1520EE2
:1051A000E8CFF7F19F0EE8CFF8F189EC0EF025EE8D
:1051B00033F0100E0A6F096BFF0EE8CFF4F11C0EEE
:1051C0000925E8CFF5F11C0E0925E8CFF6F1092BEA
:1051D000092B640EE8CFF7F1DECFF8F1D890F83361
:1051E000D890F833640EF8279D0EF861F86FCAEC7A
:1051F0000EF00A2FE1D725EE43F0100E0A6F096B6F
:10520000FF0EE8CFF4F1560E0925E8CFF5F1560E62
:105210000925E8CFF6F1092B092B640EE8CFF7F149
:10522000DECFF8F1D890F833D890F833640EF82731
:105230009D0EF861F86FCAEC0EF00A2FE1D7540EFC
:10524000E8CF7DF0200EE8CF7CF0FF0E28EC10F0C8
:1052500020EE60F04E0EDE6E320EDE6E26EC0EF0AC
:10526000540EE8CF7DF05A0EE8CF7CF0FF0E28EC0C
:1052700010F020EE60F0480EDE6E650EDE6E26EC5D
:105280000EF0120023EC2AF0010EE8CF7FF0030E9F
:105290005DEC0BF0000EE8CF7FF0440E5DEC0BF000
:1052A000450E5DEC0BF0460E5DEC0BF0470E5DEC31
:1052B0000BF0480E5DEC0BF0490E5DEC0BF04A0E66
:1052C0005DEC0BF0120023EC2AF0010EE8CF7FF02A
:1052D000030E5DEC0BF0000EE8CF7FF04B0E5DECA3
:1052E0000BF04C0E5DEC0BF04D0E5DEC0BF04E0E2A
:1052F0005DEC0BF04F0E5DEC0BF0500E5DEC0BF027
:10530000510E5DEC0BF0120023EC2AF0010EE8CFF9
:105310007FF00F0E5AEC0BF0000EE8CF7FF0100E6E
:105320005AEC0BF0110E5AEC0BF0120E5AEC0BF07B
:10533000130E5AEC0BF012002BB5120020BF120016
:1053400020BD12006A0E39EC1AF0A80EE8CF7CF0EE
:10535000410EE8CF7DF0000EE8CF7EF0000EE8CFE2
:105360007FF0FF0E28EC10F020EE60F018C532F14F
:10537000326706D0070E53EC0BF026EC0EF012004D
:10538000336B1F8F030E29EC0DF01F9F26EC0EF0E0
:10539000120030EC80F001011A0E5AEC0BF020EEF6
:1053A00060F0230EDE6E63C532F163C50AF11F8F14
:1053B000386B382B376B20EC0DF0200EDE6E280E8C
:1053C000DE6E100E0A6105D04E0EDE6E320EDE6EFF
:1053D00004D0480EDE6E650EDE6E290EDE6E200EE7
:1053E000DE6E640EE8CF7DF0190EE8CF7CF0000E83
:1053F000E8CF7EF0FF0E28EC10F026EC0EF020EE49
:1054000060F015EE33F00A2BE6CF32F10A2FFCD70D
:10541000386B382B376B20EC0DF0250EDE6E200E2E
:10542000DE6E640EE8CF7DF0320EE8CF7CF0000E29
:10543000E8CF7EF0FF0E28EC10F026EC0EF01F9F58
:105440001200000E01D0FF0EE8CFF4F1000EE8CFFD
:10545000F5F11A0EE8CFF6F1000EE8CFF7F19F0E46
:10546000E8CFF8F1CAEC0EF012002BB5120028BFFD
:1054700012002ABB12002BB912006B0E39EC1AF085
:105480005A0EE8CF7CF0000EE8CF7DF0000EE8CF9A
:105490007EF0FF0E28EC10F020EE60F0430EDE6E82
:1054A0004E0EDE6E530EDE6E3A0EDE6E65C532F1C6
:1054B0001F8F386B382B376B20EC0DF01F9F250E9C
:1054C000DE6E26EC0EF01200400EA4EC0DF0010E84
:1054D000A8622BD0C80EE8CF7CF0000EE8CF7DF09C
:1054E000000EE8CF7EF0000EE8CF7FF0E00E28EC53
:1054F00010F020EE60F0400E326F180E336F322B3A
:1055000090EC2AF07D0EA86201D004D0A8CFDEFF77
:10551000332FF5D726EC0EF0FF0E28EC10F012001A
:1055200032C1A9FFD1EC0DF01200180E396FC80E70
:10553000E8CF7CF0000EE8CF7DF0A5EC1CF0120067
:105540001200120025BD12001A0EA4EC0DF0A8CF17
:105550000AF1690E0A611200630E0A65120032C177
:105560004CF133C14DF1640E4E6F4F6BF0EC0BF00C
:105570000AC14EF14F6B34EC0CF048C132F149C115
:1055800033F112003B6F010EBD27000EBE23BEAFEC
:1055900002D0BD6BBE6B3B2FF6D712003B6F010EE6
:1055A000BD5F000EBE5BBEAF02D07F0EBE6F3B2F55
:1055B000F6D712009CD8010EBD27000EBE23239102
:1055C000BEAF1200BD6BBE6B2381120023B31CD88B
:1055D00023A30BD82383000EBD2BBE232391BEAF84
:1055E0001200BD6BBE6B238112003B6FC580A4D837
:1055F000A60EC96EA1D894D8BEC1C9FF9DD890D8B7
:10560000BDC1C9FF99D88CD83BC1C9FF95D888D8EE
:1056100012003B6B3C6B229F229DC5848DD8C580B8
:105620008BD8A60EC96E88D8C5BCF7D73CC1C9FFB8
:1056300083D876D83BC1C9FF7FD872D8C5827CD8C1
:10564000A70EC96E79D86CD8C58676D822BD05D08C
:10565000228DFD0EC962229D11D022BF05D0228F5E
:10566000FD0EC96209D00AD0FE0EC96205D03BC149
:10567000BDF13CC1BEF10DD0229F229D010E3B2702
:10568000000E3C233CBF03D0C58856D8DDD7BD6B88
:10569000BE6BC58451D8229F229D1200C5844CD870
:1056A000C5804AD8A60EC96E47D8C5BCF7D7BEC1BB
:1056B000C9FF42D835D8BDC1C9FF3ED831D8C5824F
:1056C0003BD8A70EC96E38D82BD8C58635D8C95057
:1056D000C58432D81200E2DF010EBD27000EBE23C2
:1056E0002391BEAF1200BD6BBE6B238112003B6FD6
:1056F000C58022D8A60EC96E1FD812D8BEC1C9FF58
:105700001BD80ED8BDC1C9FF17D80AD83BC1C9FFE5
:1057100013D806D8C58410D8060EDAEC0CF01200A7
:10572000C5BC01D812004D0E39EC1AF001EC4AF05C
:105730000BD89E96C46B1200C42F01D0F4D79EA63E
:10574000FBD7C46B9E961200C66A4E0E39EC1AF057
:10575000C56AC76A949694888296090EC46F828639
:10576000000082B804D082968296C42FF8D794861F
:10577000C66A0A0EDAEC0CF0000EC76E280EC66E72
:10578000000EC56E080EC86E03EC4AF04F0E39ECE1
:105790001AF01200C56FC580CFDF900EC96ECCDF46
:1057A000BFDFC5C1C9FFC8DFBBDFC584C5DF1200CD
:1057B0009E96C580C1DF910EC96EBEDFB1DFC58682
:1057C000BBDFC9CFC5F1C588B7DFC584B5DF12001F
:1057D0002595299533EC0FF0259325972599BC6BDA
:1057E000BB6BC16B010EE8CF7FF00C0E5DEC0BF0D4
:1057F000000EE8CF7FF0A56BA66BA4EC2BF009ECB4
:105800002BF0396B3A6B050EBA6F010EE8CF7FF0C3
:105810000C0E5DEC0BF0000EE8CF7FF0229D229F76
:10582000010EA527000EA623A6BF27D0010ECEECA1
:105830002AF04EEC2BF022BD05D0228DFA0EC96263
:10584000229D10D022BF05D0228FFA0EC96207D840
:1058500009D0BDC1BFF1BEC1C0F1C12B13D0229F81
:10586000229D1200010E3927000E3A233ABF01D0C3
:10587000D7D725A912EF13F02CD0C151D8B4F9D73E
:10588000258327D0030EC2EC2AF025A704D0A75108
:10589000C163E1D264D025B31CD0F8DA050EBA6337
:1058A00016D0C1C1ACF1BFC1AAF1C0C1ABF1A5C155
:1058B00091F1A6C192F139C1F0F13AC1A8F1030EFC
:1058C000AA27000EAB23030E915F000E925BBA2F46
:1058D000C2D225A97DD723EC2AF0010EE8CF7FF0B4
:1058E0001A0E5DEC0BF0000EE8CF7FF00B0E5DECB6
:1058F0000BF0209921912193219724992497B86B3B
:10590000010E25B5AD51BA6F259525992CEC1DF0EA
:1059100031EC2FF021B3AAD221B10ED020B152EC3C
:105920003BF020B1D3EC40F0209120B912EF13F0FE
:1059300020B3F0EF47F0ECD72191060EBA6302D006
:1059400012EF13F0BAC1ADF12585BB51050DF3502F
:10595000BA25A76F33EC0FF02587C16B43D7259786
:1059600098EC1CF0000EE8CF7CF0000EE8CF7DF044
:1059700020EE60F0230EDE6E1C0E94EC10F0326709
:1059800003D0336701D016D0010E3227000E332327
:1059900032C152F133C153F1A7C154F1556BD9EC67
:1059A0000BF050C132F151C133F11F8F0A0E29ECB7
:1059B0000DF007D0A7C132F1386B382B376B1BECD9
:1059C0000DF0200EDE6E6BEC2BF0C9CF32F16BECDC
:1059D0002BF0C9CF32F1BDC1AFF1BEC1AEF1200E87
:1059E000C2EC2AF04EEC2BF0C9CFA9F1AFC1BDF14A
:1059F000AEC1BEF132C1F1F16BEC2BF0C9CFF2F1C7
:105A00006BEC2BF0C9CFF3F131EC23F0200EDE6EFE
:105A10006BEC2BF0C9CF32F1386B382B376B1BECAA
:105A20000DF03A0EDE6E6BEC2BF0C9CF32F1386B15
:105A3000382B376B1BEC0DF026EC0EF0190EE8CF6F
:105A40007CF0050EE8CF7DF020EE60F06BEC2BF0E3
:105A5000C9CF32F16BEC2BF0C9CF33F132C14CF12D
:105A600033C14DF1A40E4E6F4F6B0DEC0CF048C1DD
:105A7000C6F149C1C7F1C62B000EC7231F8F030E05
:105A800029EC0DF06D0EDE6E200EDE6E6BEC2BF051
:105A9000C9CF32F16BEC2BF0C9CF33F132C14CF1ED
:105AA00033C14DF13C0E4E6F4F6BF0EC0BF01F8F7E
:105AB000386B382B376B375129EC0DF0270EDE6E23
:105AC0006BEC2BF0C9CF32F132514827000E49233D
:105AD00048C14CF149C14DF19F0E4E6F4F6B0DEC1B
:105AE0000CF048C14CF149C14DF1A9514E6F4F6BBB
:105AF0000DEC0CF048C1C8F149C1C9F1C82B000E2A
:105B0000C9231F8F386B382B376B1BEC0DF0220E1F
:105B1000DE6E200EDE6E6BEC2BF0C9CF32F16BEC3B
:105B20002BF0C9CF33F1030E386F1F8F020E29EC13
:105B30000DF0B00EDE6E430EDE6E26EC0EF0320E71
:105B4000E8CF7CF0050EE8CF7DF020EE60F06BEC46
:105B50002BF0C9CF32F16BEC2BF0C9CF33F11F8F93
:105B6000386B382B376B375129EC0DF06D0EDE6E2C
:105B7000620EDE6E610EDE6E720EDE6E200EDE6E68
:105B8000440EDE6E650EDE6E730EDE6E610EDE6E30
:105B9000740EDE6E200EDE6E6BEC2BF0C9CF32F190
:105BA0006BEC2BF0C9CF33F1B6EC0BF01F8F3251F9
:105BB00033C132F1336F386B382B376B20EC0DF07B
:105BC0003A0EDE6E33C132F1386B382B376B1BEC7B
:105BD0000DF01F9F26EC0EF06BEC2BF06BEC2BF016
:105BE0006BEC2BF06BEC2BF06BEC2BF06BEC2BF0ED
:105BF0006BEC2BF06BEC2BF06BEC2BF06BEC2BF0DD
:105C00006BEC2BF06BEC2BF06BEC2BF06BEC2BF0CC
:105C10006BEC2BF06BEC2BF06BEC2BF06BEC2BF0BC
:105C20006BEC2BF0C9CFB1F1B199B19BB19DB19F94
:105C3000B12BB1C1EBF16BEC2BF0C9CFB2F1B29942
:105C4000B29BB29DB29FB2C1ECF16BEC2BF0C9CF0D
:105C5000B3F16BEC2BF0C9CFB4F16BEC2BF0C9CFE7
:105C6000B5F16BEC2BF0C9CFB6F16BEC2BF06BEC14
:105C70002BF0010EE8CFF4F14B0EE8CFF5F1EF0E6B
:105C8000E8CFF6F1000EE8CFF7F19F0EE8CFF8F17C
:105C9000CAEC0EF06BEC2BF0B86B6BEC2BF09E0E9D
:105CA000386F229F050EB96F4B0EDC6FB92933ECAC
:105CB0000EF0C8C1CAF1C9C1CBF1CB2B64D822BF49
:105CC00024D0C6C14EF1C7C14FF132C14CF133C12E
:105CD0004DF10DEC0CF04B0E48279EEC2EF048C118
:105CE000DCF1485142EC0EF0B92BB95133EC0EF017
:105CF000FF0E28EC10F04CEC0EF0CA4F02D043D847
:105D0000FCD7CB2FFAD7382FD4D7209921912193C4
:105D100024992497B86B31EC2FF021B179D021B3BD
:105D20001ED120B152EC3BF020B1D3EC40F02091D9
:105D300020B96ED020B3F0EF47F0EDD74851DC63C7
:105D400001D012004851DC650FD0DCC149F1490790
:105D5000495142EC0EF0FF0E28EC10F075EC0EF0FD
:105D600048514963F4D7120048C149F149074951E4
:105D700042EC0EF0FF0E28EC10F075EC0EF0DC514A
:105D80004963F4D712006BEC2BF0C9CF32F16BEC06
:105D90002BF0C9CF33F16BEC2BF0C9CFB8F1289BB6
:105DA000B8BF288BB89FFD0E326305D0FD0E33635C
:105DB00002D0228F1200B22F23D0ECC1B2F128AB57
:105DC00011D06BEC2BF0B807000EC9B8020FC9BA9E
:105DD000010FEF6FEF6701D005D06BEC2BF0B80728
:105DE000EF2FFBD7040EB86306D06BEC2BF0B8078F
:105DF0006BEC2BF0B8076BEC2BF0B82FFCD7120034
:105E0000B86701D012006BEC2BF0B82FFCD7120052
:105E10002099B86BAAC1BDF1ABC1BEF191C1A5F18A
:105E200092C1A6F1ACC1C1F1F0C139F1A8C13AF1FA
:105E3000C1072593BB07BC6B050EBA6FBB2B33ECB8
:105E40000FF0E3D425B3E9EF2BF0BC6B050EBA6F6E
:105E5000BB2B33EC0FF0BFC1BDF1C0C1BEF105EFEC
:105E60002CF024B9218324B721811200BA2B070E0C
:105E7000BA6301D0E7D7BC29BA6302D0060EBA6F65
:105E8000B86B2CEC1DF02499219342D52589BC2BAD
:105E900029B50CD023EC2AF0010EE8CF7FF01A0EC2
:105EA0005DEC0BF0000EE8CF7FF02985140EE8CFF3
:105EB0007DF0BB51050DF350C15D1E0DF350050F74
:105EC000E8CF7CF020EE60F0C1C132F1386B382BA6
:105ED000376B1BEC0DF0200EDE6E6BEC2BF0C9CF98
:105EE00032F10D0E326504D06BEC2BF0C9CF32F1DC
:105EF00032C1F1F16BEC2BF0C9CFF2F16BEC2BF06E
:105F0000C9CFF3F187EC23F06BEC2BF06BEC2BF0AB
:105F1000200EDE6E6BEC2BF0C9CF32F16BEC2BF068
:105F2000C9CF33F11F8F2485030E29EC0DF06D0EC0
:105F3000DE6E200EDE6E6BEC2BF0C9CF32F16BEC17
:105F40002BF0C9CF33F11F8F386B382B376B37519C
:105F500029EC0DF0270EDE6E26EC0EF01200010E7D
:105F6000BA6FCDEC27F06DEC28F0DFEC27F020992C
:105F70002191219324992497B86B31EC2FF021B310
:105F800015D021B10DD020B152EC3BF020B1D3ECB3
:105F900040F0209120B93CD720B3F0EF47F0EDD787
:105FA000BA4F36D7BA4F18D0BA4F07D0BA2B040E13
:105FB000BA6302D0010EBA6FD8D7B7EC20F0BA6F2F
:105FC000BA6701D025D733EC0FF00C0E5DEC0BF067
:105FD00085EC16F012EF13F0B7EC20F0BA6FBA6749
:105FE00001D016D733EC0FF00C0E5DEC0BF0010E68
:105FF000CEEC2AF0BDC1A5F1BEC1A6F1010EBF27AE
:10600000000EC023C0BFBF6BC0BFC06BA5C1BDF138
:10601000A6C1BEF14EEC2BF0C86FFE0EC86331D0A6
:10602000BFC1BDF1C0C1BEF1FE0E77EC2BF0010E79
:10603000BF27000EC023C0BFBF6BC0BFC06BBFC1B6
:10604000BDF1C0C1BEF1010EA527000EA623A6AF6B
:1060500002D0A56BA66BFF0E77EC2BF0010EC2EC05
:106060002AF0A5C152F1A6C153F1BDC154F1BEC180
:1060700055F1D9EC0BF05067EED75167ECD7E8EF4C
:106080002BF009EC2BF0020EC2EC2AF0BDC1C8F1D6
:10609000BEC1C9F1020ECEEC2AF0BDC1A5F1BEC150
:1060A000A6F1A5C1BDF1A6C1BEF14EEC2BF0BFC15A
:1060B000BDF1C0C1BEF177EC2BF0A5C1BDF1A6C109
:1060C000BEF1FF0E77EC2BF0010EA527000EA623E4
:1060D000A6BFA56BA6BFA66B010EBF27000EC023EF
:1060E000C0BFBF6BC0BFC06BA5C152F1A6C153F109
:1060F000C8C154F1C9C155F1D9EC0BF05067D1D7E3
:106100005167CFD7E8EF2BF02D939D9A0FEC4AF013
:1061100064EC49F06B0EAD6EFAEC0DF011EC4AF048
:106120009D8AD8EF39F028959D9A0FEC4AF020EC23
:1061300080F0010130EC80F0010118EC80F00101E9
:10614000010ECC6FCD6B680EAD6EFAEC0DF02085B4
:1061500011EC4AF09D8AD8EF39F028939D9A0FEC04
:106160004AF0AA6AAAD811EC4AF09D8AD8EF39F011
:106170002A9F9D9A0FEC4AF0010EAA6E9ED8AA6A39
:1061800011EC4AF09D8AD8EF39F0279F9D9A0FECC9
:106190004AF0FAEC0DF0010EAD6EFAEC0DF0330E94
:1061A000AD6E29EE4AF0100E396FFAEC0DF0DECF2D
:1061B000ADFF392FFAD711EC4AF09D8AD8EF39F0AC
:1061C000259B9D9A0FEC4AF033EC0FF023EC2AF05C
:1061D000010EE8CF7FF00F0E5DEC0BF0000EE8CF64
:1061E0007FF0050E436FAA0EAD6EFAEC0DF0432F53
:1061F000FAD7550EAD6E100E5DEC0BF009EC2BF0DE
:10620000010EBD27000EBE23110E5DEC0BF055D81C
:10621000FAEC0DF0C2C1ADFFFAEC0DF0C3C1ADFF59
:10622000FAEC0DF0010EAD6EFAEC0DF0330EAD6E22
:10623000120E5DEC0BF0436B446BC5809CEC2BF0B5
:10624000A60EC96E9CEC2BF0C5BCF7D7BEC1C9FF2A
:106250009CEC2BF090EC2BF0BDC1C9FF9CEC2BF01B
:1062600090EC2BF0C5829CEC2BF0A70EC96E9CEC39
:106270002BF090EC2BF0130E5DEC0BF0FAEC0DF024
:10628000C5869CEC2BF0C9CFADFF010E4327000E55
:10629000442344BF04D0C5889CEC2BF0EFD7C584C1
:1062A0009CEC2BF0140E5DEC0BF0FA0EDAEC0CF01B
:1062B00011EC4AF09D8A68EF39F0436BA96AD1EC82
:1062C0000DF0A8CFADFFA92AFAEC0DF0432FF7D7B8
:1062D0001200010EBA6F219921972099AA6B229D75
:1062E000229F33EC0FF023EC2AF0010EE8CF7FF071
:1062F0006F0E5DEC0BF0000EE8CF7FF0B86B2191D4
:106300002193140EE8CF7DF0230EE8CF7CF020EE31
:1063100060F0700E56EC0BF0AAC132F1322B1F8FD9
:10632000386B382B376B0AEC0DF0200EDE6E280E22
:10633000DE6EC00E56EC0BF0200EDE6E210EA4ECCD
:106340000DF0A8CFD1F1D105040DF350060FA96EC1
:10635000D1EC0DF0A8CF32F11F8F386B382B376B93
:106360000AEC0DF02F0EDE6ED105040DF350070F71
:10637000A96ED1EC0DF0A8CF32F11F8F386B382BFE
:10638000376B0AEC0DF0290EDE6E26EC0EF0140EC3
:10639000E8CF7DF0410EE8CF7CF020EE60F0610E9A
:1063A00056EC0BF0AA51240FA96ED1EC0DF0A8CF3A
:1063B00032F1336B1F8F030E29EC0DF01F9F420E3D
:1063C000DE6E610EDE6E720EDE6E200EDE6E26EC6E
:1063D0000EF0140EE8CF7DF05F0EE8CF7CF020EEDB
:1063E00060F0BE0E56EC0BF026EC0EF0140EE8CF6B
:1063F0007DF07D0EE8CF7CF020EE60F0BF0E56EC15
:106400000BF026EC0EF0140EE8CF7DF09B0EE8CFDB
:106410007CF020EE60F0590E56EC0BF0310EDE6E83
:106420002E0EDE6E300EDE6E300EDE6E26EC0EF0C0
:106430000B0E5DEC0BF0F9EC12F02CEC1DF031ECD6
:106440002FF021B30FD021B11ED020B3F0EF47F0D1
:1064500020B152EC3BF020B1D3EC40F0209120B9B8
:106460001CD0EDD7BA2B020EBA6301D0BA2B070E9F
:10647000BA6302D0010EBA6FB86B2CEC1DF0F9ECC8
:1064800012F02193DCD7BA4F3ED0BA4F0AD0BA4FA0
:1064900008D0BA4F1AD0BA4F2CD0020EBA6F66EF9E
:1064A00013F0AA51240FA96ED1EC0DF0A8CF32F150
:1064B000322BFB0E326302D0FA0E326F32C1A8FFCC
:1064C000D5EC0DF0030EBA6F19D7AA51240FA96E9F
:1064D000D1EC0DF0A8CF32F13207FF0E326302D0BB
:1064E000000E326F32C1A8FFD5EC0DF0040EBA6F6A
:1064F00005D7AA51240FA96E640EA86ED5EC0DF035
:10650000050EBA6FFBD6AA2B030EAA6301D0AA6BA5
:10651000010EBA6FF3D633EC0FF023EC2AF0010E24
:10652000E8CF7FF0720E5DEC0BF0000EE8CF7FF04D
:10653000230EE8CF7CF0000EE8CF7DF0000EE8CF10
:106540007EF020EE60F0730E56EC0BF0320EA4ECF1
:106550000DF0A8CF32F1330EA4EC0DF0A8CF33F13B
:106560001F8F386B382B376B375129EC0DF0200E0D
:10657000DE6E280EDE6E340EA4EC0DF0A8CF32F1E4
:10658000350EA4EC0DF0A8CF33F11F8F386B382BEC
:10659000376B375129EC0DF0290EDE6E26EC0EF02C
:1065A000410EE8CF7CF020EE60F0750E56EC0BF05B
:1065B0002F0EA4EC0DF0A8CFF1F1300EA4EC0DF0ED
:1065C000A8CFF2F1310EA4EC0DF0A8CFF3F131EC2D
:1065D00023F026EC0EF05F0EE8CF7CF020EE60F0AA
:1065E000760E56EC0BF0280EA4EC0DF0A8CF32F18D
:1065F000290EA4EC0DF0A8CF33F1010E386F1F8FD8
:10660000020E29EC0DF01F9F560EDE6E26EC0EF0EA
:106610007D0EE8CF7CF020EE60F0770E56EC0BF0AC
:106620002A0EA4EC0DF0A8CFF1F12B0EA4EC0DF086
:10663000A8CFF2F12C0EA4EC0DF0A8CFF3F131ECC1
:1066400023F026EC0EF09B0EE8CF7CF020EE60F0FD
:10665000780E56EC0BF0360EA4EC0DF0A8CF32F10C
:10666000370EA4EC0DF0A8CF33F1030E386F1F8F57
:10667000020E29EC0DF01F9FB00EDE6E200EDE6EB6
:10668000280EDE6E380EA4EC0DF0A8CFF1F1390E15
:10669000A4EC0DF0A8CFF2F13A0EA4EC0DF0A8CFC7
:1066A000F3F131EC23F0290EDE6E200EDE6E26ECC7
:1066B0000EF0B90EE8CF7CF020EE60F0790E56ECCB
:1066C0000BF03B0EA4EC0DF0A8CF32F13C0EA4EC85
:1066D0000DF0A8CF33F1030E386F1F8F020E29EC97
:1066E0000DF01F9FB00EDE6E200EDE6E280EDE6EE9
:1066F0003D0EA4EC0DF0A8CFF1F13E0EA4EC0DF090
:10670000A8CFF2F13F0EA4EC0DF0A8CFF3F131ECDD
:1067100023F0290EDE6E200EDE6E26EC0EF081A038
:10672000FED724972499219131EC2FF021B10DD07F
:1067300020B3F0EF47F020B152EC3BF020B1D3ECA6
:1067400040F0209120B901D0EFD7030EBA6F66EF69
:1067500013F0010EBA6F33EC0FF0B86B2099219152
:10676000219323EC2AF0010EE8CF7FF06A0E5DEC56
:106770000BF0000EE8CF7FF0AA6BA56B050E096F3A
:10678000020E0A6F140EE8CF7DF0040E0A271E0ECB
:1067900009270951E8CF7CF020EE60F0470EDE6E4D
:1067A000AAC132F1322B1F8F386B382B376B0AECB2
:1067B0000DF03A0EDE6EF6EC37F026EC0EF0280EF9
:1067C000E8CF7DF00951E8CF7CF020EE60F0210E9B
:1067D000A96ED1EC0DF0A804AA6302D02A0EDE6ED9
:1067E000F6EC37F026EC0EF0300EE8CF7DF00951D4
:1067F000E8CF7CF020EE60F00AC1A9FFA92AD1EC15
:106800000DF0A8CF32F13253000E32651AD0EFEC02
:1068100037F00AC1A9FFD1EC0DF0A8CF32F1386BE7
:10682000382B376B20EC0DF02F0EDE6EA92AD1EC41
:106830000DF0A8CF32F1386B382B376B20EC0DF010
:106840003FD00AC1A9FFD1EC0DF0A8CF32F13253ED
:10685000150E326517D0640E326108D0E8EC37F0BF
:10686000386B382B376B20EC0DF02AD04F0EDE6ED4
:10687000320EDE6E200EDE6E386B382B376B20EC5E
:106880000DF01ED0326353EC34F0410EDE6E490E33
:10689000DE6E520EDE6E200EDE6E386B382B376BDE
:1068A00020EC0DF00DD0450EDE6E520EDE6E520E57
:1068B000DE6E200EDE6E386B382B376B20EC0DF061
:1068C000F6EC37F026EC0EF0690EE8CF7DF00951BA
:1068D000E8CF7CF020EE60F0200EDE6E690EDE6EFA
:1068E0006E0EDE6E200EDE6EAA511C0FA96ED1EC6C
:1068F0000DF0A8CF32F1386B382B376B20EC0DF050
:106900006D0EDE6EF6EC37F026EC0EF0FF0E28EC86
:1069100010F0AA2B050EAA63C2EF33F00B0E5DEC4C
:106920000BF0F9EC12F02CEC1DF031EC2FF021B350
:106930000FD021B11ED020B3F0EF47F020B152ECC0
:106940003BF020B1D3EC40F0209120B90ED0EDD730
:10695000BA2B070EBA6302D0010EBA6FB86B2CECDB
:106960001DF0F9EC12F02193E0D7020EBA6F15EF8B
:1069700013F0BA4F09D0BA4F0CD0BA4F0FD0BA4F5C
:1069800012D0BA4F15D0F1D7000EAA6F000EA56F26
:1069900014D0010EAA6F040EA56F0FD0020EAA6FBD
:1069A000080EA56F0AD0030EAA6F0C0EA56F05D0B6
:1069B000040EAA6F100EA56F00D0010EBA6F2993B6
:1069C000219921972099229D33EC0FF01E0E5DEC4A
:1069D0000BF00B0E5DEC0BF0B86B219121934ADAB2
:1069E000410EE8CF7CF0140EE8CF7DF020EE60F091
:1069F0004F0EDE6E320EDE6E3A0EDE6E200EDE6E54
:106A0000A551060FA96ED1EC0DF0A8CF32F1386B6D
:106A1000382B376B20EC0DF0250EDE6E200EDE6E6F
:106A2000280EDE6E4D0EDE6E4F0EDE6E440EDE6EF6
:106A30003A0EDE6E120E80EC10F00A0DF3CF4CF120
:106A4000F4CF4DF1A551060FA96ED1EC0DF0A8CFF2
:106A50004EF14F6B0DEC0CF00A0E485F48C132F15D
:106A6000000E495B49C133F1386B382B376B375116
:106A700029EC0DF06D0EDE6E290EDE6E200EDE6E40
:106A8000200EDE6E26EC0EF05F0EE8CF7CF020EEDE
:106A900060F0480EDE6E650EDE6E3A0EDE6E200E83
:106AA000DE6EA551070FA96ED1EC0DF0A8CF32F123
:106AB000386B382B376B20EC0DF0250EDE6E200E78
:106AC000DE6E200EDE6E26EC0EF07D0EE8CF7CF042
:106AD00020EE60F02B0EDE6E2F0EDE6E2D0EDE6EC3
:106AE0003A0EDE6E200EDE6E2B0E22BD2D0EDE6EF9
:106AF00026EC0EF09B0EE8CF7CF020EE60F0590EF5
:106B000056EC0BF0A551040FA96ED1EC0DF0A8CFF7
:106B100032F1386B382B376B20EC0DF02F0EDE6E18
:106B2000A551050FA96ED1EC0DF0A8CF32F1386B4D
:106B3000382B376B20EC0DF0200EDE6E200EDE6E53
:106B400026EC0EF0F9EC12F02CEC1DF031EC2FF0ED
:106B500021B30FD021B11AD020B3F0EF47F020B10C
:106B600052EC3BF020B1D3EC40F0209120B918D08A
:106B7000EDD7BA2B070EBA6302D0010EBA6FB86B0D
:106B80002CEC1DF0F9EC12F02193E0D7BA4F90D025
:106B9000BA4F11D0BA4F43D0BA4F06D0BA4F69D0CE
:106BA000AAC1BAF1BA2BD7D5227D040EBA6F14D779
:106BB000010EBA6F09D7A551060FA96ED1EC0DF0E1
:106BC000A8CF32F122BD07D0322B650E326310D030
:106BD000040E326F0DD03207030E326309D0A55177
:106BE000070FA96ED1EC0DF0640E326FA850325F22
:106BF000A551070FA96ED1EC0DF0A8503225336FC7
:106C0000650E336302D0040E326FA551060FA96ED4
:106C100032C1A8FFD5EC0DF0020EBA6FDDD6A5513A
:106C2000070FA96ED1EC0DF0A8CF32F122BD06D02E
:106C3000322B5C0E326307D0326B05D03207FF0E69
:106C4000326301D0326BA551060FA96ED1EC0DF065
:106C5000A8503225336F650E336301D03207A5513A
:106C6000070FA96E32C1A8FFD5EC0DF0030EBA6F65
:106C7000B3D6A551040FA96ED1EC0DF0A8CF32F117
:106C8000A551050FA96ED1EC0DF0A8CF33F1A55198
:106C9000060FA96E32C1A8FFD5EC0DF0A551070F64
:106CA000A96E33C1A8FFD5EC0DF0050EBA6F94D6CE
:106CB00033EC0FF0010EBA6F6D0E5DEC0BF00B0EA6
:106CC0005DEC0BF0B86B21912193D4D89ED9410E85
:106CD000E8CF7CF0140EE8CF7DF020EE60F0690E76
:106CE00056EC0BF01B0EA4EC0DF0AAC132F1322BC6
:106CF000A832322FFDD7D8A004D0600E56EC0BF08E
:106D000006D0200EDE6E200EDE6E200EDE6E26EC2D
:106D10000EF05F0EE8CF7CF0140EE8CF7DF020EE91
:106D200060F0580E56EC0BF0200EDE6E210EA96EB0
:106D3000D1EC0DF0A804AA6304D0600E56EC0BF061
:106D400006D0200EDE6E200EDE6E200EDE6E26ECED
:106D50000EF07D0EE8CF7CF0140EE8CF7DF020EE33
:106D600060F06B0E56EC0BF026EC0EF09B0EE8CFAD
:106D70007CF0140EE8CF7DF020EE60F06C0E56EC47
:106D80000BF026EC0EF0F9EC12F02CEC1DF031ECCF
:106D90002FF021B30FD021B11AD020B3F0EF47F07C
:106DA00020B152EC3BF020B1D3EC40F0209120B95F
:106DB000F7D6EDD7BA2B070EBA6302D0010EBA6F21
:106DC000B86B2CEC1DF0F9EC12F02193E0D7BA4F20
:106DD000EFD6BA4F11D0BA4F05D0BA4F23D0BA4F21
:106DE00035D0DED6AAC1A8FFA82A210EA96ED5ECFF
:106DF0000DF0030EBA6F66D71B0EA4EC0DF0AAC1FE
:106E000032F1322B324FA870324FA872324FA87431
:106E1000324FA876324FA8781B0EA2EC0DF0020E6E
:106E2000BA6F50D7AA511C0FA96ED1EC0DF0A8CFA4
:106E300032F1322B640E326302D0630E326F32C1F4
:106E4000A8FFD5EC0DF0040EBA6F3CD7AA511C0F69
:106E5000A96ED1EC0DF0A8CF32F13207FF0E3263EC
:106E600002D0000E326F32C1A8FFD5EC0DF0050E36
:106E7000BA6F28D723EC2AF0010EE8CF7FF0020E7C
:106E8000E8CF7CF0000EE8CF7DF020EE60F05F0EE2
:106E900056EC0BF0AAC132F1322B1F8F386B382B16
:106EA000376B0AEC0DF03A0EDE6E200EDE6E26EC2D
:106EB0000EF0020EE8CF7CF0320EE8CF7DF020EE2F
:106EC00060F0A551070FA96ED1EC0DF0A8CF32F1FB
:106ED0003253000E32651DD0EFEC37F0A551060F8E
:106EE000A96ED1EC0DF0A8CF32F1386B382B376B8F
:106EF00020EC0DF02F0EDE6EA551070FA96ED1EC20
:106F00000DF0A8CF32F1386B382B376B20EC0DF039
:106F100041D0A551060FA96ED1EC0DF0A8CF32F1EA
:106F20003253150E3263326517D0640E326108D0C9
:106F3000E8EC37F0386B382B376B20EC0DF02AD0AB
:106F40004F0EDE6E320EDE6E200EDE6E386B382B8C
:106F5000376B20EC0DF01ED032630ED0410EDE6E8A
:106F6000490EDE6E520EDE6E200EDE6E386B382B52
:106F7000376B20EC0DF00ED0450EDE6E520EDE6E3D
:106F8000520EDE6E200EDE6E386B382B376B20EC27
:106F90000DF000D0200EDE6E690EDE6E6E0EDE6E1F
:106FA000200EDE6EAA511C0FA96ED1EC0DF0A8CFF9
:106FB00032F1386B382B376B20EC0DF06D0EDE6E36
:106FC000200EDE6E26EC0EF0000EE8CF7FF01200F1
:106FD0004E0EDE6E580EDE6E200EDE6E1200540E69
:106FE000DE6E580EDE6E200EDE6E12001B0EA4EC5E
:106FF0000DF0AAC132F1322BA832322FFDD7FF0E8D
:10700000D8A0490E28EC10F01200A551060FA96E69
:10701000D1EC0DF0A8CF33F1AA511C0FA96ED1EC21
:107020000DF0A8CF32F10A0E322733513203F3CFDD
:107030004CF1F4CF4DF10A0E4E6F4F6B0DEC0CF08E
:1070400048C132F149C133F1370EE8CF7DF0230E4C
:10705000E8CF7CF020EE60F0280EDE6E700EDE6E63
:10706000700EDE6E4F0EDE6E320EDE6E3A0EDE6E8D
:10707000030E29EC0DF0420EDE6E610EDE6E720E16
:10708000DE6E290EDE6E200EDE6E26EC0EF0120095
:1070900025BD1FD0AECF43F1600E435F434F258B1C
:1070A000434F248B434F258D434F2681434F278FDA
:1070B000434F2881434F2883434F2885434F2B81DB
:1070C000434F2A8F434F2D83AE509E9AAB98AB8887
:1070D00012002CB7F9D70FEC4AF0AE6601D0AE2AF9
:1070E000AE50640DF3CFC6F1F4CFC7F1EDD7F292F5
:1070F000D5BE09D02487D58E1200F090D5BE03D01E
:107100002489D58E1200F294D56AD76AD66AD58EB4
:107110001200F294D59ED76AD66A1200F19C2A9189
:10712000000ED56ED58E1200F18C1200F19A2A93C2
:10713000000ED56ED58E1200F18A1200A192B19E7A
:10714000CA9412009E9007EC4AF0080ECF60412BC3
:10715000080ECF5E412B0F0E416502D010EC39F0C6
:1071600020A901D0120023BF1200422B010E42635E
:107170000AD0239D3F6B406B9B6B9C6B02EC19F01C
:10718000F2EC18F01200020E42630FD0F9EC18F086
:10719000FFEC18F0DAEC17F08D513F278E514023A9
:1071A00097519B2798519C231200030E426301D0F4
:1071B000E5D7040E426301D0E9D7050E426301D042
:1071C000DDD7060E426301D0E1D7070E426301D03E
:1071D000D5D7DCDF426B020E3E6FD89040333F3391
:1071E000D8909C339B333E2FF8D740C18EF13FC1DE
:1071F0008DF19CC198F19BC197F1238D25AD04D0F1
:10720000E80E9F6F030EA06F1F979F518D5D8F6FCC
:10721000A0518E59906FD8A812008F6B906B1200FE
:10722000416B2081D89420A31CD0A82BA905A86568
:1072300002D0A86B2287172BD8B4182B22A911D003
:10724000A72B3B0EA76505D0A76B2087A52BD8B42D
:10725000A62B2AAB06D0DD2B3B0EDD6502D0DD6B05
:10726000DC2B032B3B0E03651200036B2085042BE4
:107270003B0E04651200046B052B170E056512000A
:10728000056B062B07C176F1764F1F0E764F1C0E4D
:10729000764F1F0E764F1E0E764F1F0E764F1E0E28
:1072A000764F1F0E764F1F0E764F1E0E764F1F0E17
:1072B000764F1E0E764F1F0E06651200010E066FEA
:1072C000072B0C0E07651200010E076F082B12002A
:1072D0004AEC48F0326B32C118F5BAEC0FF0A4EC6E
:1072E0002BF0E3EC0DF071EC0FF057EC25F0B4EC63
:1072F0001CF0BBEC23F0A3C100F5A4C101F5A3C1B0
:1073000002F5A4C103F528BF0CD02ABB0AD0F0ECCB
:1073100021F026EC22F0C3EC28F020EC20F060EC09
:107320001FF028AF03D0670E5DEC0BF02AAB03D043
:10733000740E5DEC0BF0B86BB96B209D209F239D04
:10734000956B966B996B9A6B050EB76F11EC4AF0C3
:1073500003EC4AF0259D2C97000EE8CF7CF0000E40
:10736000E8CF7DF0000EE8CF7EF0000EE8CF7FF092
:10737000FF0E28EC10F02497249964EC2AF0010EFB
:10738000CF6F470E39EC1AF00C0E80EC10F00A6F3C
:107390000AC113F50B0E80EC10F00A6F0AC112F54A
:1073A00030EC80F00101480E39EC1AF0F9EC12F0E3
:1073B00020A11BD029A101D000D0B4EC1CF090EC8E
:1073C0003AF052EC3BF076EC45F08EEC22F01AEC01
:1073D0003BF063EC3AF074EC12F020EC20F060EC3F
:1073E0001FF02CB148EF45F0209133EC3BF023BD6A
:1073F0005FEC22F023BD75EC1EF023BDD3EC40F012
:10740000239D20B52CEC3AF020BF12EF13F020B3EF
:107410005EEF3BF020B98BEF44F025BBE0EF30F09E
:1074200024BBF2EF46F026B1ABEF0DF02BB1A6EF87
:107430000DF027BFC5EF30F028B148EF47F028B373
:10744000ADEF30F028B593EF30F02ABFB8EF30F051
:107450002DB384EF30F0ACD7BBEC23F067EC3AF0FF
:107460009BEC46F064EC2AF053EC3AF028BF09D0CC
:107470002ABB07D026EC22F0F0EC21F020ADC3ECC3
:1074800028F045EC3AF0209512002781010ECC5FE0
:10749000000ECD5BCC671200CD671200279115EC72
:1074A0004AF0CC2B120020C532F121C533F13267EE
:1074B00005D0336703D0196B1A6B1200010E192720
:1074C000000E1A23120027B117EC4AF012000BEC41
:1074D0004AF0490E39EC1AF09FC102F5A0C103F53C
:1074E0000A6B0AC111F54F0E0A6F0AC110F58DC162
:1074F00000F58EC101F50B0E80EC10F00A6F0AC189
:1075000012F50C0E80EC10F00A6F0AC113F540EC76
:1075100080F001014A0E39EC1AF00DEC4AF012002D
:1075200094928282249182A42481829294820A0E6F
:10753000AEEC0CF0249382A424839492829224B122
:1075400074D024B364D0948229A944D0299F299966
:10755000320EA4EC0DF0A8CF39F1330EA4EC0DF0EF
:10756000A8CF3AF1D890010E3927000E3A2339C13D
:10757000A8FF320EA2EC0DF03AC1A8FF330EA2EC28
:107580000DF0340EA4EC0DF0A8CF39F1350EA4ECBB
:107590000DF0A8CF3AF1D890010E3927000E3A230A
:1075A00039C1A8FF340EA2EC0DF03AC1A8FF350E88
:1075B000A2EC0DF007C1A8FF2F0EA2EC0DF006C142
:1075C000A8FF300EA2EC0DF008C1A8FF310EA2EC0E
:1075D0000DF0120029AF1200299F320EA4EC0DF01D
:1075E000A8CF39F1330EA4EC0DF0A8CF3AF1D89022
:1075F000010E3927000E3A2339C1A8FF320EA2EC42
:107600000DF03AC1A8FF330EA2EC0DF0120005EC0C
:107610004AF0640EDAEC0CF007EC4AF0640EDAEC97
:107620000CF005EC4AF02989120005EC4AF0298F8C
:107630002999120020AD1200B92B040E80EC10F035
:10764000B9651200209D21EC2AF028BF04D02ABB86
:1076500002D0C3EC28F05FEC22F057EC25F0B96BB8
:1076600024972499120024B718D024B907D0D59EA6
:10767000F294D76AD66AF292F0901200249923EC21
:107680002AF0010EE8CF7FF0040E5DEC0BF0000E47
:10769000E8CF7FF0208DB86B1200249720AD120048
:1076A000208F1200B82B030E80EC10F0050FD8B01D
:1076B000FF0EE806B8651200208912001EEC41F0AA
:1076C000520E39EC1AF033EC0FF035EC1BF010ECE5
:1076D0001FF0A4EC1EF02ABB208728BF04D02ABBD1
:1076E00002D05BEC1BF020A13FD028BF09D02ABB01
:1076F00017D029B118D06DEC3EF037EC3CF018D023
:1077000020AD15EC24F061EC40F02CB3F2EC24F049
:1077100024BF04D0248FF9EC40F00AD0249F08D075
:10772000E4EC3BF005D09CEC29F037EC3CF000D0C9
:1077300061EC40F023B78EEC22F020BDDAEC3BF098
:1077400020BF3FEC44F014EC3CF02CB148EF45F086
:107750002CB3F2EC24F02091260E80EC10F0326F66
:10776000010E326301D0268326A30BD020BD08D0A2
:1077700015EC24F029B19CEC29F027B56DEC3EF016
:10778000269320AFD6EC41F020BF1BEC42F020A3A3
:1077900032D323BD86EC40F0239D20B5A5EC40F00C
:1077A00022B752EC3DF020BF04D025BD02D003002B
:1077B000000099D7B92B040E80EC10F0B9651200C7
:1077C000209DDAEC23F0120088EC24F022B90DD0D1
:1077D00046EC24F0E22B3C0EE26302D0E26BE12B9C
:1077E000269722B912002687120026A712000BD86E
:1077F00076EC24F0E06BE26BE16BDD6BDC6B916BA4
:10780000926B26971200DEC152F1DFC153F191C194
:1078100054F192C155F1D9EC0BF01FA7120091C1A0
:10782000DEF192C1DFF1120003EC4AF032C532F111
:107830000E0E80EC10F0326131EC3CF027BB01EC15
:107840004AF01FC532F1322D120066C532F10E0E1C
:1078500080EC10F0326131EC3CF027BB01EC4AF0D7
:10786000120001EC4AF0020EB06F288B120024BF08
:10787000CDD0248FF9EC40F038EC3EF08DC14CF1C6
:107880008EC14DF10A0E4E6F000E4F6B0DEC0CF0D9
:1078900048C14CF149C14DF1D0C14EF14F6BF0ECF4
:1078A0000BF048C14CF149C14DF1640E4E6F000E12
:1078B0004F6B0DEC0CF048C107F529B118C507F561
:1078C00028EC80F0010165C532F11B0E80EC10F050
:1078D000325DD8B035EC2AF025A18DD08FC14CF1A6
:1078E00090C14DF1640E4E6F4F6B0DEC0CF0326B8E
:1078F0001B0EA4EC0DF0A8A00AD01C0EA4EC0DF0F9
:107900004851A86004D0A8CF32F1010E336F1B0E8E
:10791000A4EC0DF0A8A210D01D0EA4EC0DF048515F
:10792000A8600AD01D0EA4EC0DF03251A86404D05A
:10793000A8CF32F1020E336F1B0EA4EC0DF0A8A4F9
:1079400010D01E0EA4EC0DF04851A8600AD01E0EF7
:10795000A4EC0DF03251A86404D0A8CF32F1030E8C
:10796000336F1B0EA4EC0DF0A8A610D01F0EA4ECD4
:107970000DF04851A8600AD01F0EA4EC0DF0325152
:10798000A86404D0A8CF32F1040E336F1B0EA4EC10
:107990000DF0A8A810D0200EA4EC0DF04851A8605E
:1079A0000AD0200EA4EC0DF03251A86404D0A8CF68
:1079B00032F1050E336F450E39EC1AF0330732C140
:1079C0001BF53351040DF350070FA96ED1EC0DF0E8
:1079D000A8CF1DF53351040DF350060FA96ED1EC5D
:1079E0000DF01DC50AF1D880640E0A55D880A8563E
:1079F000A8CF1CF50AD0460E39EC1AF0326B32C112
:107A00001BF532C11CF532C11DF51200249F28BFA1
:107A100012002ABB1200420E39EC1AF028EC3DF09D
:107A200000EC80F00101430E39EC1AF023C5CEF1D1
:107A3000CE6712002BC50AF10A6729D025B15BEC8D
:107A40001BF02591AA6B22C5ABF170EC1BF0120064
:107A50008DC100F58EC101F50B0E80EC10F00A6FA0
:107A60000AC112F50C0E80EC10F00A6F0AC113F572
:107A7000100E80EC10F00A6F0AC117F51D0E80EC95
:107A800010F00A6F0AC11EF54AEC48F0120025A159
:107A900095EC1BF025812BC5AAF124C5ABF1A0EC18
:107AA0001BF01200229726830DEC4AF022BB08D06F
:107AB000228BBDC1BFF1BEC1C0F12F0EC2EC2AF0B6
:107AC0008F51DAEC2AF09051DAEC2AF0AE6BB12D3E
:107AD00002D0020EAE27B22D02D0020EAE27B32D79
:107AE00002D0020EAE27B42D02D0030EAE27B52D64
:107AF00002D0090EAE27B62D02D0000EAE2728AB5D
:107B000011D0010EAE27AF6BB051AF27B06B28A7D5
:107B100003D0020EAE27AF8928A903D0010EAE27ED
:107B2000AF8BAE8FAE51DAEC2AF028AB16D0AF5146
:107B3000DAEC2AF028A70CD0180EA4EC0DF0A8500F
:107B4000DAEC2AF0190EA4EC0DF0A850DAEC2AF0C9
:107B500028A903D0D151DAEC2AF0289B289728993C
:107B6000B12F01D07AD8B22F01D06CD8B32F01D069
:107B70005ED8B42F01D04DD8B52F01D018D8B62F6C
:107B800001D010D8B1BFB16BB2BFB26BB3BFB36B92
:107B9000B4BFB46BB5BFB56BB6BFB66B440E39ECB2
:107BA0001AF012001A0E80EC10F0B66F120031C9F4
:107BB000B5F1B551DAEC2AF030C9B5F1B551DAECCE
:107BC0002AF033C9B5F1B551DAEC2AF032C9B5F172
:107BD000B551DAEC2AF035C9B5F1B551DAEC2AF035
:107BE00034C9B5F1B551DAEC2AF037C9B5F1B55160
:107BF000DAEC2AF036C9B5F1B551DAEC2AF038C919
:107C0000B5F1B551DAEC2AF0190E80EC10F0B56F31
:107C10001200000EDAEC2AF0000EDAEC2AF0000E68
:107C2000DAEC2AF0180E80EC10F0B46F1200000E9F
:107C3000DAEC2AF0000EDAEC2AF0170E80EC10F0E5
:107C4000B36F1200AA51DAEC2AF0AB51DAEC2AF049
:107C5000160E80EC10F0B26F12009751DAEC2AF099
:107C60009851DAEC2AF0150E80EC10F0B16F12008A
:107C700020A32DD08DC152F18EC153F195C154F185
:107C800096C155F18DC195F18EC196F1D9EC0BF0ED
:107C900050C14CF151C14DF1270E4E6F4F6BF0ECBE
:107CA0000BF048C145F149C146F1070E476FC3ECDF
:107CB0000BF0630E456501D0456F050E80EC10F0AA
:107CC000455DD8A004D0218B69EC1CF0120021ABDB
:107CD0001200219B8EEC1CF0120029B112008DC104
:107CE0004CF18EC14DF10A0E4E6F4F6B0DEC0CF046
:107CF00048C14CF149C14DF1D0C14EF14F6BF0EC90
:107D00000BF048C154F149C155F1130E80EC10F04D
:107D1000640DF3CF52F1F4CF53F1D9EC0BF027956A
:107D20001FB72785279B48C154F149C155F1120E51
:107D300080EC10F0640DF3CF52F1F4CF53F1D9EC95
:107D40000BF01FA704D0278B050EB06F288B48C1FE
:107D500054F149C155F1110E80EC10F0640DF3CFD0
:107D600052F1F4CF53F1D9EC0BF01FB705D0278BAC
:107D70002785040EB06F288B27B506D027A307D020
:107D8000FCEC1EF0279303D0D3EC1EF027831200E7
:107D900020C54CF121C54DF14C6707D04D6705D08A
:107DA000010ECC6FCD6B279112004CC104F54DC173
:107DB00005F50D0E80EC10F04E6F4EC106F54B0E22
:107DC00039EC1AF01CEC80F001014C0E39EC1AF081
:107DD00004C54CF105C54DF14C6707D04D6705D082
:107DE000010ECC6FCD6B279112004CC1CCF14DC16F
:107DF000CDF12781120020A757EF40F02ABB03DD09
:107E0000A3C100F5A4C101F50C0E80EC10F00A6FBF
:107E10000AC113F5470E39EC1AF030EC80F001017D
:107E2000B7DF480E39EC1AF0FD0EDAEC2AF0FD0E41
:107E3000DAEC2AF0FE0EDAEC2AF0BFC1BDF1C0C1C7
:107E4000BEF1FA0EDAEC2AF0FA0EDAEC2AF0200E85
:107E5000DAEC2AF00751DAEC2AF00651DAEC2AF0D3
:107E60000851DAEC2AF00551DAEC2AF00451DAEC88
:107E70002AF02AAB11D0DEC132F1DFC133F1A2EC1E
:107E80002AF032C1DEF133C1DFF1DE51DAEC2AF043
:107E9000DF51DAEC2AF010D091C132F192C133F106
:107EA000A2EC2AF032C191F133C192F19151DAEC96
:107EB0002AF09251DAEC2AF0A551DAEC2AF0A65118
:107EC000DAEC2AF0A751DAEC2AF0AC51DAEC2AF01D
:107ED000AD51DAEC2AF0A351DAEC2AF0A451DAEC35
:107EE0002AF020C532F121C533F13251DAEC2AF003
:107EF0003351DAEC2AF0060EA4EC0DF0A850DAECBF
:107F00002AF0070EA4EC0DF0A850DAEC2AF00A0EC5
:107F1000A4EC0DF0A850DAEC2AF00B0EA4EC0DF056
:107F2000A850DAEC2AF00E0EA4EC0DF0A850DAEC12
:107F30002AF00F0EA4EC0DF0A850DAEC2AF0120E85
:107F4000A4EC0DF0A850DAEC2AF0130EA4EC0DF01E
:107F5000A850DAEC2AF0160EA4EC0DF0A850DAECDA
:107F60002AF0170EA4EC0DF0A850DAEC2AF0180E47
:107F7000A4EC0DF0A850DAEC2AF0190EA4EC0DF0E8
:107F8000A850DAEC2AF0210EA4EC0DF0A850DAEC9F
:107F90002AF0010EDAEC2AF0330EDAEC2AF0C251A4
:107FA000DAEC2AF0C351DAEC2AF0140E80EC10F06F
:107FB0002ABB010EDAEC2AF0020E396F393B150E9E
:107FC00080EC10F03925DAEC2AF0020E396F393BDB
:107FD000160E80EC10F03925DAEC2AF0020E396F1B
:107FE000393B170E80EC10F03925DAEC2AF0030E3D
:107FF000396F393B180E80EC10F03925DAEC2AF095
:10800000090E396F393B190E80EC10F03925DAEC86
:108010002AF0000E396F393B1A0E80EC10F039252A
:10802000DAEC2AF01A0EA4EC0DF0A850DAEC2AF0E3
:10803000000EDAEC2AF0FB0EDAEC2AF0FB0EDAEC9A
:108040002AF0020EA4EC0DF0A8CF39F1030EA4EC37
:108050000DF0A8CF3AF1D890010E3927000E3A233F
:1080600039C1A8FF020EA2EC0DF03AC1A8FF030E21
:10807000A2EC0DF01C0E94EC10F0326703D03367C5
:1080800001D012D0010E3227000E3323700E820F62
:10809000A96E32C1A8FFD5EC0DF0700E830FA96E4A
:1080A00033C1A8FFD5EC0DF0259D11EC4AF02DB1A0
:1080B0006FEC49F060EC80F00101196B1A6B68EF0E
:1080C00039F020A712002ABB0ED025BD19D020936D
:1080D000B72B020E80EC10F0020FD8B0FF0EE806AE
:1080E000B76520831200B72B3C0EB7631200B76B45
:1080F0002093E02B1E0E80EC10F0E0632083120032
:108100002093B72B050EB76520831200D3EC40F007
:1081100020B3AFEC40F020B3C2EC40F0219D97516A
:108120009963218D98519A63218D21BDA4EC1EF095
:10813000219F8D519563218F8E519663218F25BD8F
:10814000218F21BF39EC21F0120076EC45F0E9ECEB
:1081500040F0ECEC23F09BEC46F02095120091C12E
:1081600052F192C153F18FC154F190C155F1D9EC44
:108170000BF01FA712008FC191F190C192F1ECECAE
:1081800023F01200ACC152F1ADC153F197C154F1CB
:1081900098C155F1D9EC0BF01FB7120097C1ACF1A3
:1081A00098C1ADF112002299000E80EC10F0526FD0
:1081B000536B8FC154F190C155F1D9EC0BF01FA74F
:1081C00005D020B7B76B20832289120020A7209307
:1081D000120023B709D00C0EC36501D01200070EA0
:1081E000B06F288B238712000D0EC365F8D7239735
:1081F00012008FC115F190C116F1155111271651BA
:108200001223000E13231423155111271651122384
:10821000000E1323142317C14EF118C14FF111C1E1
:1082200048F112C149F113C14AF114C14BF134ECC8
:108230000CF048C193F149C194F11200510E39EC90
:108240001AF0916B926B936B946BF1EC0FF05A0EEA
:10825000A4EC0DF0000EA864BAEC0FF0116B126BD9
:10826000136B146B010E176F186B010EDE6FDF6B53
:10827000E16BE26BDC6BDD6BA56BA66BA76BA86B90
:10828000E06BB76BB86BB06B289B2B9BD269E86B2C
:10829000259109EC2BF0A4C103F5A3C102F597C108
:1082A000ACF198C1ADF10A6B0AC14EF20AC14FF2AE
:1082B00002EE50F0200E0A6FEE6A0A2FFDD702EE92
:1082C00070F0200E0A6F010EEE6E0A2FFCD702EE40
:1082D00090F0EE6AEE6A200E80EC10F0A8CF15F553
:1082E000210E80EC10F0A8CF14F52C83290E80EC21
:1082F00010F0326F010E32632C93140E80EC10F0EC
:10830000A96F150E80EC10F0B16F160E80EC10F016
:10831000B26F170E80EC10F0B36F180E80EC10F0F7
:10832000B46F190E80EC10F0B56F1A0E80EC10F0DF
:10833000B66F2AAB02D0010EA96F240EA4EC0DF08B
:1083400029B1A8CF18F515EC4AF02397229B209D60
:108350002097268325ADF2EC0DF0210EA4EC0DF054
:10836000A8CFD1F1D105040DF350070FA96ED1ECC0
:108370000DF0A8CF11F5D105040DF350060FA96E2D
:10838000D1EC0DF0A8CFD0F111C50AF1D880640E60
:108390000A55D880A856A8CF10F5326B32C11BF50C
:1083A00032C11CF532C11DF52B95120024B718D02F
:1083B00024A91200249724992A99208D209FB96B13
:1083C0002ABB0AD0010EE8CF7FF0040E5DEC0BF063
:1083D000000EE8CF7FF012008D0E5DEC0BF0120066
:1083E0002497249920AD14D02AAB03D02093209D4C
:1083F0001200208F209DCDEC27F09AEC25F02C99CF
:108400002B9F010EBA6FDFEC27F0249924971200FE
:108410002CB7ABD00BEC4AF0060EB06F288B2CA318
:108420001200116B126B136B146B020E176F186B2B
:10843000F9EC40F0120024B715D024A912002DB990
:10844000FFD026B91CD126BDF3D02499B96BBA2B25
:10845000060E2BBD040EBA6302D0010EBA6FDFEC1C
:1084600027F0120024972499208F209DB96B2DB9F5
:10847000E7D026BBB0D126B902D126BDD9D026B5CA
:1084800000D12CB9C4EF42F02BBF0BD0BA4FDAD0D9
:10849000BA4F8AD1BA4F53D0BA4F45D0BA4F05D24E
:1084A0001200BA4FBCD0BA4F17D0BA4FC3D0BA4F90
:1084B00003D0BA4FFAD112002C732CA30AD0116B3F
:1084C000126B136B146B020E176F186BF9EC40F004
:1084D000ECD1E0EC24F0E9D15A0EA4EC0DF0A86642
:1084E00008D0F1EC0FF0010EA86E5A0EA2EC0DF0C0
:1084F00007D0BAEC0FF0000EA86E5A0EA2EC0DF0E9
:1085000010EC1FF0A4EC1EF039EC21F0ECEC23F0A1
:108510002ABBCBD128BFC9D125B195EC1BF025A131
:108520005BEC1BF0C2D1CDEC27F0B8EC25F0010ECE
:10853000BA6F2B8FDFEC27F024992497120029B112
:1085400026D12685CDEC27F0D0C1A8FF180EA2ECCD
:108550000DF011C5A8FF190EA2EC0DF0CBEC25F023
:10856000010EBA6FDFEC27F01200208F209D2499B6
:1085700024972C89CDEC27F005EC26F02B9F010EDB
:10858000BA6FDFEC27F01200BA4F8FD1BA4F39D053
:10859000BA4F3ED0BA4F2ED0BA4F25D086D105EC77
:1085A00026F0980E526F3A0E536FC6C154F1C7C1F0
:1085B00055F1D9EC0BF01FA705D0980EC66F3A0EF7
:1085C000C76F1200E80E526F030E536FC6C154F10D
:1085D000C7C155F1D9EC0BF01FB71200E80EC66FFA
:1085E000030EC76F1200E80EC65F030EC75B050ED1
:1085F000BA6FD5D7E80EC627030EC723040EBA6F8D
:10860000CED7640EC627000EC723020EBA6FC7D797
:10861000640EC65F000EC75B030EBA6FC0D7268D0F
:10862000CDEC27F030EC80F00101C0EC28F0120016
:10863000269D3BD12D89CDEC27F0C9EC29F0120005
:108640002D9933D12689220EA4EC0DF0030EA864D7
:108650000DD00CD02B8533EC0FF0A0EC2AF023C505
:10866000CEF1CE671200A1EC2AF01200CDEC27F07B
:1086700023C5CEF1CE6712004DEC26F012002699EC
:1086800014D1BA4F6FD0BA4F4ED0BA4F38D0BA4F7C
:1086900017D0BA4F01D01200190EA4EC0DF0A8CFDC
:1086A00032F13207FF0E326301D0322B32C1A8FF04
:1086B000190EA2EC0DF0CBEC25F0050EBA6F1200EE
:1086C000190EA4EC0DF0A8CF32F1322B650E3263F7
:1086D00002D0040E326F180EA4EC0DF0A850322513
:1086E000336F650E336301D0320732C1A8FF190E14
:1086F000A2EC0DF0CBEC25F0040EBA6F1200180EB0
:10870000A4EC0DF0A8CF32F13207030E326301D092
:10871000322B32C1A8FF180EA2EC0DF0CBEC25F0E5
:10872000030EBA6F1200180EA4EC0DF0A8CF32F1B0
:10873000322B650E326302D0050E326F190EA4EC97
:108740000DF0A8503225336F650E336301D0320728
:1087500032C1A8FF180EA2EC0DF0CBEC25F0020EF2
:10876000BA6F1200190EA4EC0DF0A8CF11F5180E77
:10877000A4EC0DF0A8CFD0F111C50AF1D880640E99
:108780000A55A856A8CF10F52887288B8ED0268B9F
:10879000CDEC27F029912A8947EC27F02981010E99
:1087A000BA6FDFEC27F0120029B10AD0268BCDEC8E
:1087B00027F047EC27F0010EBA6FDFEC27F012002C
:1087C0002B8D268BCDEC27F098EC27F0010EBA6F9D
:1087D000DFEC27F012002AB92FD029A12DD0230ECB
:1087E000BA25A96ED1EC0DF0A8CF18F52B9D210E5E
:1087F000A4EC0DF0A8CFD1F1D105040DF350070F73
:10880000A96ED1EC0DF0A8CF11F5D105040DF350F0
:10881000060FA96ED1EC0DF0A8CFD0F111C50AF169
:10882000D880640E0A55D880A856A8CF10F507EC5A
:108830001FF02889288B39D0326B32C118F5269B5E
:10884000BAC1D1F1BA05040DF350070FA96ED1ECEE
:108850000DF0A8CF11F5BA05040DF350060FA96E5F
:10886000D1EC0DF0A8CFD0F111C50AF1D880640E7B
:108870000A55A856A8CF10F52889288B16D020AF06
:1088800012002DB945D02CB93ED026A908D02BB561
:1088900031D023C5CEF1CE6702D04DEC26F0B92BF6
:1088A0000A0E80EC10F0B96512002BA50DD02B95A7
:1088B00033EC0FF0A4EC1EF0ECEC23F025B195ECBA
:1088C0001BF025A15BEC1BF02B95209F209D10EC4D
:1088D0001FF0CDEC27F035EC1BF015EC24F0B96B54
:1088E00026992D99269B269D26952B9D2C9924977C
:1088F00024991200A0EC2AF023C5CEF1CE67CFD781
:10890000A1EC2AF0CCD705EC26F0DFEC27F0C7D796
:10891000C9EC29F0C4D729EE4AF0100E396FDE6693
:108920000DD0392FFCD733EC0FF0010E5DEC0BF0BE
:10893000020E5DEC0BF070EC80F0010181EC0EF0AA
:10894000F2EC0DF0A56BA66B939C939E819C819E8F
:1089500020B509D820B14FD820A9F0EF47F000008A
:1089600003000000F5D776EC45F02CB148EF45F058
:1089700053EC3AF045EC3AF0A62B0E0EA66526D045
:1089800072D89BEC46F01AEC80F00101A1C1A3F172
:10899000A2C1A4F18DC1A1F18EC1A2F1A66B070EF7
:1089A00094EC10F032C152F133C153F1A1C154F132
:1089B000A2C155F1D9EC0BF01FB701D007D0070EBB
:1089C00094EC10F032C1A1F133C1A2F18DC100F5D8
:1089D0008EC101F50B0E80EC10F00A6F0AC112F582
:1089E0000C0E80EC10F00A6F0AC113F540EC80F019
:1089F00001012095120090EC3AF027A105D013EC6C
:108A00004AF000000300000015EC4AF0A52B050E0B
:108A1000A56512D028D8060E94EC10F032C152F1A0
:108A200033C153F18DC154F18EC155F1D9EC0BF026
:108A300020891FB72099A56B209124B70AD024B9AB
:108A400008D0F292F0902A932A9124992497D59EE7
:108A50001200F292F0902A932A9124992497D59E9D
:108A6000209927871200FFEC18F003000000030094
:108A70000000030002EC19F0F2EC18F00300000013
:108A8000030000000300F9EC18F0DAEC17F0120014
:108A9000F26AF16AF06AC290F2EC0DF0100E926E7A
:108AA000806A936A816A1D0E946E826A956A836AEF
:108AB000966A846AD56ACD6ACA6A9B6A020ED36EC8
:108AC000D180EAC137F10F0E396F03000000392F52
:108AD000FCD701EC4AF00400050EAEEC0CF003EC00
:108AE0004AF003000000372FF4D7EBD7C280000014
:108AF000C282C2B2FED7C4CF4DF1C3CF4CF1C60E75
:108B00004E6F030E4F6FF0EC0BF0640E4E6F4F6B19
:108B100034EC0CF048C1C2F149C1C3F1C290C2C1EA
:108B200054F1C3C155F1280E526F0A0E536FD9ECA0
:108B30000BF02C911FB703D0020EEA6F2C818DC170
:108B400054F18EC155F1990E526F3A0E536FD9EC14
:108B50000BF02C911FA703D0030EEA6F2C81299BE9
:108B6000299D280EA4EC0DF0A8CF54F1290EA4ECF9
:108B70000DF0A8CF55F1D00E526F070E536FD9EC00
:108B80000BF01FA7298B940E526F110E536FD9EC67
:108B90000BF01FA7298D29AB73D029AD71D0680EBA
:108BA000A86E280EA2EC0DF0100EA86E290EA2ECF5
:108BB0000DF007C1A8FF2A0EA2EC0DF006C1A8FF18
:108BC0002B0EA2EC0DF008C1A8FF2C0EA2EC0DF0AC
:108BD00097C1A8FF2D0EA2EC0DF098C1A8FF2E0E94
:108BE000A2EC0DF0A86A2F0EA2EC0DF0A86A300ED0
:108BF000A2EC0DF0A86A310EA2EC0DF0A86A320EBC
:108C0000A2EC0DF0A86A330EA2EC0DF0A86A340EA7
:108C1000A2EC0DF0A86A350EA2EC0DF097C1A8FFEA
:108C2000360EA2EC0DF098C1A8FF370EA2EC0DF0A5
:108C300007C1A8FF380EA2EC0DF006C1A8FF390E3F
:108C4000A2EC0DF008C1A8FF3A0EA2EC0DF097C1FE
:108C5000A8FF3B0EA2EC0DF098C1A8FF3C0EA2ECC1
:108C60000DF007C1A8FF3D0EA2EC0DF006C1A8FF54
:108C70003E0EA2EC0DF008C1A8FF3F0EA2EC0DF0D5
:108C8000280EA4EC0DF0A8CF54F1290EA4EC0DF0A1
:108C9000A8CF55F1C2C152F1C3C153F1D9EC0BF0C9
:108CA0001FA71200C2C1A8FF280EA2EC0DF0C3C17D
:108CB000A8FF290EA2EC0DF007C1A8FF2A0EA2EC16
:108CC0000DF006C1A8FF2B0EA2EC0DF008C1A8FF05
:108CD0002C0EA2EC0DF097C1A8FF2D0EA2EC0DF00A
:108CE00098C1A8FF2E0EA2EC0DF01200800ECF6EE0
:108CF000CE6A3C0E036111D03C0E04610ED0180EFA
:108D000005610BD0200E066108D00C0E076105D05E
:108D1000640E086102D09D801200000E036F000EE9
:108D2000046F0C0E056F020E066F080E076F090E1A
:108D3000086F9D801200360EA4EC0DF0A8CF54F100
:108D4000370EA4EC0DF0A8CF55F197C152F198C1A0
:108D500053F1D9EC0BF01FA719D097C1A8FF360E1D
:108D6000A2EC0DF098C1A8FF370EA2EC0DF007C1E0
:108D7000A8FF380EA2EC0DF006C1A8FF390EA2EC38
:108D80000DF008C1A8FF3A0EA2EC0DF03B0EA4ECCA
:108D90000DF0A8CF54F13C0EA4EC0DF0A8CF55F186
:108DA00097C152F198C153F1D9EC0BF01FB71200E3
:108DB00097C1A8FF3B0EA2EC0DF098C1A8FF3C0E96
:108DC000A2EC0DF007C1A8FF3D0EA2EC0DF006C10C
:108DD000A8FF3E0EA2EC0DF008C1A8FF3F0EA2ECCA
:108DE0000DF01200249B9D9A0FEC4AF09E9A620EA1
:108DF000AD6EFAEC0DF000EC0EF0AECF05F1180EF2
:108E00000561056B00EC0EF0AECF04F13C0E046181
:108E1000046B00EC0EF0AECF03F13C0E0361036B6C
:108E200000EC0EF0AECF07F10C0E076501D0076F16
:108E300000EC0EF0AECF06F107C132F1324F1F0E3B
:108E4000324F1C0E324F1F0E324F1E0E324F1F0E6E
:108E5000324F1E0E324F1F0E324F1F0E324F1E0E5C
:108E6000324F1F0E324F1E0E324F1F0E066502D0BC
:108E7000010E066F00EC0EF0AECF08F1640E086133
:108E8000086B11EC4AF09E9A20859D8AD8EF39F044
:108E900028919D9A0FEC4AF09E9A660EAD6EFAEC00
:108EA0000DF000EC0EF0AECF32F100EC0EF0AECFD4
:108EB00033F1596BFA0EDAEC0CF0FA0EDAEC0CF036
:108EC000FA0EDAEC0CF0FA0EDAEC0CF032C152F1D8
:108ED00033C153F197C154F198C155F1D9EC0BF05E
:108EE00050511FB7000E506F50C1ADFF50C1A8FFC9
:108EF00050C159F1010EAA6E000EA96ED5EC0DF00D
:108F0000000EAA6E11EC4AF09E9A9D8AD8EF39F0B5
:108F10000101B1EC48F020B36AEC1AF0FC6A01EEF2
:108F200009F0EE6A0A0EEA62FCD7F2EC0DF076EC7C
:108F300046F008EC19F0239D23ADFED78F6B906BA4
:108F4000196B1A6B208933EC45F020998DC19FF184
:108F50008EC1A0F18DC1A1F18EC1A2F18DC1A3F18D
:108F60008EC1A4F1CC2B0A6B0AC111F54F0E0A6F0A
:108F70000AC110F58DC100F58EC101F520EC80F01D
:108F8000010130EC80F0010118EC80F0010167EC88
:108F90003AF0010140EC80F00101010EA96E010ED2
:108FA000AA6ED1EC0DF0A8CF39F1A92AD1EC0DF0C1
:108FB000A8CF3AF1AA6A010E396304D0330E3A639E
:108FC00001D00ED0010EA96E010EAA6E010EA86E80
:108FD000D5EC0DF0A92A330EA86ED5EC0DF0AA6AD7
:108FE00007EC4AF015EC4AF071EC0FF0000EE8CFF8
:108FF0007CF0000EE8CF7DF0000EE8CF7EF0000E92
:10900000E8CF7FF0FF0E2E6F2EC17AF0FF0E2E6F8D
:109010002EC17BF0A4EC2BF0A3C19FF1A4C1A0F161
:10902000AA6A5C0EA4EC0DF0290EA86201D006D04D
:109030002DD8290EA86E5C0EA2EC0DF01F0E94EC3C
:1090400010F09A0E326304D0020E336301D006D0C2
:1090500027B77DEC48F027B798EC48F01F6B206BE2
:10906000216B226B236B246B256B266B276B286B84
:10907000296B2A6B2B6B2C6B2D6B270EA4EC0DF040
:109080002A85010EA8622A9568EF39F084EC29F050
:10909000140E53D0289F29912A9BAA6A220EA4EC71
:1090A0000DF0010EA86206D0288F000E0A6F0AC1CB
:1090B0001FF51200020EA86206D02981000E0A6F69
:1090C0000AC11FF51200030EA86206D02A8B000EFB
:1090D0000A6F0AC11FF51200040EA86205D0010E26
:1090E0000A6F0AC11FF51200050EA862120029813D
:1090F000010E0A6F0AC11FF5120033EC0FF042ECAB
:1091000029F00A0E396FC80EDAEC0CF02497249976
:1091100020B1D3EC40F020B139072091396701D05C
:10912000120020B3120024B7120024B91200F0D7A5
:1091300033EC0FF063EC29F0E4D7396FC80EDAECAA
:109140000CF02497249920B1D3EC40F020B13907DA
:109150002091396701D0120024B7120024B91200FF
:10916000F2D76C0ED36E110E926E806A030E936E60
:10917000816ADD0E946E826A000E966E846A000E1D
:10918000956E836A400E9B6E1F0ED56E070ECD6ED8
:10919000D00EF26E050EF16E080EF06E210E9D6E71
:1091A000000EA06ED06A000EC26E0E0EC16E8A0E48
:1091B000C06EC66A000EC76E280EC66E000EC56E63
:1091C000080EC86EBD6ABA6A070EB46E200E6F6EC6
:1091D000240EAC6E900EAB6E080EB86EB06A220E06
:1091E000AF6EAE6A9E6A1200010EEB6F0F0EEC6F4F
:1091F000010EBA6FB86B208F218733EC0FF057EC5C
:109200001EF024972499219121932AEC1CF02CEC38
:109210001DF03FEC13F020A109D052EC3BF0D3EC51
:1092200040F090EC3AF076EC45F0209121B123EF3C
:1092300049F020AF12EF13F020B964EF13F020B320
:10924000F0EF47F0E6D7BA4F1CD0BA4F0AD0BA4F6A
:1092500010D0BA4F79D0BA4F58D0040EBA6F66EF1B
:1092600013F0020EEB27C70EEB61EB6F020EBA6F25
:10927000C8D7030EEC27630EEC61EC6F030EBA6FD8
:10928000C0D7258D2C87ECC14CF14D6B640E4E6F11
:109290004F6BF0EC0BF0E80E4827030E492348C152
:1092A000C6F149C1C7F1C6C18DF1C7C18EF1219187
:1092B0002193209F2497249964EC49F02083500E39
:1092C00039EC1AF05EEF3BF02D81530E39EC1AF0B9
:1092D00062EC80F00101540E39EC1AF012002D916D
:1092E000530E39EC1AF064EC80F00101540E39ECA5
:1092F0001AF0470E39EC1AF030EC80F00101C8EC9E
:109300003EF0480E39EC1AF0120033EC0FF022EC6C
:1093100043F02497249920A109D052EC3BF0D3ECE0
:1093200040F090EC3AF076EC45F0209124B709D06B
:1093300024B907D020B964EF13F020B3F0EF47F061
:10934000EAD7050EBA6F56D71EEC41F0258D2C8753
:10935000ECC14CF14D6B640E4E6F4F6BF0EC0BF0AB
:10936000E80E4827030E492348C1C6F149C1C7F199
:10937000C6C18DF1C7C18EF164EC49F0010EE8CF92
:109380007FF00C0E5DEC0BF0000EE8CF7FF01E0EB0
:10939000ED6F2AEC1CF009EC4AF06CEC3CF028EC88
:1093A0003DF000EC80F00101430E39EC1AF0ED2F96
:1093B000F2D7EB2FECD723C5CEF1CE6716D005EC54
:1093C0004AF06FEC49F0259D2C97FA0EDAEC0CF080
:1093D000FA0EDAEC0CF0FA0EDAEC0CF007EC4AF0CC
:1093E000010EEB6F050EBA6F05D76CEC3CF028EC64
:1093F0003DF000EC80F0010123C5CEF1CE67F5D73A
:10940000DED781881200819812008188120081982D
:1094100012008178120081881200819812008186E2
:1094200012008196120081861200819612008176C8
:109430001200FFFFFFFFFFFFFFFFFFFFFFFFFFFF28
:10944000FFFFFFFFFFFFFFFFFFFFFFFFFFFFFFFF2C
:10945000FFFFFFFFFFFFFFFFFFFFFFFFFFFFFFFF1C
:10946000FFFFFFFFFFFFFFFFFFFFFFFFFFFFFFFF0C
:10947000FFFFFFFFFFFFFFFFFFFFFFFFFFFFFFFFFC
:109A0000AF9BAFAFAFAFD1AFB205B007B008AF09F2
:109A1000AF09AF09AF09B108B2079B049F9F9F9F91
:109A2000AE9FFFFFFFFFFFFFFFFFFFFFFFFFFFFFF7
:109A3000FFFFFFFFFF8F82FFAC04A1149B1A96204B
:109A400092248F288A0E8C10940B8A0C9609870F0B
:109A5000960885129707830785079706850783076A
:109A600096068708820796058A07810696058C0761
:109A7000810594058E088005940490078005930461
:109A80009107800591049208800590049407800551
:109A90008E05950780058C05960880058A06960830
:109AA000820588069707820685079708840683073C
:109AB00097088507800898078707970F8908950DED
:109AC0008B0A8C108E0E912894269922A01CAA1520
:109AD0009707FFFFD7FFB701B403B404B403B4047E
:109AE000B304B304B305B205B206B205B2068136BB
:109AF0008137813781378137FF37FFFFFFFFACFFA9
:109B0000FFFF90FF8903A8008705A5038607A3052B
:109B10008508A007840A9F08840B9F06830D9F0673
:109B2000820E9F06810882049E05830882049E049B
:109B3000840881049D05850881049C0587078104AC
:109B40009C04880781049B04890781049A048A077E
:109B5000810499048B07810498048C07810496057D
:109B60008D07810495058E07810494058F07810474
:109B70009206900782049006910782048E0792074E
:109B800083048B07930883048609940A8404951937
:109B900085049617860498148704991289049B0EED
:109BA0008C049D08B305BA05FFFF8EFFB7008A023B
:109BB000A8018804A5038607A3058608A5058407D0
:109BC000A7058406A8058206AA058205AA058105BF
:109BD00091059504800591059504800591059504EE
:109BE00080059204950480059204950480059204F2
:109BF00095048005920494058005900594068005DF
:109C00009005940680058F05920882058E059208BE
:109C100082058C06900A82068A078E0C84068707C6
:109C200081068C06850781158907870883138918A3
:109C300085118B16870F8D148A0C91128E07AC0E2E
:109C4000FF0AFFB88BFFB205B006AF08AD09AC0B39
:109C5000AA0CA90E8107A7058208A6058407A405FA
:109C60008607A3058707A10589079F058A089E0522
:109C70008C079C058D089B058F0799059008980512
:109C80009207960594079505950793059707920502
:109C9000813581378137813781378137A437B305E3
:109CA000B305B305B305B305B3058F05FFFF8CFFFF
:109CB000A20192009203901085058F1C84078E1DCF
:109CC00083088E1D8308911C8207931B82068E05D4
:109CD000950581068E05970481058E0597048105FB
:109CE0008D05980580058D05990480058D059904DD
:109CF00080058D05990480058D05990480058D05E5
:109D0000990480058D05990480058D0599048005C9
:109D10008D05990480058D05970581058D059705AD
:109D200081058E05950581068E05930682068E05B2
:109D3000910782078F058D0883089005870A830B9A
:109D40009105841C9205851A930586189405A5151E
:109D5000AA11C50CFFFF11F11BA2219A269429908C
:109D60002B8E0D8C05850E850B880588098B088840
:109D70000689088E0786058B07910784058B069355
:109D80000683058C06950582058D05960681048D52
:109D900006970580058D05980580058D059804803A
:109DA000048E0B99048E0B99058E0B98058E0B98DB
:109DB000058E05980480068E05960481058F05960C
:109DC0000581068E05940582078F07900583098E0D
:109DD000088C07840B8D0A8607851B8E05871990D2
:109DE00003891792008B13960FA707ADFFC8FFFFDB
:109DF000059605B305B305B305B305B301AF0581FA
:109E000004AC058107A905810AA605810CA405817A
:109E10000FA10581129E0581139B0583139805866A
:109E2000129605891293058C1290058F118E05925A
:109E3000118B0595108905981086059B0F84059E4A
:109E4000108115A012A310A60DA80BAB09AD06AF8B
:109E500004B2A7FFFFFF03CA0BB10FAB0790118F2E
:109E60000C8D148A0F8A1688118818861486078428
:109E7000088715850683078B068408860681068D6C
:109E8000068307890480069005820C8B0591058165
:109E90000A8D05920481088F05940480069005952B
:109EA000048006900B9505910B9505910B950592F5
:109EB0000B94069105940480079105930580088F03
:109EC000049305810A8E059106810C8C068F06820B
:109ED00006890681058E088308850781068C15840E
:109EE0000883078813860A850A82118716870F89D7
:109EF00014890C8B128C068F10900CAA06AFFFC52C
:109F0000E9FFAC09980F8D0095138A029217880417
:109F1000901986068E1B850788098F0A83068D088F
:109F20009007820590078F078205930690058005AC
:109F300094068F06800596058F05800597058F048A
:109F4000800598048F04800598048E05980B8E0573
:109F5000980B8F04800598048E04810597058E0464
:109F6000810596058D05810695068E048305940569
:109F70008D05830693068D04850690078B0586075D
:109F80008D098A058808880B8706890C8C2D8F2BF4
:109F9000932796249D1FA917D30700FFFFFFFFFFFC
:109FA000000022003500D2000001A8014302AC02EB
:109FB0005403ED035404FF049A0500EE00F00D0E67
:109FC000EE6AEA62FDD71200FFFFFFFFFFFFFFFF0F
:109FD000FFFFFFFFFFFFFFFFFFFFFFFFFFFFFFFF91
:109FE000FFFFFFFFFFFFFFFFFFFFFFFFFFFFFFFF81
:109FF000FFFFFFFFFFFFFFFFFFFFFFFFFFFFFFFF71
:10A0000000000F0016006B008300DC002D016601CC
:10A01000C10116024C02AB0202031B032A034403D4
:10A020006F0375039F9F03BA049A059A0499039BD3
:10A030009F9F9FC0BF9F9F7FBF9F03CD0E96128E95
:10A04000168A0487078B0385038C04800383048BA3
:10A0500004820282048B03840281038B02870281C3
:10A06000038A028802810488038902800387028BA5
:10A0700003810385028C03820482038C03830480A2
:10A08000038C0685048C168713890E8E0395FFCDED
:10A090000084019E029C029B029C039B029B1D9BD1
:10A0A0001D811D81FFFFFCC0850194008403910286
:10A0B0008305900382069003820790028103810248
:10A0C0008F02820481028E02830481028D02840445
:10A0D00081028D02850381028C02860381028A033C
:10A0E000870382028802880482028603890483022D
:10A0F0008A0D84028C0A85028D0887029003E00293
:10A100009AFF8501920283049303820495028203DD
:10A110009602810289028A02810289028A028102F0
:10A1200089028A02810289028A02810288028A03E4
:10A130008202870289048202850387068303810ADB
:10A1400084038404810A870C84068A0A8802FF0734
:10A15000D3849A0299049705960781039402820496
:10A160009302840391028504900287038E0288047F
:10A170008D028A038B028B048A02811C811D811D42
:10A18000941D9C029C029C02C80200FA068D028863
:10A190000F8304870F82038809820281038A028168
:10A1A0000287028C02810287028C02810187028D64
:10A1B00002810187028E02800187038D028002875F
:10A1C000028C02810287028C02810387038A02814A
:10A1D0000388048802810588058402820E8902832F
:10A1E0000C8A0894ECE591088B1188158517840575
:10A1F0008602840585038902830386038A0281031C
:10A2000086038C02810287028C02810287028D0202
:10A21000800287028C02810287028C0281028702FF
:10A220008B038102880289038302870284058305E8
:10A230008703850E8A00950CE60680FF9C029C022F
:10A240009C029702810294028105910281088F028B
:10A2500082098C0285098902880987028B08840299
:10A260008D0982029008930B950998069A04FC01C7
:10A2700005F4038A088807870A8509850483058110
:10A280000B8303810485028206850388028105878A
:10A29000028902810388028A02810388028A02817C
:10A2A0000289028A02810388028A02810488028963
:10A2B00003810686028803820383038102860B835F
:10A2C0000581048208840B84058709860597E7E5E4
:10A2D00098048B098600890C8402880E8203880307
:10A2E000880382028A02870381028C02870281022C
:10A2F0008C02870280038C02870281028C02870213
:10A3000081028C02870281028A0387028203890309
:10A3100086028303870485028504810781038708F9
:10A320008A168F12E90C9F9F03AB038A048B048962
:10A33000048B0589048A0489028C038B9F9F9FC02C
:10A34000C89F9401940A940A96089F05B99FA9FF93
:10A350009B009403940A95099806FF0302830A94CC
:10A360000A9407940497BAFF15C815891589028BBA
:10A37000019B019C019D029D049C159A148A138BDC
:10A38000028A029B019C019D029D159C1589148ADD
:10A39000118DFFA0FFFFFFFF00FF00000E001B005C
:10A3A00048007D00B400E700F0000D012A014B01D8
:10A3B0006401700185018E01A301D601E20115023D
:10A3C000460267029C02CB02EA02210352036003A9
:10A3D00071039C03CD03F8031B045C047D04B804E3
:10A3E000E5040E05410564059705AC05CD05EA05B4
:10A3F0000F0624063D0656067F06A406D50600076E
:10A40000390752076B0784079D07C607DF0718083F
:10A4100037084C086B087C089508A108D408F9088F
:10A42000200945097A099B09E409F909140A330A44
:10A43000540A710A8A0A9F0AC80AED0A120B270BEE
:10A440005A0B770B8C0BA50BBE0BE30B040C390CD2
:10A450005C0C630C860C9F0CAD0CD60C050D2A0D04
:10A46000610D6C0DAB0DB80D050E3C0E5D0E700E42
:10A47000730EBA0ECB0EE40E150F3C0F610F6B0F6F
:10A48000860F8A0FDB0FE20F03F8018A0C85028228
:10A490000A85028394FF00CD0591039101C70591C0
:10A4A00003919DDA83018F0183018F018301880667
:10A4B000870D81078F0183018F0183018F01820145
:10A4C0008607890D83058F0183018F018301A20017
:10A4D00002B40186048A0186018802810185008810
:10A4E000018300860287028201851285018502842C
:10A4F000018400870185018301880284018201892A
:10A50000058403929A9F9203880585018301850142
:10A51000860283018400890282058B0382039202F2
:10A5200082028C02830289048402820186018503EF
:10A53000830186008701820191019D0403A4069195
:10A5400004880281028208860185008602840185D2
:10A5500000860384018401860582018306860282C7
:10A560000180038803850294069201900082FF9D7A
:10A570000194069002918BFF07E70C8C03890387F7
:10A580000286028B0184028E018201910181029177
:10A5900000800093B0B093008100910181018F028F
:10A5A00082028D0284028B028602870389038D0B4F
:10A5B000E707009F019601950282009002810491B5
:10A5C000078D078F04940092028101900183018F0F
:10A5D0000095A0A6950195019501950191018B0A21
:10A5E000900B9501950195019501A40188FF8201C9
:10A5F0008F0190069404FC0001B801950195019526
:10A60000019501950195019501950195FFBC018783
:10A610000295029494FF01C1039304900490049066
:10A6200003900391039103910193A0C490028B0ABC
:10A6300085028903860187058601830186018600DC
:10A6400084018601840085028601820186028601DA
:10A6500080028701880184048B03900AA30201CA47
:10A66000019501941095108694FF00B3018B01872A
:10A670000389018604890186028801800086018899
:10A68000018200860187018301860185018402869B
:10A69000018301850687018604880187BFB488018C
:10A6A0008B0087018C01860185008501860185006C
:10A6B0008501860185008501860183018502860169
:10A6C000810280018301880182049205B70300A4FE
:10A6D0000294049202910180028F0182028E018312
:10A6E000028C0185108B1086029001940096B7A110
:10A6F0008501880083088702820285018701840022
:10A700008700860184008700860184008700860117
:10A710008400860186018400850187018500870801
:10A720008600B60608B50C8C028901820283018777
:10A7300001830186018601830186008600840187EA
:10A7400000860184018601860283018401870884D2
:10A75000058FB1B7960096008D0086018A008604A9
:10A760008700880585008B0482008D059006930381
:10A77000C30104BB04890682028702800180018331
:10A780000187028301850086018501850086018598
:10A790000185018602830185028601810180018392
:10A7A0000588068102890484B3B68605880084077B
:10A7B0008701840284018601860184008601870066
:10A7C000830186018700840086018501830187015A
:10A7D0008402820188028B0DB80901FE0186028C79
:10A7E0000285028B028594FF01FF018601820286A9
:10A7F0000685028704850094A0FC950193029303CB
:10A80000810091018101900183018F0184018D01FB
:10A8100085018D0186018B0187018B0188018901EA
:10A8200089019E01009E00840090008400900084B5
:10A8300000900084009000840090008400900084C8
:10A8400000900084009000840090008400900084B8
:10A85000009000849AA189018A0188018A018701F8
:10A860008C0186018C0185018E0184018E0183019A
:10A870009001810192018100920194039402A4014C
:10A8800001B101950194019501940188028201842E
:10A890000486028101850284018402860282068F79
:10A8A00004919DBF8D0781048A04870288028B0171
:10A8B0008701840183038700840082058601830069
:10A8C0008201820186018300840082008601820168
:10A8D0008400820086018102830082018701820A4E
:10A8E0008A00A10802A70491048F068F048D0182BB
:10A8F000038B0185048C0183048F018005910494EE
:10A9000004950294999C8610861085008501860125
:10A910008500860086018500860086018500860008
:10A9200086018500850186018301850286018301F8
:10A9300084028702800581028902820393059F02B7
:10A94000069E0A8E038A0385018902890187028B8C
:10A950000086018D0086018D0086018D0186018CA7
:10A960000186018B028802880089008A999E8610E0
:10A9700086108D0086018D0086018D0086018D0078
:10A9800086018C0186018C0186018A02880186037A
:10A990008B028E0AA20510B1108600860185018502
:10A9A0000086018501850086018501850086018577
:10A9B0000185008601850185008601850185008667
:10A9C000018501850086018DB1B486108610850051
:10A9D0008E0185008F0085008F0085008F00850027
:10A9E0008F0085008F0085008F00C400069E0B8DB0
:10A9F000028A02870288018A0187018C0086018D04
:10AA00000086018D0086008701840186008601840E
:10AA10000186008600840288068400890585B19E2F
:10AA200086108D10950195019501950195018E0176
:10AA30008610B41000B1008E0086018D0086018D55
:10AA40000086018D108610860086018D0086018D9E
:10AA50000086018DBFCC9601950186018D0086018F
:10AA60008D0086018C008701870F890D9600960066
:10AA7000AC0010991086028D02930493029102801B
:10AA8000028F0282018D0385018A02880188038A70
:10AA90000086018D0096B19C861095109501950158
:10AAA00095019501950195019501B40110991086C4
:10AAB00003870395039503950293029203920391F2
:10AAC00010921086999C8610861095039502950326
:10AAD0009503950395039502870386109C10089DA6
:10AAE0000C8C028903870187018B0187018C00860A
:10AAF000018D0086018D0186018C0186018B028803
:10AB000002880C89088CB1A08610861086008E0001
:10AB100086008E0086008E0086008E0084018E01E5
:10AB200084018E0182028F029206A702089D0C8C7E
:10AB3000028902880187028B0186018C0086028EC1
:10AB40000084048E0182018C01810182018C0181CB
:10AB50000283028801820C8401830886B1A08610DA
:10AB6000861086008E0086008E0086008E0086008D
:10AB70008D0184018B04840180018903830788038C
:10AB800086058A028A009C0003B302860588018636
:10AB90000187028201860186018301860086018584
:10ABA0000185008601850185008601850185018674
:10ABB0000185028302860284028101880585019352
:10ABC00099A0960096009600960096008610861032
:10ABD0009600960096009600AC000C990E8A02959D
:10ABE00001950196019501950195019402940E87B6
:10ABF0000C8899A0950194049405940594059205F8
:10AC00008F048F048F048F049204AB0105990A927C
:10AC100009920490058E048E05900694069406927F
:10AC20000989068AA9A686008B0186028803880303
:10AC300084038B0381038F0391058F0581038C03AC
:10AC400085028803870387038B0196029C00009985
:10AC500002960395039503950A94098D048B04903D
:10AC6000039002920094A9AC86008C0086028A00B0
:10AC700086048900800286018700810386018500A1
:10AC80008303860184008502860182008603860193
:10AC90008000880386018A0386018B0295019C014E
:10ACA00015DF0181019101810191018101910181F2
:10ACB0000191018101910181019100820091B0B265
:10ACC00095019503950395039503940495049503C5
:10ACD0009503B30100B000910182019101810191BE
:10ACE0000181019101810191018101910181019114
:10ACF0001581CEE19401920292029402960295028D
:10AD00009503D60100AB009600960096009600963B
:10AD1000009600960096009600960096E09A95019F
:10AD2000950395029502FF00A68993018C04830187
:10AD300080018B02830082018A01830184008A00E2
:10AD4000830184008A00830184008A0083018300D8
:10AD50008C00820182008C018C0BB40A12AF11842A
:10AD6000018C0186008C0188018A0188018A018892
:10AD7000018A0188018B0286038B0283088D04906F
:10AD8000B8A08F068D0884028C0286018A02880191
:10AD90008A0188018A0188018A0188018B01860164
:10ADA0008C0185028D01A60004A10890028D028409
:10ADB000018C0286018A0188018A0188018A018842
:10ADC000008B0088018C018611861284A2B4920245
:10ADD0008E0780048C03810182018B018201830133
:10ADE0008A01820183018A01820183018A01820131
:10ADF00083018B01810183018B0182058D01830415
:10AE0000B50001B601950195109003850181018F70
:10AE10000183008F0184018E0184018E00840190E2
:10AE20000295AAAB8902810480018704810B860107
:10AE300083018101830186008500820083008501F2
:10AE400085008200830085018500820083008501E2
:10AE500083018201830086018305830086008405C7
:10AE600081018601890087048B009A0112AF128448
:10AE7000018C019400950195019502950B950A8C22
:10AE8000CDB488018A0188018A0188018501820187
:10AE9000850C8201950C95019501CC0101C40196A8
:10AEA0000185018D0185018D0185018D0185018C53
:10AEB0000181108202810F810182AFDC84128F1226
:10AEC0009402940192038001900282018E02840117
:10AED0008C0286018A03890096019C0000B0018ED5
:10AEE0000184018E0184018E0184018E12841284FA
:10AEF00001950195019500969DB48A0C8B0C9500E7
:10AF0000950195018B0C8B0B9401950195018B0C90
:10AF10009C0B0CB50C8A018C019400950195019550
:10AF200002950B950A8CA1B491048E0782028C03C2
:10AF300086018B0188018A0188018A0188018A01C2
:10AF400088018B0186018C0183038D029008A00487
:10AF500011B5108501870186008C0088018B01885E
:10AF6000018A0188018A0188018B0286028B028492
:10AF7000088D0490A1A090048D0883028C038700A3
:10AF80008A0288018A0188018A0188018B01880070
:10AF90008C0086018C01860FAF110CCD0C8A018CC0
:10AFA0000194009501950195019501960095B8A72A
:10AFB00085008C0183048C0184048A018201830151
:10AFC0008A01820183018A01820183018A0183014E
:10AFD00082018B01830082018B0182018D05830038
:10AFE000B60301B5019501950E920F88018A01887B
:10AFF000018A0188018A0188018A01880194B5B516
:10B000008C0A950B950296019600950095008B0190
:10B010008A0CB40C009D0396049404950494049443
:10B020000393039103910490039000939DA89305CB
:10B03000930893058F038F04920495039405930559
:10B040008C038B09A20601B50188028A0286028C54
:10B050000382028E02800491049202910280028E89
:10B060000383028B0286008A0189ACB486018C02BC
:10B0700085018905880187048A0184048E0191076E
:10B080008F0490048F0490049303A70100A9018A00
:10B090000287018A0386018A0485018A028401806D
:10B0A000018A02820182018A02810183018A02806F
:10B0B0000184048A0185028A0187018A0188019539
:10B0C000A29C960095019301810586028107830861
:10B0D0008A06810291018101920181009201810021
:10B0E0009201C80090FF8115FF15C8909201810060
:10B0F0009201810092018100910182018506810106
:10B10000830381078A0881058F019501BA01009F99
:10B11000019501950194019501960295019501957E
:10B12000019501940195F8A6890185048103850C98
:10B130008302FF0AA19491028E0782038C03860189
:10B140008B0188018A0186008607860E84088701A4
:10B15000810088018A0187018B028601B60100A95E
:10B16000018C0186048902850E8702870682018090
:10B170000187018300860087018401860086018D96
:10B180000186008D0186008D01950195B49C860095
:10B190008E008F0882018F0184018F0084018E014F
:10B1A00084018E018401900082018F018E08860047
:10B1B000B90001B100870081038901840081038BFC
:10B1C00001820081028D018100810A8F0A8C038A2D
:10B1D00001800081038B0182008103890184008149
:10B1E0000189018600810089FFAC099008820981EC
:10B1F000088290FF02B800850486048002830784D9
:10B20000018101840184018201830184018201831F
:10B21000018301840182018401820184008301840D
:10B2200001830182018402840780018504830480F4
:10B23000018EC8BB94019502C50194019502DC0101
:10B2400002890791018E0285018B02820082008BA8
:10B2500005810082018900810183008100890181CB
:10B2600001840080008901810184008001890180BE
:10B2700000840081008A018101820081018A0081AD
:10B280000185018B0186028D02820490BC898F01A9
:10B2900081038A01810181048A0182008101800188
:10B2A0008A018200820080018A018200820080017E
:10B2B0008A018101810081018A0181088B01810756
:10B2C0009501B80101BA03940292018002900182B3
:10B2D000018F018401910394029201800290018206
:10B2E000018F0184D0B6950190018B0C8D0A8F08D7
:10B2F000910693049502BC00FFFF89CF91028E074F
:10B3000085018B0288018B00800081078900800104
:10B310008107890081008200840089008100820009
:10B32000840089008001800182038A0081008102FB
:10B3300081018A0088018B0186018D0182029002C1
:10B34000890400C900960096009600960096009623
:10B350000096CBDC930191058101900183018F015F
:10B3600083018F01830191009205D803009F00871C
:10B37000008D0187008C0187008C0187008C01877C
:10B380000B8701810B870181008C0187008C01876D
:10B39000008C0187008C0187008C0087CA9D860085
:10B3A0008D0084018C0284018C03840180008C0157
:10B3B000830180018C01820181018D0182048E0153
:10B3C0008302D30100D1018E0184018D0186018C9D
:10B3D00000820182018C00820182018C0181018244
:10B3E000058D0180018F0381FFD4019103930193A7
:10B3F00000959DF68511950B960195019501950196
:10B4000094008B02950B9502950195018500FFFF35
:10B4100080CE0195029403920491008604890386EC
:10B4200005870286068504860782048709800F86C1
:10B4300007870780068706800788058008870381BD
:10B4400007880180018106880580058907800488B6
:10B450000A8003860C8002850C8001860B800C8894
:10B46000088B8F8BFFFFFFFF90EC5BF0120000005A
:10B47000849083C083FF80948084120085C000F094
:10B48000016A00C086F084C087F0848086C083FF94
:10B490008094808487C083FF8094808412008EC053
:10B4A00083FF809480848094808412007AC083FF1C
:10B4B000809480847BC083FF80948084120000018C
:10B4C000350E836FD5DF00017D510001846F856BE0
:10B4D0000001D89084378537D1DF0001360E836FA5
:10B4E000C7DF00013F0E846F010E856FC7DF0001CB
:10B4F000370E836FBDDF00017C510001846F856BC7
:10B50000020E00017E5D07E13A0E00018427000E65
:10B510000001852310D000017E0507E1200E000107
:10B520008427000E0001852306D0180E0001842711
:10B53000000E0001852300018407000E855B0001D9
:10B54000EF0ED8808455000E855504E2EF0E000101
:10B55000846F856B7CC000F000C001F0006A005071
:10B560000001841301500001851388DF0001200EC3
:10B57000836F7EDF00017C510001846F856B7EDF6D
:10B580000001210E836F74DF00017D510001846F83
:10B59000856B0001D8908437853770DF1200200E4C
:10B5A0000001825D03E10001B60E826F000182514D
:10B5B0007E0803E2220E0001825F210E0001825DFF
:10B5C00004E300018251A30803E20001820E826FAE
:10B5D000210E0001825DF66EF76AD890F636F736D6
:10B5E0009A0EF626A30EF7220900F5CF88F00A007E
:10B5F000F5CF89F000018229DF0FF66EF76AD89047
:10B60000F636F7369A0EF626A30EF7220900F5CF86
:10B610008AF00A00F5CF8BF01200270E0001825D40
:10B6200003E100013B0E826F220E0001825D03E107
:10B6300000013C0E826F6D0E0001825D03E100018E
:10B640003D0E826F200E0001825D03E100013E0E7F
:10B65000826F2E0E0001825D04E3000182513E08DC
:10B6600003E200013E0E826F2E0E0001825DF66E37
:10B67000F76AD890F636F736000EF626A00EF722B7
:10B680000900F5CF88F00A00F5CF89F00001822982
:10B69000D20FF66EF76AD890F636F736000EF62619
:10B6A000A00EF7220900F5CF8AF00A00F5CF8BF043
:10B6B0001200200E0001825D03E100012F0E826F57
:10B6C0002E0E0001825D04E300018251390803E27D
:10B6D00000012F0E826F2E0E0001825DF66EF76A5A
:10B6E000D890F636F736A00EF6269F0EF722090000
:10B6F000F5CF88F00A00F5CF89F000018229D20F3A
:10B70000F66EF76AD890F636F736A00EF6269F0E3C
:10B71000F7220900F5CF8AF00A00F5CF8BF012006E
:10B7200000017C51006E016A013404E20050E60819
:10B73000000E015403E20001E60E7C6F00017D5112
:10B74000006E016A013404E200509B08000E0154AF
:10B7500003E200019B0E7D6FB2DE0001220E836FBB
:10B7600087DE84800001816B00018151EA6A600FED
:10B77000E96E000EEA22EFCF82F00001825106E16D
:10B7800000013A0E826F0001190E816FF86A000104
:10B79000825101E1DCD01A0E0001815D01E3D7D0B6
:10B7A000020E00017E5D02E184DF06D000017E050D
:10B7B00002E133DF01D0F3DE00018E6B88C08CF034
:10B7C00089C08DF000018A5100018C5D00018B5110
:10B7D00000018D5901E3AFD0020E00017E5D1DE135
:10B7E0008CC0F6FF8DC0F7FF010E0F0B05E0D8905F
:10B7F000F732F632E806FBE1010ED890F636F7365E
:10B80000E806FBE1000EF6269A0EF7220900F5CFB6
:10B8100084F00A00F5CF85F03CD000017E051DE1E3
:10B820008CC0F6FF8DC0F7FF010E0F0B05E0D8901E
:10B83000F732F632E806FBE1010ED890F636F7361D
:10B84000E806FBE1240EF626A00EF7220900F5CF4C
:10B8500084F00A00F5CF85F01CD08CC0F6FF8DC0B7
:10B86000F7FF010E0F0B05E0D890F732F632E8062D
:10B87000FBE1010ED890F636F736E806FBE1880EBC
:10B88000F626A40EF7220900F5CF84F00A00F5CFC2
:10B8900085F000018C51010B05E00001845100018D
:10B8A000806F05D085C000F0016A00C080F0000103
:10B8B0008051006E016A0050800B1DE07F0E000178
:10B8C000805F00017F5109E000018051000804E21F
:10B8D00000018007EBDDF8D70DD08EC083FF00019B
:10B8E0008051000807E200018007809480848094E2
:10B8F0008084F5D71BD00001802B00017F510EE022
:10B900008EC083FF00018051000807E2000180071C
:10B910008094808480948084F5D708D00001805181
:10B92000000804E200018007C1DDF8D700018C2B7C
:10B93000000E8D2347D70001812B00018151EA6A57
:10B94000600FE96E000EEA22EFCF82F020D70001EF
:10B95000836B8EDD1200FFFFFFFFFFFFFFFFFFFF86
:10B96000FFFFFFFFFFFFFFFFFFFFFFFFFFFFFFFFE7
:10B97000FFFFFFFFFFFFFFFFFFFFFFFFFFFFFFFFD7
:10B98000FFFFFFFFFFFFFFFFFFFFFFFFFFFFFFFFC7
:10B99000FFFFFFFFFFFFFFFFFFFFFFFFFFFFFFFFB7
:10C000000901306B316B326B336B3451040B04E03C
:10C01000080E346F356B03D0040E346F356B366BFE
:10C02000376B386934C4B5F935C4B6F936C4B7F9D5
:10C0300037C4B8F938C4B9F939C4BAF93AC4BBF944
:10C040003BC4BCF91FC583F91EC584F90CC485F92E
:10C050000DC486F90EC487F90FC488F997C289F90F
:10C0600098C28AF999C28BF99AC28CF99BC28DF950
:10C070009CC28EF99DC28FF99EC290F9EFC591F9CD
:10C08000F0C592F9F1C593F9F2C594F9F3C595F9A4
:10C09000F4C596F9F5C597F9F6C598F9F7C599F974
:10C0A000F8C59AF9F9C59BF9FAC59CF95FC99DF9DC
:10C0B00060C99EF961C99FF962C9A0F963C9A1F974
:10C0C00064C9A2F965C9A3F966C9A4F96FC9A5F93C
:10C0D00070C9A6F971C9A7F972C9A8F977C9A9F9F0
:10C0E00078C9AAF979C9ABF97AC9ACF97BC9ADF9B4
:10C0F0007CC9AEF97DC9AFF97EC9B0F97FC9B1F984
:10C1000080C9B2F981C9B3F982C9B4F905011F51D7
:10C1100002E0090130812C6A2D6A2E6A2F6AEFC570
:10C1200027F0F0C528F0F1C529F0F2C52AF0C2ECDD
:10C130006EF0010A02E009013083100E0901BE6FA2
:10C14000BF6B200EBFAF02D0D89003D0BE5D000EF3
:10C15000BF592DE2BEC9E9FFBFC9EAFFD890E93651
:10C16000EA36D890E936EA36800EE926040EEA224D
:10C17000EECF00F0EECF01F0EECF02F0EFCF03F004
:10C180002C6A2D6A2E6A2F6A00C027F001C028F0A1
:10C1900002C029F003C02AF0C2EC6EF0010A02E0EE
:10C1A000090130850901BE2B000EBF23CAD72C6AB6
:10C1B0002D6A2E6A2F6AF3C527F0F4C528F0F5C55D
:10C1C00029F0F6C52AF0C2EC6EF0010A02E009017E
:10C1D0003087A40E2C6E700E2D6E7D0E2E6E3F0ECF
:10C1E0002F6E77C927F078C928F079C929F07AC964
:10C1F0002AF0D2EC6EF0010A02E109013089660EE4
:10C200002C6E2D6EA60E2E6E3F0E2F6E77C927F068
:10C2100078C928F079C929F07AC92AF0C9EC6EF0FA
:10C22000010A02E10901308B5C0E2C6E8F0E2D6E1F
:10C23000420E2E6E3E0E2F6E97C227F098C228F047
:10C2400099C229F09AC22AF0D2EC6EF0010A02E1FA
:10C250000901308DAE0E2C6E470E2D6E810E2E6EA6
:10C260003F0E2F6E97C227F098C228F099C229F08E
:10C270009AC22AF0C9EC6EF0010A02E10901308F7E
:10C280009A0E2C6E990E2D6E190E2E6E3F0E2F6E7D
:10C290009BC227F09CC228F09DC229F09EC22AF0C2
:10C2A000D2EC6EF0010A02E109013181AE0E2C6E72
:10C2B000470E2D6E810E2E6E3F0E2F6E9BC227F005
:10C2C0009CC228F09DC229F09EC22AF0C9EC6EF0F3
:10C2D000010A02E10901318338C42CF039C42DF080
:10C2E0003AC42EF03BC42FF034C427F035C428F0F4
:10C2F00036C429F037C42AF0F8EC6CF027C000F0FF
:10C3000028C001F029C002F02AC003F0330E2C6EC1
:10C310002D6E730E2E6E3F0E2F6E00C027F001C0E3
:10C3200028F002C029F003C02AF0C9EC6EF0010A1F
:10C3300002E10901318538C42CF039C42DF03AC42A
:10C340002EF03BC42FF034C427F035C428F036C497
:10C3500029F037C42AF0F8EC6CF027C000F028C0B0
:10C3600001F029C002F02AC003F0CD0E2C6ECC0ED5
:10C370002D6E4C0E2E6E3D0E2F6E00C027F001C0AC
:10C3800028F002C029F003C02AF0D2EC6EF0010AB6
:10C3900002E1090131872C6A2D6A800E2E6E3E0E55
:10C3A0002F6E7FC927F080C928F081C929F082C982
:10C3B0002AF0C9EC6EF0010A02E109013189050198
:10C3C0001E51080802E20901318B2C6A2D6A2E6A7F
:10C3D0002F6AA5C927F0A6C928F0A7C929F0A8C9BE
:10C3E0002AF0C2EC6EF0010A2FE063C92CF064C998
:10C3F0002DF065C92EF066C92FF05FC927F060C91E
:10C4000028F061C929F062C92AF0F8EC6CF027C065
:10C4100000F028C001F029C002F02AC003F0330E5A
:10C420002C6E2D6E730E2E6E3F0E2F6E00C027F0F9
:10C4300001C028F002C029F003C02AF0C9EC6EF058
:10C44000010A02E10901318D2C6A2D6A2E6A2F6AD8
:10C45000A5C927F0A6C928F0A7C929F0A8C92AF0BC
:10C46000C2EC6EF0010A30E063C92CF064C92DF013
:10C4700065C92EF066C92FF05FC927F060C928F0A2
:10C4800061C929F062C92AF0F8EC6CF027C000F00D
:10C4900028C001F029C002F02AC003F0CD0E2C6E96
:10C4A000CC0E2D6E4C0E2E6E3D0E2F6E00C027F062
:10C4B00001C028F002C029F003C02AF0D2EC6EF0CF
:10C4C000010A02E10901318F2C6A2D6A400E2E6E9D
:10C4D0002F6E08C427F009C428F00AC429F00BC441
:10C4E0002AF0C9EC6EF0010A02E10901328108C4A8
:10C4F0002CF009C42DF00AC42EF00BC42FF00CC48C
:10C5000027F00DC428F00EC429F00FC42AF0F7EC70
:10C510006CF027C000F028C001F029C002F02AC04A
:10C5200003F0CD0E2C6ECC0E2D6E4C0E2E6E3E0EEC
:10C530002F6E00C027F001C028F002C029F003C010
:10C540002AF0C9EC6EF0010A02E1090132832C6A7B
:10C550002D6A400E2E6E3F0E2F6E0CC427F00DC4B8
:10C5600028F00EC429F00FC42AF0D2EC6EF0010AB4
:10C5700002E1090132857B0E2C6E140E2D6E8E0E9B
:10C580002E6E3F0E2F6E0CC427F00DC428F00EC483
:10C5900029F00FC42AF0C9EC6EF0010A02E109018A
:10C5A0003287330E2C6E2D6E2E6E3F0E2F6E7BC992
:10C5B00027F07CC928F07DC929F07EC92AF0D2EC89
:10C5C0006EF0010A02E109013289AE0E2C6E470EAF
:10C5D0002D6E810E2E6E3F0E2F6E7BC927F07CC90B
:10C5E00028F07DC929F07EC92AF0C9EC6EF0010A55
:10C5F00002E10901328B9BC22CF09CC22DF09DC23E
:10C600002EF09EC22FF097C227F098C228F099C250
:10C6100029F09AC22AF0C9EC6EF0010A02E1090180
:10C62000328D12000901349536951200FF0E090172
:10C63000385D20E10501B80ED88000550B0E01557C
:10C6400019E222C538F938C900F0016A00BE016854
:10C65000FF0E001801E101500DE138C900F0016A38
:10C6600000BE0168FE0E001801E1015002E0000E5C
:10C6700001D0010E1200D9CFE6FFE1CFD9FF0901A9
:10C68000C06BC16B34C42CF035C42DF036C42EF011
:10C6900037C42FF0B5C927F0B6C928F0B7C929F0BB
:10C6A000B8C92AF0C2EC6EF0010A14E138C42CF0CB
:10C6B00039C42DF03AC42EF03BC42FF0B9C927F08D
:10C6C000BAC928F0BBC929F0BCC92AF0C2EC6EF087
:10C6D000010A02E00901C081EFC52CF0F0C52DF080
:10C6E000F1C52EF0F2C52FF091C927F092C928F0BC
:10C6F00093C929F094C92AF0C2EC6EF0010A02E055
:10C700000901C08377C92CF078C92DF079C92EF0C2
:10C710007AC92FF0A9C927F0AAC928F0ABC929F016
:10C72000ACC92AF0C2EC6EF0010A14E17BC92CF00E
:10C730007CC92DF07DC92EF07EC92FF0ADC927F040
:10C74000AEC928F0AFC929F0B0C92AF0C2EC6EF02A
:10C75000010A02E00901C08905011F510901835D39
:10C7600001E0C08B0CC42CF00DC42DF00EC42EF0D3
:10C770000FC42FF085C927F086C928F087C929F092
:10C7800088C92AF0C2EC6EF0010A02E00901C08DEE
:10C790003AD0100E0901BE6FBF6B200EBFAF02D0A2
:10C7A000D89003D0BE5D000EBF592DE2BEC9E9FF8F
:10C7B000BFC9EAFFD890E936EA36D890E936EA36BA
:10C7C000800EE926040EEA22EECF00F0EECF01F053
:10C7D000EECF02F0EFCF03F02C6A2D6A2E6A2F6A9B
:10C7E00000C027F001C028F002C029F003C02AF0E1
:10C7F000C2EC6EF0010A02E00901C08F0901BE2BF4
:10C80000000EBF23CAD7F7C52CF0F8C52DF0F9C527
:10C810002EF0FAC52FF099C927F09AC928F09BC9C4
:10C8200029F09CC92AF0C2EC6EF0010A02E009016D
:10C83000C1816FC92CF070C92DF071C92EF072C979
:10C840002FF0A5C927F0A6C928F0A7C929F0A8C9C3
:10C850002AF0C2EC6EF0010A28E15FC92CF060C931
:10C860002DF061C92EF062C92FF09DC927F09EC935
:10C8700028F09FC929F0A0C92AF0C2EC6EF0010A85
:10C8800014E163C92CF064C92DF065C92EF066C9A6
:10C890002FF0A1C927F0A2C928F0A3C929F0A4C983
:10C8A0002AF0C2EC6EF0010A02E00901C1837FC9DF
:10C8B0002CF080C92DF081C92EF082C92FF0B1C9AA
:10C8C00027F0B2C928F0B3C929F0B4C92AF0C2ECE4
:10C8D0006EF0010A02E00901C18505011E5109013E
:10C8E000845D01E0C18797C22CF098C22DF099C2F7
:10C8F0002EF09AC22FF089C927F08AC928F08BC977
:10C9000029F08CC92AF0C2EC6EF0010A14E19BC236
:10C910002CF09CC22DF09DC22EF09EC22FF08DC92E
:10C9200027F08EC928F08FC929F090C92AF0C2ECEF
:10C930006EF0010A02E00901C1892C6A2D6A500ECD
:10C940002E6E410E2F6E08C427F009C428F00AC4C9
:10C9500029F00BC42AF0C9EC6EF0010A02E10901CA
:10C96000C18D08C42CF009C42DF00AC42EF00BC4EC
:10C970002FF00CC427F00DC428F00EC429F00FC40A
:10C980002AF0F7EC6CF027C000F028C001F029C0B5
:10C9900002F02AC003F0CD0E2C6ECC0E2D6E4C0E84
:10C9A0002E6E3E0E2F6E00C027F001C028F002C090
:10C9B00029F003C02AF0C9EC6EF0010A02E1090176
:10C9C000C18FFE0EDB5006E00901C0513613C15184
:10C9D000371305D00901C0513413C1513513E55245
:10C9E000E7CFD9FF1200E66A46DEE5521200010EDB
:10C9F000E66E41DEE55212000201706B05011F0573
:10CA000001E0D7D30201925101E04CD1F00E2C6E1F
:10CA1000850E2D6E990E2E6E3E0E2F6EBBC227F028
:10CA2000BCC228F0BDC229F0BEC22AF08EEC6DF067
:10CA300027C014F428C015F429C016F42AC017F42E
:10CA4000A40E2C6E700E2D6E7D0E2E6E3F0E2F6E70
:10CA500014C427F015C428F016C429F017C42AF00E
:10CA6000F8EC6CF093EC6EF028C004F429C005F4E7
:10CA700004011F0ED8800455000E055503E21F0E59
:10CA8000046F056B000E045D000E055902E2046B95
:10CA9000056B04C4C6F2030E0201C603F3CFC5F250
:10CAA000C5C229F0D1EC6CF027C000F028C001F01D
:10CAB00029C002F02AC003F0960E2C6EB20E2D6E25
:10CAC000CC0E2E6E3D0E2F6E00C027F001C028F058
:10CAD00002C029F003C02AF0E1EC6DF027C014F485
:10CAE00028C015F429C016F42AC017F47FC92CF009
:10CAF00080C92DF081C92EF082C92FF014C427F00F
:10CB000015C428F016C429F017C42AF0F8EC6CF00C
:10CB100027C000F028C001F029C002F02AC003F0AD
:10CB20000CC42CF00DC42DF00EC42EF00FC42FF049
:10CB300000C027F001C028F002C029F003C02AF08D
:10CB4000F8EC6CF027C0E8F228C0E9F229C0EAF25C
:10CB50002AC0EBF20201C65105E1A76BA86BA96BD5
:10CB6000AA6B26D0C6C229F0D1EC6CF027C000F029
:10CB700028C001F029C002F02AC003F000C02CF048
:10CB800001C02DF002C02EF003C02FF09FC227F08D
:10CB9000A0C228F0A1C229F0A2C22AF08EEC6DF04A
:10CBA00027C0A7F228C0A8F229C0A9F22AC0AAF279
:10CBB0002C6A2D6A2E6A2F6AA7C227F0A8C228F015
:10CBC000A9C229F0AAC22AF0D2EC6EF0010A05E14E
:10CBD0000201A76BA86BA96BAA6B9FC22CF0A0C225
:10CBE0002DF0A1C22EF0A2C22FF0A7C227F0A8C23A
:10CBF00028F0A9C229F0AAC22AF0C9EC6EF0010AF5
:10CC000008E19FC2A7F2A0C2A8F2A1C2A9F2A2C2E3
:10CC1000AAF22C6A400E2D6E1C0E2E6E460E2F6E42
:10CC2000A7C227F0A8C228F0A9C229F0AAC22AF0F8
:10CC3000E1EC6DF093EC6EF028C042F229C043F2B3
:10CC40002C6A2D6A7A0E2E6E440E2F6EE8C227F0E3
:10CC5000E9C228F0EAC229F0EBC22AF0E1EC6DF05B
:10CC600093EC6EF028C048F229C049F22C6A2D6A74
:10CC70007A0E2E6E440E2F6EAFC227F0B0C228F08F
:10CC8000B1C229F0B2C22AF0E1EC6DF093EC6EF083
:10CC900028C04AF229C04BF2C6C24EF20201010E70
:10CCA000926FC76BC75153E1C6C2C7F2C7C229F022
:10CCB000D1EC6CF027C004F028C005F029C006F0C4
:10CCC0002AC007F0A7C22CF0A8C22DF0A9C22EF0EE
:10CCD000AAC22FF004C027F005C028F006C029F032
:10CCE00007C02AF0E1EC6DF027C000F028C001F089
:10CCF00029C002F02AC003F000C02CF001C02DF0C2
:10CD000002C02EF003C02FF09BC227F09CC228F077
:10CD10009DC229F09EC22AF0F7EC6CF027C0A3F266
:10CD200028C0A4F229C0A5F22AC0A6F20201C75168
:10CD3000EA6A700FE96E020EEA22EF500401046FF6
:10CD4000056B04C408F30301210E096F04D0010E22
:10CD50000401046F056B0401010E041901E1055182
:10CD600001E091D10201C7050401046F056B010EBA
:10CD7000041901E1055101E07FD0C3C228F0C4C20B
:10CD800029F004C42DF005C42EF04EEC6EF026C040
:10CD900004F027C005F004C028F005C029F0E2EC3B
:10CDA0006CF027C000F028C001F029C002F02AC0B2
:10CDB00003F0960E2C6EB20E2D6ECC0E2E6E3D0E26
:10CDC0002F6E00C027F001C028F002C029F003C078
:10CDD0002AF0E1EC6DF027C014F428C015F429C046
:10CDE00016F42AC017F42C6A2D6A400E2E6E2F6E90
:10CDF000A7C227F0A8C228F0A9C229F0AAC22AF027
:10CE00008EEC6DF027C000F028C001F029C002F0C0
:10CE10002AC003F0C3C208F0C4C209F0060ED880CD
:10CE20000856000E095608C028F009C029F0E2ECA7
:10CE30006CF027C004F028C005F029C006F02AC015
:10CE400007F004C02CF005C02DF006C02EF007C07E
:10CE50002FF000C027F001C028F002C029F003C065
:10CE60002AF0E1EC6DF027C0ABF228C0ACF229C08B
:10CE7000ADF22AC0AEF25FD0045105111FE1146B70
:10CE8000156B166B176BA3C22CF0A4C22DF0A5C2B4
:10CE90002EF0A6C22FF09BC227F09CC228F09DC2A4
:10CEA00029F09EC22AF0F7EC6CF027C0ABF228C044
:10CEB000ACF229C0ADF22AC0AEF23DD0030E286E0E
:10CEC000296A04C42DF005C42EF04EEC6EF026C085
:10CED00004F027C005F004C028F005C029F0E2ECFA
:10CEE0006CF027C000F028C001F029C002F02AC071
:10CEF00003F0960E2C6EB20E2D6ECC0E2E6E3D0EE5
:10CF00002F6E00C027F001C028F002C029F003C036
:10CF10002AF0E1EC6DF027C014F428C015F429C004
:10CF200016F42AC017F4A7C2ABF2A8C2ACF2A9C289
:10CF3000ADF2AAC2AEF20CC42CF00DC42DF00EC49A
:10CF40002EF00FC42FF014C427F015C428F016C417
:10CF500029F017C42AF0F8EC6CF027C014F428C0AC
:10CF600015F429C016F42AC017F4ABC22CF0ACC2D9
:10CF70002DF0ADC22EF0AEC22FF0A3C227F0A4C296
:10CF800028F0A5C229F0A6C22AF0F8EC6CF027C060
:10CF900004F028C005F029C006F02AC007F0B3C28B
:10CFA0002CF0B4C22DF0B5C22EF0B6C22FF004C0E2
:10CFB00027F005C028F006C029F007C02AF0E1ECF0
:10CFC0006DF027C000F028C001F029C002F02AC08F
:10CFD00003F0AFC22CF0B0C22DF0B1C22EF0B2C23D
:10CFE0002FF000C027F001C028F002C029F003C0D4
:10CFF0002AF0F8EC6CF027C010F428C011F429C016
:10D0000012F42AC013F414C42CF015C42DF016C465
:10D010002EF017C42FF010C427F011C428F012C44A
:10D0200029F013C42AF0C9EC6EF0010A04E10401EE
:10D03000046B056B27D004C4C7F2ABC22CF0ACC2A2
:10D040002DF0ADC22EF0AEC22FF0A3C227F0A4C2C5
:10D0500028F0A5C229F0A6C22AF0F8EC6CF027C08F
:10D06000A3F228C0A4F229C0A5F22AC0A6F20201A8
:10D07000C751EA6A700FE96E020EEA22EF5004010E
:10D08000046F056B68D60201C751000801E386D022
:10D09000F00E006E850E016E990E026E3E0E036E4E
:10D0A000C7C229F0D1EC6CF027C004F028C005F00D
:10D0B00029C006F02AC007F004C02CF005C02DF0EE
:10D0C00006C02EF007C02FF000C027F001C028F0E6
:10D0D00002C029F003C02AF0E1EC6DF027C014F47F
:10D0E00028C015F429C016F42AC017F47FC92CF003
:10D0F00080C92DF081C92EF082C92FF014C427F009
:10D1000015C428F016C429F017C42AF0F8EC6CF006
:10D1100027C000F028C001F029C002F02AC003F0A7
:10D120000CC42CF00DC42DF00EC42EF00FC42FF043
:10D1300000C027F001C028F002C029F003C02AF087
:10D14000F8EC6CF027C020F428C021F429C022F4A8
:10D150002AC023F40201C70505E1C3C2BFF2C4C25D
:10D16000C0F205D0030EC703F350BF6FC06B210E92
:10D170000301095D12E1C7C209F30201C751EA6A5E
:10D18000700FE96E020EEA22EFCF0AF303010C29B9
:10D190000C6F640E0C5D01E10C6B0AD00CC420F422
:10D1A0000DC421F40EC422F40FC423F4BF6BC06B72
:10D1B000E8D00CC42CF00DC42DF00EC42EF00FC41A
:10D1C0002FF074C427F075C428F076C429F077C412
:10D1D0002AF0F7EC6CF027C010F428C011F429C035
:10D1E00012F42AC013F42C6A2D6A2E6A2F6A10C416
:10D1F00027F011C428F012C429F013C42AF0D2EC8D
:10D200006EF0010A01E1B2D0F00E2C6E850E2D6E8B
:10D21000990E2E6E3E0E2F6E10C427F011C428F00A
:10D2200012C429F013C42AF08EEC6DF027C010F45C
:10D2300028C011F429C012F42AC013F4A40E2C6ED5
:10D24000700E2D6E7D0E2E6E3F0E2F6E10C427F0C9
:10D2500011C428F012C429F013C42AF0F8EC6CF0C1
:10D2600093EC6EF028C0BFF229C0C0F2030E286E06
:10D27000296ABFC22DF0C0C22EF04EEC6EF026C05F
:10D28000BFF227C0C0F20201BF51C01109E10CC4B6
:10D2900020F40DC421F40EC422F40FC423F465D08D
:10D2A000C351BF5DC451C05904E2C3C2BFF2C4C27E
:10D2B000C0F2BFC228F0C0C229F0E2EC6CF027C077
:10D2C00000F028C001F029C002F02AC003F0960E39
:10D2D0002C6EB20E2D6ECC0E2E6E3D0E2F6E00C03B
:10D2E00027F001C028F002C029F003C02AF0E1ECC9
:10D2F0006DF027C010F428C011F429C012F42AC020
:10D3000013F47FC92CF080C92DF081C92EF082C999
:10D310002FF010C427F011C428F012C429F013C450
:10D320002AF0F8EC6CF027C000F028C001F029C00A
:10D3300002F02AC003F00CC42CF00DC42DF00EC472
:10D340002EF00FC42FF000C027F001C028F002C05B
:10D3500029F003C02AF0F8EC6CF027C020F428C0B4
:10D3600021F429C022F42AC023F40BD00CC420F4E9
:10D370000DC421F40EC422F40FC423F40201BF6BC8
:10D38000C06B120005011F051DE1200E0401046F92
:10D39000056B006B0451005D000E055513E2005152
:10D3A000EA6AC80FE96E020EEA22EF50E66E0051FB
:10D3B000EA6A500FE96E020EEA22E552E750EF6E7C
:10D3C000002BE8D7120005011F050EE10401006BD8
:10D3D000200E005D09E20051EA6AC80FE96E020EF4
:10D3E000EA22EF6A002BF4D7120005011F0523E1A2
:10D3F0000201C751EA6AC80FE96E020EEA22EF5035
:10D40000006E016AD890015004E6FF0E005C000E29
:10D41000015811E2C751EA6AC80FE96E020EEA220A
:10D42000EF28E66EC751EA6AC80FE96E020EEA22DB
:10D43000E552E750EF6E120005011F0501E145D0EE
:10D440002C6A2D6A2E6A2F6A2CC427F02DC428F06E
:10D450002EC429F02FC42AF0D2EC6EF0010A1BE191
:10D460007BC92CF07CC92DF07DC92EF07EC92FF030
:10D470002CC427F02DC428F02EC429F02FC42AF084
:10D48000E1EC6DF027C02CF428C02DF429C02EF457
:10D490002AC02FF41AD077C92CF078C92DF079C999
:10D4A0002EF07AC92FF02CC427F02DC428F02EC4FA
:10D4B00029F02FC42AF0E1EC6DF027C02CF428C02D
:10D4C0002DF429C02EF42AC02FF412000001130EEF
:10D4D0008A6F1C0E8B6F976BF50E986F996B9A6B1A
:10D4E000300E9B6F390E9C6F86EF6AF000010C0EB8
:10D4F0008A6F100E8B6F976BE10E986F996B9A6B1A
:10D500002E0E9B6F3E0E9C6F86EF6AF00001906BB3
:10D5100090C0DEFF84820001706B0001875103E13F
:10D520000001010E876F0001865103E10001010E29
:10D53000866F00018B510001D880885502E28BC0B4
:10D5400088F00001875100018825410806E2410E5C
:10D550000001D88087550001886F86C092F00001D5
:10D56000916B00019151912BEA6A600FE96E000EF8
:10D57000EA22EFCF93F05BD80001906B0001010E1F
:10D58000946F0001935152E00001940501E1F1D83C
:10D59000FFD8010E000194190001946F0001940559
:10D5A00008E1CED8400E0001925D02E20001922B0C
:10D5B000A5D90001902B040E0001905D02E2000E3F
:10D5C00001D0010E036E3C0E0001935D02E0000EDF
:10D5D00001D0010E026E3A0E0001935D02E0000ED2
:10D5E00001D0010E016E2E0E0001935D02E0000ECF
:10D5F00001D0010E011002100314006E00018A51C7
:10D600000001905D02E2000E01D0010E00100DE05D
:10D6100000019151912BEA6A600FE96E000EEA2237
:10D62000EFCF93F004D80001906BABD7120000014C
:10D630009C51D880935502E3000E01D0010E006E7C
:10D640009B51935D02E3000E01D0010E001006E035
:10D650008C6B8D6B8E6B8F6B956B71D09B51935DCB
:10D660008C6F8D6B8E6B8F6B8B29FE0BE842006E7F
:10D67000016A026A036A8CC026F08DC027F08EC052
:10D6800028F08FC029F000C02BF001C02CF002C0A0
:10D690002DF003C02EF048EC70F022C08CF023C0B7
:10D6A0008DF024C08EF025C08FF08AC000F0016A92
:10D6B000026A036A8CC026F08DC027F08EC028F065
:10D6C0008FC029F000C02BF001C02CF002C02DF05B
:10D6D00003C02EF048EC70F022C08CF023C08DF017
:10D6E00024C08EF025C08FF0000197518C279851EF
:10D6F0008D2399518E239A518F233C0E935D02E026
:10D70000000E01D0010E016E3A0E935D02E0000E94
:10D7100001D0010E006E2E0E935D02E0000E01D0CE
:10D72000010E001001100BE08B51E824006E000187
:10D73000005000018C27000E8D238E238F231200B2
:10D740000001750E966FF0D800018705966FECD832
:10D7500000013F0E966FE8D80001150E966FE4D8D1
:10D7600000019205966FE0D800019205966F94EF44
:10D770006CF00001956B8851955D09E29551EA6A5C
:10D78000000FE96E080EEA22EF6A952BF4D712001B
:10D7900000018C518D118E118F1101E1AED000016D
:10D7A0008C510001956F95C0F6FF8DC000F08EC0C2
:10D7B00001F08FC002F00001036A00500001956F74
:10D7C00095C0F7FF8EC000F08FC001F00001026A23
:10D7D000036A00500001956F95C0F8FF0001956B3A
:10D7E000000188510001955D01E37AD00900F5CF71
:10D7F00096F0000189511CE000018939F00B006EA0
:10D80000F00E00019615005C07E200018939F00B6B
:10D810000001965D0001966F0F0E00019615000144
:10D82000895D06E2000189510001965D0001966F55
:10D83000000194051EE1F00E00019615E66E000150
:10D840009551EA6A000FE96E080EEA22E552E750A8
:10D85000EF6E00019639F00BF00BE66E0001952992
:10D86000EA6A000FE96E080EEA22E552E750EF6E11
:10D8700033D0000196390F0B0F0B006E000195514C
:10D88000EA6A000FE96E080EEA22EF50F00B001072
:10D89000E66E00019551EA6A000FE96E080EEA2271
:10D8A000E552E750EF6E0F0E00019615006E000175
:10D8B0009529EA6A000FE96E080EEA22EF50F00B94
:10D8C0000010E66E00019529EA6A000FE96E080E65
:10D8D000EA22E552E750EF6E020E0001952780D74D
:10D8E00000018B29FE0BE842006E00010050000190
:10D8F0008C27000E8D238E238F231200848200013B
:10D90000956B000188510001955D0DE20001955174
:10D91000EA6A000FE96E080EEA22EFCF96F007D808
:10D920000001952BEED71200849201D8120001015C
:10D9300084900001839096BF8382839096AF8392F8
:10D94000838096BD8382839096AD8392838096BBBD
:10D950008382839096AB8392838096B983828390EF
:10D9600096A98392838096B78382839096A78392A9
:10D97000838096B58382839096A58392838096B3A5
:10D980008382839096A38392838096B183828390CF
:10D9900096A1839283808480010100010001966B2F
:10D9A0001200219E05D0219E29AE02D0296C218E25
:10D9B00029C023F0226A336A326A860E246E256AF1
:10D9C0004CEF6FF0219E08D0219E29AE05D0286C27
:10D9D000291EE86A2922218E29C023F028C022F0BE
:10D9E000336A326A8E0E246E256A4CEF6FF02F7EFA
:10D9F000216A88EC6FF0A0EC6FF021B630EF6FF089
:10DA000021A20AD021AA03D021BE30EF6FF021A4B9
:10DA10003CEF6FF039EF6FF021AA05D021AC3CEF5D
:10DA20006FF039EF6FF021A00AD021A808D021BEF5
:10DA300004D021A402D045EF6FF049EF6FF0326AB5
:10DA4000256A2F502A5C316E10E327C033F028C0BE
:10DA500022F029C023F02AC030F02CC027F02DC0BE
:10DA600028F02EC029F0213A09D02CC033F02DC067
:10DA700022F02EC023F02FC030F0316C219E21BC4B
:10DA8000218E30C024F021B078EF6FF01A0E316093
:10DA900078EF6FF0246A2A6A21A408D0276C281E28
:10DAA000291E2A1EE86A282229222A2221AC08D00F
:10DAB000336C221E231E241EE86A222223222422E3
:10DAC000266A315207E02A34293228322732263298
:10DAD000312EF9D7275033262850222229502322CD
:10DAE0002A50242226C032F0219E24AE0BD0326C64
:10DAF000331E221E231E241EE86A332222222322E2
:10DB00002422218E24A006D0D88023322232333220
:10DB10003232302A30C024F04CEF6FF0216A88ECAA
:10DB20006FF0A0EC6FF021B630EF6FF021A205D0BE
:10DB300021BA30EF6FF037EF6FF021BA43EF6FF09B
:10DB400021A005D021B830EF6FF043EF6FF021B87E
:10DB500037EF6FF0256A7F0E2A24246EE86A2522AB
:10DB60002F50245EE86A255A1A0E306E2A6A326AED
:10DB7000336A226A236A2C50275E2D50285A2E5071
:10DB8000295A000E2A5A09E72C5027262D50282200
:10DB90002E502922000E2A2201D0328AD890273610
:10DBA000283629362A36D89032363336223623366E
:10DBB000302EE1D7295028102710D8A4328A4CEFF4
:10DBC0006FF0216A88EC6FF0A0EC6FF021B630EFB7
:10DBD0006FF021A205D021B830EF6FF037EF6FF072
:10DBE00021AA05D021B030EF6FF037EF6FF021B0F0
:10DBF00002D021A802D043EF6FF0256A2F502A24CB
:10DC0000246EE86A25227E0E245EE86A255A326A6E
:10DC1000336A226A236A2E502902F4CF23F0F3CF0D
:10DC200022F02D502902F3503326F4502222000E08
:10DC300023222E502802F3503326F4502222000EC5
:10DC400023222C502902F3503226F4503322000EA6
:10DC5000222223222D502802F3503226F450332260
:10DC6000000E222223222E502702F3503226F45097
:10DC70003322000E222223222C502802F450322676
:10DC8000000E3322222223222D502702F450322666
:10DC9000000E3322222223224CEF6FF028C032F0F4
:10DCA00028502D02F4CF27F0F3CF26F029502E0272
:10DCB000F4CF29F0F3CF28F02D02F3502726F450AB
:10DCC0002822E86A292232502E02F3502726F450E7
:10DCD0002822E86A2922000C216A88EC6FF021B61C
:10DCE00076EF6EF021A20AD021B403D07F0E296E08
:10DCF00019D0800E296E16D0296A14D021B0FCD715
:10DD0000870E2A60F1D77E0E2A64F6D7860E2A5C2B
:10DD100004E0D89029322A2AF9D721A403D0296C0B
:10DD200029AEEAD71200216A88EC6FF021B69DEF88
:10DD30006EF021A20ED021B405D07F0E296EFF0E09
:10DD4000286E1FD0800E296E286A1BD0296A286A87
:10DD500018D021B0FBD78F0E2A60EDD77E0E2A6433
:10DD6000F5D78E0E2A5C05E0D890293228322A2A6F
:10DD7000F8D721A406D0286C291EE86A292229AEEA
:10DD8000E5D71200DBEC6EF021B6000C21B0010CDF
:10DD9000000CDBEC6EF021B6000C21B0000C21B4BD
:10DDA000000C010CDBEC6EF021B6000C21B0000C75
:10DDB00021A4000C010C216A88EC6FF0A0EC6FF03C
:10DDC00021B6120021AE08D021A004D021A802D093
:10DDD00021801200219012002F502A5C0BE12E505E
:10DDE000295C08E12D50285C05E12C50275C02E1FC
:10DDF00021801200D8A002D0218E10D02A502FC02E
:10DE00002AF02F6E29502EC029F02E6E28502DC0DA
:10DE100028F02D6E27502CC027F02C6E2F502A5C36
:10DE200010E0FF0F09E0219021B403D021AE21843E
:10DE3000120021AE219412002F2AD8902E322D32BA
:10DE40002C322C50275E2D50285A2E50295A29BE8C
:10DE5000EAD7D8902736283629362A2EF8D7C8D7B9
:10DE60007F0E2A6EFF0E296E286E276E12007F0E1F
:10DE700021BEFF0E2A6E02D07F0E2A6E800E296E02
:10DE8000286A276AF3D721AE04D0800E2A6E296A49
:10DE9000F7D72A6A296AF4D7235022103310321098
:10DEA000F8E025BEF0D723BE0CD024502510EBE0BF
:10DEB000D89032363336223623362406D8A02506AB
:10DEC000F2D72550D4E12428D2E032AE11D07F0E13
:10DED000321402E133A00CD0332AE86A2222232232
:10DEE00007E3D880233222323332242A2428BFE0A9
:10DEF0002450C9E033C027F022C028F02334296E13
:10DF000024302A6E29322A9E21BE2A8E36EF6FF0E7
:10DF100029362A3602E32184217E06E121802A6AFD
:10DF2000296A286A276A12002A2803E0D880293241
:10DF30001200D890293202E12182120021861200BB
:10DF40002E362F3602E3218C217E06E121882F6AAE
:10DF50002E6A2D6A2C6A12002F2803E0D8802E32F8
:10DF60001200D8902E32EAE1218A1200D9CFE6FFC2
:10DF7000DACFE6FFE1CFD9FFE2CFDAFF0C0EE124E2
:10DF800002E3E168E652E16ED950FA0FE96EFF0E46
:10DF9000DA20EA6E010EEECFDBFF020EEECFDBFFE2
:10DFA000030EEECFDBFF040EEECFDBFF63D8D950BC
:10DFB000010FE96E000EDA20EA6EEECFE6FFEECF3B
:10DFC000E6FFEECFE6FFEFCFE6FF72EC80F0006EEB
:10DFD000060EE15C02E2E16AE552E16E0050DF6E9E
:10DFE000850EDF1404E04DD8EE6AED6A23D0090EE9
:10DFF000DBCF00F00A0EDBCF01F0820E0026FF0E11
:10E0000001223FD800C0EEFF01C0EDFF7E0EF36E8F
:10E01000090EF3CFDBFF0A0EDB6AD950010FE66E63
:10E02000000EDA20E66E26D82DEC76F0E552E552A9
:10E03000E552E552010EDBCF00F0020EDBCF01F01E
:10E04000030EDBCF02F0040EDBCF03F000C026F09E
:10E0500001C027F002C028F003C029F00C0EE15CDB
:10E0600002E2E16AE552E16EE552E5CFDAFFE7CF81
:10E07000D9FF1200D950050FE66E000EDA20E66EC9
:10E080001200F80EDBCFE9FFF90EDBCFEAFF12003A
:10E0900026502B02F3CF22F0F4CF23F02C02F350C2
:10E0A0002326000EF420246E26502D02F350242641
:10E0B000000EF420256E26502E02F3502526275000
:10E0C0002B02F3502326F4502422000E2522275041
:10E0D0002C02F3502426F450252227502D02F35011
:10E0E000252628502B02F3502426F45025222850B0
:10E0F0002C02F350252629502B02F350252612001E
:10E10000000000000000000000000000000000000F
:10E1100000000000000000000000000000000000FF
:10E1200000000000000009800000000000006FF007
:10E130000000000000003FE00000000000000000C0
:10E1400000000000000000000000000000000000CF
:10E1500000000000000000000000000000000000BF
:10E16000000000000000000000000000000000208F
:10E170000000000000003AF000000000004BFFA08B
:10E18000000000005CFF91000000006DFE710000C7
:10E1900000017EFD60000000018FFD5000000000C6
:10E1A0009FFB400000000000FA300000000000006B
:10E1B000200000000000000000000000000000003F
:10E1C0000000000000000000000169BCCA720000ED
:10E1D000009FFEDCDFFFB2001DF8200005FDFF30D0
:10E1E000AF3000009F902ED0F800002CF50006F014
:10E1F000F80004ED300005F0AF308FB100000CE006
:10E200001DFDF8000016DF40009FFFDCDEFFC300AD
:10E21000000169BCCA73000000000000000000009B
:10E2200000000000000000000000000000000000EE
:10E2300002900000000001300AB00000000004F06D
:10E240002F600000000004F0AF977777777779F0C0
:10E25000FFFFFFFFFFFFFFF012222222222226F003
:10E2600000000000000004F000000000000003D0E7
:10E27000000000000000000000000000000000009E
:10E28000000000000000000000000000000001404D
:10E2900007D0000000007FF04F800000001CFEF05F
:10E2A000CC00000002EF57F0F70000002EE207F06C
:10E2B000F8000001DE2007F0CE10002DE20007F08C
:10E2C0004FD658FE300007F006FFFFB1000007F000
:10E2D0000014520000000580000000000000000053
:10E2E000000000000000000000000000000002002C
:10E2F0000920000000007F506F40000000002ED079
:10E30000DB000059000007F0F800008E000004F068
:10E31000EA0000CF100006F09F3007FF90001EE0DB
:10E320001EFCDF87FB79EF50019DC6007EFFD50004
:10E3300000000000002100000000000000000000BC
:10E340000000000000000000000000002BB00000F2
:10E3500000000006FFE00000000002CF69E00000BE
:10E3600000007FB109E00000002CE60009E0000099
:10E3700007FB100009E00000CFFCCCCCCEFDDDD0C7
:10E38000DEEEEEEEEFFEEEE00000000009E0000041
:10E390000000000008C000000000000000000000B5
:10E3A000000000000000000000000000000012005B
:10E3B00078ABCDED0000CE20FFEDCCFA00005FB0D1
:10E3C000F90006F0000008F0F9000AB0000004F0BF
:10E3D000F9000AC0000004F0F90008F300000BF097
:10E3E000F90001FE6213BF90F900004EFFFFFB0031
:10E3F000110000016AA940000000000000000000B8
:10E40000000000000000000000000356653000001E
:10E41000004BFFFFFFFFA20008FE968F956AFF30BA
:10E420006F9001F800003ED0EC0008F0000006F00C
:10E43000F6000AE0000004F0F70007F3000009F01E
:10E44000CD1001EF7213AF904D20002DFFFFF900AA
:10E4500000000000478610000000000000000000DF
:10E46000000000000000000011000000000000009B
:10E47000FA00000000000000FA0000000000049014
:10E48000FA0000000039EFF0FA0000017DFFE940DA
:10E49000FA0005BFFF940000FA18EFFB50000000DF
:10E4A000FEFFD71000000000FFB4000000000000D5
:10E4B000520000000000000000000000000000000A
:10E4C0000000000000000000000000000278500082
:10E4D00003ADB4007FFFFC003FFCFF66FA43AFA032
:10E4E000CD101CFE70000BF0F50001FE000005F0E1
:10E4F000F50000BF100004F0EC0007FFB0000AF0C8
:10E500006FD9CF78FB329F9007EFE6009FFFFB00AB
:10E51000000100000388500000000000000000001F
:10E520000000000000000000000355200000000073
:10E5300004DFFFFB10000B604FD7459FD0001CE0AD
:10E54000DD000005F50005F0F7000000F80004F01C
:10E55000F8000000F70008F0BE200006F2005FA0FF
:10E560002EF9547F947CFC0002AFFFFFFFFE700089
:10E570000001467775300000000000000000000038
:10E58000000000000000000000000000000000008B
:10E59000000000000000000000000000000000007B
:10E5A000000006A10000098000001FF900006FF0C4
:10E5B00000000DF500003FE000000010000000002A
:10E5C000000000000000000000000000000000004B
:10E5D000000000000000000000000000000000003B
:10E5E000000000000000000000000000000000002B
:10E5F0000000300000000000BAAEF0000000000093
:10E60000FFE930000000000053000000000000009F
:10E610000000100000000000978CF00000000000D7
:10E62000FFFB50000000000075100000000000001B
:10E6300000000000000000000000000000000000DA
:10E6400000000000000000000000000000000000CA
:10E6500000000000000000000000000000000000BA
:10E660000000000000000000756AE00000000000EB
:10E67000FFFD700000000000A83000000000000056
:10E68000000000000000000000000000000000008A
:10E69000000000000000000000000000000000007A
:10E6A000000000000000000000000000000000006A
:10E6B00000100000000000002CFFA000000000007F
:10E6C000DD78FA0000000000F2005F0000000000AA
:10E6D000F0004F1000000000EA23DC000000000002
:10E6E0004FFFE200000000000154000000000000A5
:10E6F000000000000000000000000000000000001A
:10E7000000001111111111100000FFFFFFFFFFF0B9
:10E7100000009FA7777777700000D6000000000008
:10E720000002F300000000000001FFCBBBBBBBB048
:10E7300000004FFEEEEEEEE00000AB200000000017
:10E740000001F100000000000002FA555555555037
:10E750000000AFFFFFFFFFF00000024444444440CC
:10E76000D9CFE6FFDACFE6FFE1CFD9FFE2CFDAFF7C
:10E77000260EE12402E3E168E652E16ED950050F6E
:10E78000E1D972EC80F0006E060EE15C02E2E16A13
:10E79000E552E16E0050DF6E800EDF5C05E00B0E8F
:10E7A000DB5012E0DF0410E0210E04017C6F7D6B72
:10E7B000010EDB68020EDB68030EDB687F0EF36E72
:10E7C000040EF3CFDBFF8FD1040EDF5C0EE13EDAE7
:10E7D000010EEECFDBFF020EEECFDBFF030EEECF1E
:10E7E000DBFF040EEECFDBFF7ED1DF0410E1210E54
:10E7F00004017C6F7D6B010EDB6A020EDB6A800E0A
:10E80000F36E030EF3CFDBFF040EDB686CD1D9503F
:10E810000C0F98D9B6EC6FF0006E060EE15C02E2C8
:10E82000E16AE552E16E0050FA0E26C0DBFFFB0EF6
:10E8300027C0DBFFFC0E28C0DBFFFD0E29C0DBFF7D
:10E84000A6D9F30E2C6E040E2D6E350E2E6E3F0ED5
:10E8500087D9C9EC6EF0010A09E1B3D984D9F7EC84
:10E860006CF067D9EDD984D9ACD916D00C0EDB0683
:10E870000D0E01E2DB068BD92C6A2D6A2E6A3F0E43
:10E880006FD976D9160EDBCF04F0170EDBCF05F06B
:10E89000180EDBCF06F0190E66D9E1EC6DF049D900
:10E8A000CFD9F8EC6CF01A0E27C0DBFF1B0E28C086
:10E8B000DBFF1C0E29C0DBFF1D0E2AC0DBFF160E7E
:10E8C000DBCF27F0170EDBCF28F0180EDBCF29F0B7
:10E8D000190EDBCF2AF01A0EDBCF2CF01B0EDBCF8C
:10E8E0002DF01C0EDBCF2EF01D0EDBCF2FF08EECAB
:10E8F0006DF01FD9120E27C0DBFF130E28C0DBFFFF
:10E90000140E29C0DBFF150E2AC0DBFF4DD9120EF5
:10E91000DBCF2CF0130EDBCF2DF0140EDBCF2EF05F
:10E92000150E62D90E0E27C0DBFF0F0E28C0DBFFCD
:10E93000100E29C0DBFF110E2AC0DBFF3D0EF36E67
:10E940001E0EF3CFDBFF7E0EF36E1F0EF3CFDBFF49
:10E950000D0EF36E200EF3CFDBFFBF0EF36E210E14
:10E96000F3CFDBFF0E0EDBCF00F00F0EDBCF01F09D
:10E97000100EDBCF02F0110EDBCF03F03A0E2C6E3F
:10E980003F0E2D6ED40E2E6EC00EEAD8F8EC6CF051
:10E99000220E27C0DBFF230E28C0DBFF240E29C078
:10E9A000DBFF250E2AC0DBFF0E0EDBCF27F00F0E9C
:10E9B000DBCF28F0100EDBCF29F0110EDBCF2AF0D1
:10E9C0001E0EDBCF2CF01F0EDBCF2DF0200EDBCF89
:10E9D0002EF0210E09D9220EDBCF2CF0230EDBCF37
:10E9E0002DF0240EDBCF2EF0250EDBCF2FF08EEC9A
:10E9F0006DF007D9120EDBCF00F0130EDBCF01F064
:10EA0000140EDBCF02F0150EDBCF03F0CDD8010ED4
:10EA1000DBCF2CF0020EDBCF2DF0030EDBCF2EF080
:10EA2000040EE2D827C004F028C005F029C006F083
:10EA30002AC007F078D8046A800E056E310E066E83
:10EA40003F0E076EC9D827C008F028C009F029C0BA
:10EA50000AF02AC00BF0CCD8E1D8E1EC6DF069D80F
:10EA6000830E146E800E156E5E0E166EB90E176E46
:10EA7000B3D827C018F028C019F029C01AF02AC04E
:10EA80001BF0B6D814C027F015C028F016C029F026
:10EA900017C02AF0E1EC6DF027C010F028C011F08B
:10EAA00029C012F02AC013F0010EDBCF1CF0020EB9
:10EAB000DBCF1DF0030EDBCF1EF0040EDBCF1FF00B
:10EAC0001CC02CF01DC02DF01EC02EF01FC02FF05A
:10EAD000F8EC6CF027C00CF028C00DF029C00EF047
:10EAE0002AC00FF020D8010EDBCF00F0020EDBCFE2
:10EAF00001F0030EDBCF02F0040EDBCF03F000C009
:10EB000026F001C027F002C028F003C029F0260E2D
:10EB1000E15C02E2E16AE552E16EE552E5CFDAFF3F
:10EB2000E7CFD9FF120064D882D8F8EC6CF001EF7F
:10EB300076F027C000F028C001F029C002F02AC0FA
:10EB400003F01200E66E000EDA20E66E7FD8EECFFC
:10EB5000E6FFEECFE6FFEECFE6FFEFCFE6FF1200D7
:10EB60002F6E17EF76F0DBCF07F06AD80EEF76F056
:10EB7000F7EC6CF0160E27C0DBFF170E28C0DBFF8A
:10EB8000180E29C0DBFF190E2AC0DBFF1200FA0E97
:10EB9000DBCF00F0FB0EDBCF01F0FC0EDBCF02F091
:10EBA000FD0EDBCF03F01200120EDBCF27F0130EA9
:10EBB000DBCF28F0140EDBCF29F0150EDBCF2AF0C7
:10EBC0001200FA0EDBCF04F0FB0EDBCF05F0FC0EDB
:10EBD000DBCF06F0FD0E12000C0EDBCF28F00D0E81
:10EBE000DBCF29F0E4EF6CF0DBCF2FF0E1EF6DF03D
:10EBF00027C02CF028C02DF029C02EF02AC02FF0FD
:10EC00001200010E27C0DBFF020E28C0DBFF030E3F
:10EC100029C0DBFF040E2AC0DBFF120004C027F06E
:10EC200005C028F006C029F007C02AF0120000C075
:10EC300027F001C028F002C029F003C02AF012001A
:10EC40002C6A2D6A2E6A3F0E2F6E1200D950FA0FD1
:10EC5000E96EFF0EDA20EA6E1200D9CFE6FFDACFB6
:10EC6000E6FFE1CFD9FFE2CFDAFF5BD8013411E252
:10EC70000050FE08000E01540CE276D805E06CD876
:10EC8000800EEE6EEE6847D067D8800EEE6E7F0E77
:10EC90000ED047D8D890015004E6010E005C000E5B
:10ECA00001580BE261D805E057D8EE6A800EEE6E8F
:10ECB00032D052D8EE6AEE6A2ED047D8EECF00F0AE
:10ECC000EECF01F0EECF02F0EFCF03F032D800C06C
:10ECD000EEFF01C0EEFF02C0EEFF03C0EEFF21D841
:10ECE0000050010B05E025D8020E3AD8EF8E04D073
:10ECF00020D8020E35D8EF9E14D8D89001320032B9
:10ED000018D8030E2DD800C0EFFF1AD804E011D890
:10ED1000030E26D8EF8EE552E5CFDAFFE7CFD9FF15
:10ED2000120013D8040E1CD8EECF00F0EFCF01F084
:10ED30001200FA0EDBCFE9FFFB0EDBCFEAFF120079
:10ED400004D8060E0DD8EF501200FC0EDBCFE9FF01
:10ED5000FD0EDBCFEAFF1200ECDFEE6AEE6A120076
:10ED6000E926000EEA221200220E04017C6F7D6B60
:10ED7000A0EF76F0FFFFFFFFFFFFFFFFFFFFFFFFAA
:10ED8000FFFFFFFFFFFFFFFFFFFFFFFFFFFFFFFF93
:10ED9000FFFFFFFFFFFFFFFFFFFFFFFFFFFFFFFF83
:10EDA000FFFFFFFFFFFFFFFFFFFFFFFFFFFFFFFF73
:10EDB000FFFFFFFFFFFFFFFFFFFFFFFFFFFFFFFF63
:10F5100000037ACDEEDCA84000000000000018DFF8
:10F52000FFFFFFFFFFFE920000000007EFFFFFDC80
:10F53000BBCEFFFFFF91000000BFFFC76543223332
:10F5400057BFFFFD20000BFFC40000000000002497
:10F550006EFFD1007FFA000000000000000001BF34
:10F56000FA00EFC00000000000000000000DFF20C6
:10F57000FF6000000000000000000005FF60FF4089
:10F5800000000000000000000003FF70FF8000008A
:10F590000000000000000006FF50CFF30000000054
:10F5A00000000000001DFF104FFE300000000000B2
:10F5B000000001CFF80007FFD71000000000000195
:10F5C0007EFFB000005EFFFB9854333458BFFFFA53
:10F5D000000000019FFFFFFFFFFFFFFFFD50000045
:10F5E0000000017BFFFFFFFFFFE94000000000007B
:10F5F00000000246776541000000000000000000A6
:10F6000000000000000000000000000000000000FA
:10F6100000000000000000000000000000000000EA
:10F6200000000000000000010000000000000000D9
:10F6300000000000001FA00000000000000000010A
:10F640004400009F90000000000000000004FF0044
:10F6500002FF50000000000000000004FF000AFF4D
:10F6600010000000000000000004FF003FFC00004C
:10F670000000000000000004FF00BFFC77777777F0
:10F68000777777777779FF00FFFFFFFFFFFFFFFFB7
:10F69000FFFFFFFFFF00FFFFFFFFFFFFFFFFFFFF79
:10F6A000FFFFFF00333333333333333333333336F6
:10F6B000FF00000000000000000000000004FF0048
:10F6C000000000000000000000000004FF00000037
:10F6D00000000000000000000004FF000000000027
:10F6E0000000000000000003CC000000000000004B
:10F6F000000000000000000000000000000000000A
:10F7000000000000000000000000000000000000F9
:10F7100000000000000000000000000000000000E9
:10F7200000000000000000000000000000000000D9
:10F7300000083000000000000000002AFF0000BFA9
:10F74000D10000000000000008FFFF000AFFB30026
:10F75000000000000003DFFFFF004FFA0000000080
:10F760000000006FFFDBFF00CFE0000000000000A2
:10F7700008FFF808FF00FF800000000000009FFE67
:10F780004008FF00FF40000000000009FFD2000811
:10F79000FF00FF4000000000009FFD100008FF0078
:10F7A000FF800000000008FFD1000008FF00FFE01C
:10F7B000000000008FFE20000008FF009FFA0000FC
:10F7C000001AFFE200000008FF002EFFD62138EFEC
:10F7D000FD2000000008FF0004FFFFFFFFFFC10045
:10F7E00000000008FF00003DFFFFFFE700000000F1
:10F7F0000008FF00000059BB950000000000000B4E
:10F80000FF000000000000000000000000000000F9
:10F8100000000000000000000000000000000000E8
:10F8200000000000000000000000000000000000D8
:10F8300000000000000000000000002000000000A8
:10F8400000000000005E300004F80000000000002E
:10F85000000008FFD0001EFE200000000000000095
:10F8600004DFF8007FF50000000000000000002F1A
:10F87000FE00DFC000000007950000000009FF3017
:10F88000FF700000000CF70000000004FF60FF5054
:10F890000000000EF80000000003FF70FF60000091
:10F8A000002FFA0000000004FF60FFB00000007F9E
:10F8B000FE0000000009FF30BFF4000002EFFF70FF
:10F8C0000000002FFE004FFE60005EFDBFF500004F
:10F8D00003EFF70009FFFFDFFFF32FFFB656BFFF6F
:10F8E000C000008FFFFFFE4004FFFFFFFFFC100081
:10F8F00000028CDB7100002BFFFFFE800000000087
:10F90000000000000000156630000000000000004C
:10F9100000000000000000000000000000000000E7
:10F9200000000000000000000000000000000000D7
:10F930000000000000000000000000000004EFC014
:10F940000000000000000000000001AFFFC0000048
:10F9500000000000000000005EFFFFC0000000008B
:10F9600000000000001BFFD4CFC00000000000001A
:10F97000000006EFF800CFC0000000000000000209
:10F98000BFFC3000CFC0000000000000007FFF700F
:10F990000000CFC00000000000002CFFB2000000FB
:10F9A000CFC0000000000007FFE600000000CFC04D
:10F9B0000000000003CFFA1000000000CFC00000DC
:10F9C00000008FFFEAAAAAAAAAAAEFEAAAAAAA0096
:10F9D000FFFFFFFFFFFFFFFFFFFFFFFFFF00FFFF36
:10F9E000FFFFFFFFFFFFFFFFFFFFFF004444444412
:10F9F00044444444DFD44444440000000000000078
:10FA00000000CFC000000000000000000000000067
:10FA1000CFC000000000000000000000000079706E
:10FA200000000000000000000000000000000000D6
:10FA300000000000000000000000000000000000C6
:10FA40000000000000000000000000200000000096
:10FA5000001234567200000003F80000ABCDEFFF37
:10FA6000FFFFF80000001EFF8000FFFFFFFFFFFF09
:10FA7000F900000028FFF300FFDAA98767FFB00054
:10FA80000000007FFB00FF70000006FF1000000078
:10FA9000000CFF10FF7000000BFA000000000005D2
:10FAA000FF50FF7000000DF7000000000002FF7023
:10FAB000FF7000000EF7000000000002FF70FF70F2
:10FAC00000000EFA000000000004FF60FF7000005C
:10FAD0000BFE10000000000AFF30FF70000006FF60
:10FAE000B0000000006FFD00FF70000000DFFD406F
:10FAF000000029FFF500FF700000003FFFFEBABDC7
:10FB0000FFFF9000FF7000000003DFFFFFFFFFF822
:10FB1000000055200000000007DFFFFFEA30000072
:10FB2000000000000000000134420000000000005E
:10FB300000000000000000000000000000000000C5
:10FB400000000000000000000000000000000012A3
:10FB5000333321000000000000000049CEFFFFFF0A
:10FB6000FFEB7100000000007EFFFFFFFFFFFFFFC3
:10FB7000FF900000003DFFFFFCBAFFFBABEFFFFD75
:10FB8000200004FFFE83001CFD2000028EFFD10038
:10FB90001EFF900000BFE100000001CFF900AFF7A9
:10FBA000000005FF50000000001DFF10FFB0000026
:10FBB0000AFE000000000006FF50FF5000000DFB91
:10FBC000000000000002FF70FF2000000DFC00009C
:10FBD00000000003FF60FF3000000AFF200000006B
:10FBE0000008FF30FF70000005FFC1000000004F5B
:10FBF000FD00EFE1000000CFFD50000028FFF40001
:10FC00007FFD0000002DFFFFDBCDFFFF70000CD259
:10FC100000000001BFFFFFFFFFE500000110000032
:10FC20000000039DFFFEB600000000000000000081
:10FC300000000000000000000000000000000000C4
:10FC400000000000000000000000000000000000B4
:10FC500000000000000000000000000000000000A4
:10FC60000000CC7000000000000000000000000058
:10FC7000FF90000000000000000000000000FF9066
:10FC8000000000000000000000000400FF900000E1
:10FC90000000000000000049EF00FF90000000009D
:10FCA000000000049EFFFF00FF9000000000000025
:10FCB00038DFFFFFFE00FF9000000000017DFFFF26
:10FCC000FFD94000FF9000000005BFFFFFFD83004B
:10FCD0000000FF90000039EFFFFFE8300000000057
:10FCE000FF90006CFFFFFE94000000000000FF92F8
:10FCF0008EFFFFFB5000000000000000FFEFFFFF41
:10FD0000D7100000000000000000FFFFFFA400006B
:10FD10000000000000000000FFFD71000000000076
:10FD2000000000000000BA400000000000000000D9
:10FD300000000000000000000000000000000000C3
:10FD400000000000000000000000000000000000B3
:10FD500000000000000000000000000000000000A3
:10FD60000000000000000367620000000000244261
:10FD700000000004DFFFFFB20000003CFFFFC400F2
:10FD8000008FFFFFFFFE300005FFFFFFFF7008FF41
:10FD9000FB77AFFFE1003FFFA78DFFF64FFC200090
:10FDA00002DFF900BFE300008FFEDFB00000002E8D
:10FDB000FF00FF60000008FFFE1000000008FF4089
:10FDC000FF10000000CFF70000000004FF60FF00FC
:10FDD0000000003FF90000000003FF60FF2000006A
:10FDE000005FFF1000000005FF50FF80000003EFE0
:10FDF000FFA00000000AFF20DFF600005EFCCFF845
:10FE00000000004FFD004FFFC89DFFF33FFFA20021
:10FE100006FFF50007FFFFFFFE4006FFFFDCEFFFD8
:10FE2000A000004CFFFF9100005EFFFFFFFA000002
:10FE300000002430000000018EFFFB4000000000A5
:10FE400000000000000000110000000000000000A1
:10FE500000000000000000000000000000000000A2
:10FE6000000000000000000000000002210000006F
:10FE700000000000000000017DFFFFEA30000000EC
:10FE800000044000006EFFFFFFFFFA000000006F5B
:10FE9000E20008FFFFB99BEFFFC0000000BFFA00BF
:10FEA0004FFF70000005EFF80000000CFF10DFF3BB
:10FEB000000000001EFF10000006FF50FF80000041
:10FEC000000006FF50000004FF60FF40000000003B
:10FED00001FF70000004FF60FF300000000001FF20
:10FEE00070000007FF40FF700000000004FF4000AA
:10FEF000000DFE00EFE2000000000BFD0000009F7F
:10FF0000F8007FFD300000007FF400001AFFD100F0
:10FF10000BFFFB520008FF60136AFFFE200000AFDA
:10FF2000FFFFFFFFFFEFFFFFFFC200000004BFFF66
:10FF3000FFFFFFFFFFFFC500000000000269CDEFDB
:10FF4000FFEDB962000000000000000000000000AA
:10FF500000000000000000000000000000000000A1
:10FF600000000000FFFFFFFFFFFFFFFFFFFFFFFF9D
:10FF7000FFFFFFFFFFFFFFFFFFFFFFFFFFFFFFFF91
:10FF8000FFFFFFFFFFFFFFFFFFFFFFFFFFFFFFFF81
:10FF9000FFFFFFFFFFFFFFFFFFFFFFFFFFFFFFFF71
:10FFA000FFFFFFFFFFFFFFFFFFFFFFFFFFFFFFFF61
:10FFB000FFFFFFFFFFFFFFFFFFFFFFFFFFFFFFFF51
:10FFC000FFFFFFFFFFFFFFFFFFFFFFFFFFFFFFFF41
:10FFD000FFFFFFFFFFFFFFFFFFFFFFFFFFFFFFFF31
:10FFE000FFFFFFFFFFFFFFFFFFFFFFFFFFFFFFFF21
:10FFF000FFFFFFFFFFFFFFFFFFFFFFFFFFFFFFFF11
:020000040001F9
:10000000D7EC85F00501206921691200FFFFFFFF91
:10001000FFFFFFFFFFFFFFFFFFFFFFFFFFFFFFFFF0
:10002000EAEC84F057EFA4F0FFFFFFFFFFFFFFFFB4
:10003000C6EFAFF06EEFB5F0BFEFB5F00000FFFF19
:1000400080EC83F005011E6B1200FFFFFFFFFFFF36
:10005000CEEFAFF0FFFFFFFFFFFFFFFFFFFFFFFF50
:1000600057EFA4F0FFFFFFFFFFFFFFFFFFFFFFFFC2
:10007000FFFFFFFFFFFFFFFFFFFFFFFFFFFFFFFF90
:10008000C8ECA8F00501030E236F57EFA4F0FFFFA3
:10009000FFFFFFFFFFFFFFFFFFFFFFFFFFFFFFFF70
:1000A000120000EE00F00D0EEE6AEA62FDD71200BB
:1000B00066EF6AF076EF6AF0FFFFFFFFFFFFFFFFDA
:1000C00013EFA3F01AEFB6F046EFB6F0FFFFFFFF15
:1000D000FFFFFFFFFFFFFFFFFFFFFFFFFFFFFFFF30
:1000E0002FEFAEF0D9CFE6FFDACFE6FFE1CFD9FFB1
:1000F000E2CFDAFFE652006801687F0E026E036A03
:10010000D950FA0FE96EFF0EDA20EA6EEE500016B3
:10011000EE500116EE500216EE5003166AD800C0DB
:10012000EEFF01C0EEFF02C0EEFF03C0EEFFFD0ECA
:10013000DB50800B02E0010E01D0000EE66E59D8B4
:10014000060EE926000EEA22E552E750EF6EFC0E9D
:10015000DBCF00F0FD0EDBCF01F0D890003601368A
:10016000FC0E00C0DBFFFD0E01C0DBFFDB50E66EC6
:1001700040D8040EE926000EEA22E552E750EE6E62
:10018000ED6AFD0EDB50006E016AFF0E001818E1EB
:10019000015016E12ED8EECF00F0EECF01F0EECFF9
:1001A00002F0EFCF03F0005001100210031006E040
:1001B000210E04017C6F7D6B800E0BD0040E09D0E4
:1001C000FD0EDB5008E115D8EE6AEE6AEE6AEE6AC3
:1001D000010EDF6E06D0020EDF6E0BD8EE52EE522D
:1001E000EE8EDF50E552E552E5CFDAFFE7CFD9FFDB
:1001F0001200F80EDBCFE9FFF90EDBCFEAFF1200A9
:10020000BB073BBCFFD03B3C0CF83AF297493AA302
:100210003AE93A6018043A1E099039DF4C01399DD9
:100220003EE5395EED3A39258D333901BAC638CA13
:10023000DC82389E4D8438789D9F3842AC34381823
:10024000C9A33C78BD453BF902CC3BA0443E3B589A
:1002500023623B14FA313AD06DA43A93FBDD3A4F56
:10026000F8033A12718D39DB55AB39AB1277398609
:100270001EEA3952542C3924B2373900DBDA38C936
:1002800044673FA100003F809EED3F5C96533F4195
:10029000B8523F1E19CE3F01CAC13EE1CCCD3ECC83
:1002A00000003EC033333EB3B4393EA8ED913E9CCE
:1002B00026E93E91A1CB3E85F3B63E7D48E93E6EF0
:1002C00006F73FDF06253FB1902E3F98DCC73F85FC
:1002D00008313F6C0C4A3F52020C3F3B73823F2671
:1002E00051EC3F18F3B63F0D86593F08D6A13F04A5
:1002F000A2343F04816F3F0467383F040BE13F03A2
:1003000047AE3F01C2273F26E2193F3851EC3F4834
:10031000068E3F50E9103F578A723F5E18933F6444
:10032000C1553F68154D3F6C91003F6EB7803F70DF
:100330009C783F72538F3F74CFAB3F751DE73F777B
:1003400058103ED91F8A3F1317593F27E8A73F3857
:1003500019653F42B2FF3F4BF1413F53F4F13F5A21
:100360002DE03F60EAB33F6352BD3F6644D03F6833
:1003700085F03F69C7113F6AF4883F6B3C363F6D9B
:10038000AA3BC0B8AA3BC13844FEC19084D4C1D5B1
:10039000CFA2C21B0558C25DAD3BC29C2CCFC2DEB2
:1003A00040F6C31DA22BC352E459C38666EDC3AC0D
:1003B00002D0C3DCA9ABC40C9D93C4330720C46531
:1003C0006C0BC00B6C0BC08BE798C0D959DCC121FA
:1003D000ADBDC16B1F2EC1A7F2BFC1ECFCC7C227C8
:1003E000C193C26D3EA3C29FF7DEC2CB5544C30288
:1003F000540CC326AE9EC354C955C3872522C3AD32
:10040000EC0E3E22F9C93DA9F2A83D5CA08A3D163A
:10041000A1233CCFEC893C92D09A3C4FD3523C1262
:10042000B7263BCF333A3B9B787B3B72CAC03B3D00
:10043000C4D73B14BF583AE84EA53AB6FF0A3A8EE5
:1004400078BE3EBC01903E52DB713E0B57373DC13A
:100450006C183D8674223D3FFBBA3D07C21A3CC072
:10046000AB443C887C103C4CDE0E3C1F74913BFA44
:100470006ABB3BC4B56C3B99E0573B70FA8F3B3C81
:10048000000040800000410000004148000041940D
:10049000000041D833334219333342590000429AA5
:1004A000000042DA000043120000433B0000436FAB
:1004B00080004398000043C3000043F9C000441E7D
:1004C00047AE3FC147AE40410A3D4097AE1440DFC2
:1004D0005C294123AE1441673D7141A4E14841E8E4
:1004E000CCCD4224C28F425C6148428DAE1442B4EE
:1004F000947B42E66B8543133D71433C07AE4370EA
:10050000BEBE3F525D853F14EEEE3ED9FE4C3E9F8F
:10051000D9993E6785273E296EAD3DF54E043DB025
:100520005C8D3D7CEACD3D3D0BB03D152C233CEA76
:1005300012963CB84F6E3C9076823C62DE9F3C3116
:1005400066E03F7D35C63F660D7C3F4507EA3F21AB
:1005500053093EFCC4B53EC2B51C3E92F8A53E58B8
:1005600090BC3E1EB79E3DF148C33DBF42493D97FA
:1005700000D43D6F21693D3C14F53D142E983CE9B3
:10058000FFFFFFFFFFFFFFFFFFFFFFFFFFFFFFFF7B
:10059000FFFFFFFFFFFFFFFFFFFFFFFFFFFFFFFF6B
:1005A000FFFFFFFFFFFFFFFFFFFFFFFFFFFFFFFF5B
:1005B000FFFFFFFFFFFFFFFFFFFFFFFFFFFFFFFF4B
:1005C000FFFFFFFFFFFFFFFFFFFFFFFFFFFFFFFF3B
:1005D000FFFFFFFFFFFFFFFFFFFFFFFFFFFFFFFF2B
:1005E000FFFFFFFFFFFFFFFFFFFFFFFFFFFFFFFF1B
:1005F000FFFFFFFFFFFFFFFFFFFFFFFFFFFFFFFF0B
:100600002E29C943D8A2017C363DA154F0EC130633
:10061000A762F305C7C08C739398D92B4CBCCA82D0
:100620009B1E3C57D4FD16E04267186F178A12E5EF
:100630004EBED6C49EDA49DEFBA08EF52FBB7AEE05
:1006400068A99179B2153F07C2948910220B215FE6
:100650007F809A5D905A27323E35E7CCF7BF0397EB
:1006600019FFB330A548D1B55ED72A9256ACC6AAB9
:10067000B84FD238A496B67DFC76E26B749CF10438
:100680009D455970716420875B8665CF2DE602A871
:10069000601BAD25B0AEF6B9461C696140340F7ED3
:1006A000475523A351DD3AAF5CC3CEF9C5BA26EA5C
:1006B000532C6E0D28850984DFD3F4CD8141524D32
:1006C000DC6AC837C16CFAABE124087BBD0C4AB1C7
:1006D00088788B9563E36DE8CBE9FED5003B391D47
:1006E000EFF20EB75866E4D077A6F87275EB0A4BB6
:1006F0004431B450ED8F1A1F99DB338D119F148351
:100700000901BD6B0901306B316B0901326B336B31
:100710000901346B356B0901366B376B0901386998
:1007200013EE00F0010EF86E04018C0E346F4A0EC9
:10073000356F4A0E366F3F0E376F00C528F001C582
:1007400029F0E2EC6CF027C000F028C001F029C0CD
:1007500002F02AC003F02C6A2D6A7A0E2E6E440E27
:100760002F6E00C027F001C028F002C029F003C09E
:100770002AF08EEC6DF027C008F428C009F429C0D7
:100780000AF42AC00BF40401006B100E0401005D92
:1007900001E3FAD0DC0E2C6E680E2D6E800E2E6EEC
:1007A0003D0E2F6E08C427F009C428F00AC429F0B2
:1007B0000BC42AF0F7EC6CF027C004F028C005F059
:1007C00029C006F02AC007F004C02CF005C02DF0A7
:1007D00006C02EF007C02FF034C427F035C428F02F
:1007E00036C429F037C42AF0E1EC6DF027C000F0E0
:1007F00028C001F029C002F02AC003F00401005112
:10080000040DF3CFE9FFF4CFEAFF800EE926040ED2
:10081000EA2200C0EEFF01C0EEFF02C0EEFF03C0FF
:10082000EEFF020EF76E04010051002500250025A1
:10083000800FF66E0900F5CF41F40900F5CF40F4C2
:100840000900F5CF43F40800F5CF42F4800FF66EAF
:10085000F72A0900F5CF49F40900F5CF48F409005B
:10086000F5CF4BF40800F5CF4AF404010051040D14
:10087000F3CFE9FFF4CFEAFF800EE926040EEA2267
:10088000EECF08F0EECF09F0EECF0AF0EFCF0BF08D
:1008900040C42CF041C42DF042C42EF043C42FF0CC
:1008A00008C027F009C028F00AC029F00BC02AF0C0
:1008B000F7EC6CF027C004F028C005F029C006F062
:1008C0002AC007F048C42CF049C42DF04AC42EF0C9
:1008D0004BC42FF004C027F005C028F006C029F053
:1008E00007C02AF0E1EC6DF027C000F028C001F04D
:1008F00029C002F02AC003F004010051040DF3CF17
:10090000E9FFF4CFEAFF670EE926050EEA2200C0F0
:10091000EEFF01C0EEFF02C0EEFF03C0EEFF0401D8
:100920000051040DF3CFE9FFF4CFEAFF670EE9268B
:10093000050EEA22EECF00F0EECF01F0EECF02F08E
:10094000EFCF03F02C6A2D6A2E6A2F6A00C027F0C1
:1009500001C028F002C029F003C02AF0D2EC6EF0EA
:10096000010A0FE104010051040DF3CFE9FFF4CFB8
:10097000EAFF670EE926050EEA22EE6AEE6AEE6AE3
:10098000EE6A0401002B01D70401100E006F200E47
:100990000401005D12E204010051040DF3CFE9FFF0
:1009A000F4CFEAFF800EE926040EEA22EE6AEE6A30
:1009B000EE6AEE6A0401002BEAD713ECA0F0050101
:1009C000236B0501226B0501316B0501326B0501BB
:1009D000666B120013EE00F004018C0E346F4A0EA9
:1009E000356F4A0E366F3F0E376F00C528F001C5D0
:1009F00029F0E2EC6CF027C000F028C001F029C01B
:100A000002F02AC003F02C6A2D6A7A0E2E6E440E74
:100A10002F6E00C027F001C028F002C029F003C0EB
:100A20002AF08EEC6DF027C008F428C009F429C024
:100A30000AF42AC00BF402C528F003C529F0E2EC41
:100A40006CF027C000F028C001F029C002F02AC0D5
:100A500003F02C6A2D6A7A0E2E6E440E2F6E00C0A3
:100A600027F001C028F002C029F003C02AF08EEC64
:100A70006DF027C00CF428C00DF429C00EF42AC074
:100A80000FF4DC0E2C6E680E2D6E800E2E6E3D0E59
:100A90002F6E08C427F009C428F00AC429F00BC43B
:100AA0002AF0F7EC6CF027C000F028C001F029C054
:100AB00002F02AC003F000C02CF001C02DF002C0EB
:100AC0002EF003C02FF034C427F035C428F036C40C
:100AD00029F037C42AF0E1EC6DF027C024F428C0D7
:100AE00025F429C026F42AC027F40401286B296BB9
:100AF0002A6B2B6B0CC430F40DC431F40EC432F4E9
:100B00000FC433F413C529F0D1EC6CF027C000F00A
:100B100028C001F029C002F02AC003F02C6A2D6A17
:100B2000C80E2E6E420E2F6E00C027F001C028F0B6
:100B300002C029F003C02AF08EEC6DF027C07BF9CB
:100B400028C07CF929C07DF92AC07EF912C529F098
:100B5000D1EC6CF027C000F028C001F029C002F0F1
:100B60002AC003F02C6A2D6AC80E2E6E420E2F6E1C
:100B700000C027F001C028F002C029F003C02AF00D
:100B80008EEC6DF027C077F928C078F929C079F983
:100B90002AC07AF9BCEC8FF013ECA0F00501236BAE
:100BA0000501226B0501316BC0ECA0F012004FD89B
:100BB0000901BD5105E1010EBD6F00EC60F002D0EE
:100BC000F3EC64F04DDBC0ECA0F005012351030A07
:100BD00027E0020A1DE0010A12E093EC96F013EC04
:100BE000A0F0E3EC69F00301010E066F07EC8DF055
:100BF000050123510F0824E2020E236F23D093EC4A
:100C000096F04DEC94F016EC63F0050123691BD0CF
:100C1000030E235D01E117D0236B2DEC8BF013D075
:100C200013ECA0F0E3EC69F0C2EC69F00201C76BD1
:100C3000926B93EC96F0FCEC64F00501236B03D00F
:100C40002DEC8BF000D0E5EC95F0F7EF64F000C5EB
:100C500028F001C529F0E2EC6CF027C000F028C0B4
:100C600001F029C002F02AC003F02C6A2D6A7A0E26
:100C70002E6E440E2F6E00C027F001C028F002C077
:100C800029F003C02AF08EEC6DF027C008F428C0CC
:100C900009F429C00AF42AC00BF402C528F003C5E0
:100CA00029F0E2EC6CF027C000F028C001F029C068
:100CB00002F02AC003F02C6A2D6A7A0E2E6E440EC2
:100CC0002F6E00C027F001C028F002C029F003C039
:100CD0002AF08EEC6DF027C00CF428C00DF429C06A
:100CE0000EF42AC00FF410C529F0D1EC6CF027C027
:100CF00000F028C001F029C002F02AC003F02C6ADD
:100D00002D6AC80E2E6E420E2F6E00C027F001C055
:100D100028F002C029F003C02AF08EEC6DF027C045
:100D200034F428C035F429C036F42AC037F411C58C
:100D300029F0D1EC6CF027C000F028C001F029C0E8
:100D400002F02AC003F02C6A2D6AC80E2E6E420EE5
:100D50002F6E00C027F001C028F002C029F003C0A8
:100D60002AF08EEC6DF027C038F428C039F429C081
:100D70003AF42AC03BF41CC529F0D1EC6CF027C032
:100D800000F028C001F029C002F02AC003F02C6A4C
:100D90002D6AC80E2E6E420E2F6E00C027F001C0C5
:100DA00028F002C029F003C02AF08EEC6DF027C0B5
:100DB0005FF928C060F929C061F92AC062F91DC530
:100DC00029F0D1EC6CF027C000F028C001F029C058
:100DD00002F02AC003F02C6A2D6AC80E2E6E420E55
:100DE0002F6E00C027F001C028F002C029F003C018
:100DF0002AF08EEC6DF027C063F928C064F929C091
:100E000065F92AC066F917C529F0D1EC6CF027C046
:100E100000F028C001F029C002F02AC003F02C6ABB
:100E20002D6AC80E2E6E420E2F6E00C027F001C034
:100E300028F002C029F003C02AF08EEC6DF027C024
:100E40007FF928C080F929C081F92AC082F90501FB
:100E50001B515BE01BC529F0D1EC6CF027C004F0FE
:100E600028C005F029C006F02AC007F0850E2C6EB8
:100E7000EB0E2D6E1F0E2E6E410E2F6E04C027F04E
:100E800005C028F006C029F007C02AF08EEC6DF0EE
:100E900027C000F028C001F029C002F02AC003F0EA
:100EA0000CC42CF00DC42DF00EC42EF00FC42FF086
:100EB00000C027F001C028F002C029F003C02AF0CA
:100EC000F8EC6CF027C06FF928C070F929C071F9EF
:100ED0002AC072F97FC92CF080C92DF081C92EF08B
:100EE00082C92FF06FC927F070C928F071C929F0A5
:100EF00072C92AF0F8EC6CF027C06FF928C070F9BD
:100F000029C071F92AC072F905D009016F6B706BA5
:100F1000716B726B18C529F0D1EC6CF027C000F032
:100F200028C001F029C002F02AC003F02C6A2D6A03
:100F3000C80E2E6E420E2F6E00C027F001C028F0A2
:100F400002C029F003C02AF08EEC6DF027C0EFF547
:100F500028C0F0F529C0F1F52AC0F2F519C529F02D
:100F6000D1EC6CF027C004F028C005F029C006F0D1
:100F70002AC007F0660E2C6EE60E2D6EC70E2E6E82
:100F8000420E2F6E04C027F005C028F006C029F0DD
:100F900007C02AF08EEC6DF027C000F028C001F0E9
:100FA00029C002F02AC003F00CC42CF00DC42DF0AF
:100FB0000EC42EF00FC42FF000C027F001C028F09F
:100FC00002C029F003C02AF0F8EC6CF027C0F3F55A
:100FD00028C0F4F529C0F5F52AC0F6F57FC92CF034
:100FE00080C92DF081C92EF082C92FF0F3C527F0FA
:100FF000F4C528F0F5C529F0F6C52AF0F8EC6CF038
:1010000027C0F3F528C0F4F529C0F5F52AC0F6F598
:101010001AC529F0D1EC6CF027C000F028C001F00F
:1010200029C002F02AC003F02C6A2D6AC80E2E6E69
:10103000420E2F6E00C027F001C028F002C029F038
:1010400003C02AF08EEC6DF027C0F7F528C0F8F544
:1010500029C0F9F52AC0FAF513C529F0D1EC6CF0D6
:1010600027C000F028C001F029C002F02AC003F018
:101070002C6A2D6AC80E2E6E420E2F6E00C027F00D
:1010800001C028F002C029F003C02AF08EEC6DF0F8
:1010900027C07BF928C07CF929C07DF92AC07EF9D8
:1010A00012C529F0D1EC6CF027C000F028C001F087
:1010B00029C002F02AC003F02C6A2D6AC80E2E6ED9
:1010C000420E2F6E00C027F001C028F002C029F0A8
:1010D00003C02AF08EEC6DF027C077F928C078F9AC
:1010E00029C079F92AC07AF915C529F0D1EC6CF03C
:1010F00027C000F028C001F029C002F02AC003F088
:101100002C6A2D6AC80E2E6E420E2F6E00C027F07C
:1011100001C028F002C029F003C02AF08EEC6DF067
:1011200027C097F228C098F229C099F22AC09AF2F3
:1011300014C529F0D1EC6CF027C000F028C001F0F4
:1011400029C002F02AC003F02C6A2D6AC80E2E6E48
:10115000420E2F6E00C027F001C028F002C029F017
:1011600003C02AF08EEC6DF027C09BF228C09CF2E1
:1011700029C09DF22AC09EF297C22CF098C22DF091
:1011800099C22EF09AC22FF09BC227F09CC228F081
:101190009DC229F09EC22AF0F7EC6CF027C09FF2A6
:1011A00028C0A0F229C0A1F22AC0A2F20CC42CF0DF
:1011B0000DC42DF00EC42EF00FC42FF008C427F07C
:1011C00009C428F00AC429F00BC42AF0F7EC6CF02B
:1011D00027C000F028C001F029C002F02AC003F0A7
:1011E000F00E2C6E850E2D6E990E2E6E3E0E2F6E0D
:1011F00000C027F001C028F002C029F003C02AF087
:101200008EEC6DF027C014F428C015F429C016F434
:101210002AC017F414C427F015C428F016C429F006
:1012200017C42AF093EC6EF028C004F429C005F42A
:101230000401000E045D000E055902E2046B056B0B
:10124000FF0ED8800455000E055502E20469056BB7
:1012500004C44FF205011E510201C36FC46B12009A
:10126000010E02019025906F000E9121916F0501F2
:10127000185109E108C4E7F509C4E8F50AC4E9F51D
:101280000BC4EAF54ED0EFC52CF0F0C52DF0F1C53A
:101290002EF0F2C52FF008C427F009C428F00AC4C4
:1012A00029F00BC42AF0F7EC6CF027C000F028C03E
:1012B00001F029C002F02AC003F038C42CF039C470
:1012C0002DF03AC42EF03BC42FF034C427F035C4BF
:1012D00028F036C429F037C42AF0F8EC6CF027C0A7
:1012E00004F028C005F029C006F02AC007F004C0A9
:1012F0002CF005C02DF006C02EF007C02FF000C066
:1013000027F001C028F002C029F003C02AF08EECBB
:101310006DF027C0E7F528C0E8F529C0E9F52AC037
:10132000EAF508C42CF009C42DF00AC42EF00BC451
:101330002FF0E7C527F0E8C528F0E9C529F0EAC590
:101340002AF0C9EC6EF0010A08E108C4E7F509C407
:10135000E8F50AC4E9F50BC4EAF5DC0E2C6E680E5C
:101360002D6E800E2E6E3D0E2F6EE7C527F0E8C560
:1013700028F0E9C529F0EAC52AF0C9EC6EF0010AA7
:1013800001E097D0DC0E2C6E680E2D6E800E2E6E56
:101390003D0E2F6EE7C527F0E8C528F0E9C529F016
:1013A000EAC52AF0F7EC6CF027C000F028C001F085
:1013B00029C002F02AC003F000C02CF001C02DF0BB
:1013C00002C02EF003C02FF034C427F035C428F03B
:1013D00036C429F037C42AF0E1EC6DF027C024F4BC
:1013E00028C025F429C026F42AC027F4DC0E2C6E70
:1013F000680E2D6E800E2E6E3D0E2F6EE7C527F007
:10140000E8C528F0E9C529F0EAC52AF0F7EC6CF048
:1014100027C000F028C001F029C002F02AC003F064
:1014200000C02CF001C02DF002C02EF003C02FF040
:1014300038C427F039C428F03AC429F03BC42AF054
:10144000E1EC6DF027C028F428C029F429C02AF463
:101450002AC02BF408C42CF009C42DF00AC42EF0C5
:101460000BC42FF0E7C527F0E8C528F0E9C529F03F
:10147000EAC52AF08EEC6DF027C000F028C001F01C
:1014800029C002F02AC003F02C6A2D6AC80E2E6E05
:10149000420E2F6E00C027F001C028F002C029F0D4
:1014A00003C02AF0E1EC6DF06CEC6EF029C064F53D
:1014B0000BD00401246B256B266B276B286B296BE3
:1014C0002A6B2B6B0501646B0CC430F40DC431F432
:1014D0000EC432F40FC433F4BCEC8FF00501635139
:1014E000040DF3CFE9FFF4CFEAFF670EE926050EFE
:1014F000EA22EECF00F0EECF01F0EECF02F0EFCF18
:1015000003F02C6A2D6A7A0E2E6E440E2F6E00C0E8
:1015100027F001C028F002C029F003C02AF0E1EC56
:101520006DF093EC6EF028C044F229C045F205013D
:101530006351040DF3CFE9FFF4CFEAFF800EE926F3
:10154000040EEA22EECF04F0EECF05F0EECF06F067
:10155000EFCF07F0100E6325040DF3CFE9FFF4CFB2
:10156000EAFF800EE926040EEA22EECF08F0EECF65
:1015700009F0EECF0AF0EFCF0BF008C02CF009C055
:101580002DF00AC02EF00BC02FF004C027F005C0CC
:1015900028F006C029F007C02AF0F8EC6CF027C04C
:1015A00000F028C001F029C002F02AC003F02C6A24
:1015B0002D6A7A0E2E6E440E2F6E00C027F001C0E9
:1015C00028F002C029F003C02AF0E1EC6DF093ECA2
:1015D0006EF028C046F229C047F205011F051BE145
:1015E0009BC22CF09CC22DF09DC22EF09EC22FF00B
:1015F00010C427F011C428F012C429F013C42AF033
:10160000E1EC6DF027C010F428C011F429C012F4E9
:101610002AC013F408D030C410F431C411F432C419
:1016200012F433C413F410C42CF011C42DF012C4FE
:101630002EF013C42FF070C427F071C428F072C4C8
:1016400029F073C42AF0C9EC6EF0010A05E1050126
:10165000235102E1226B236912000401066B076B20
:10166000FCEC64F00201000ED880BF55000EC0559E
:1016700001E3B8D1050118513EE120C4EBF521C4C6
:10168000ECF522C4EDF523C4EEF56FC92CF070C95A
:101690002DF071C92EF072C92FF020C427F021C49B
:1016A00028F022C429F023C42AF0C9EC6EF0010A04
:1016B00011E134C467F935C468F936C469F937C42F
:1016C0006AF938C46BF939C46CF93AC46DF93BC492
:1016D0006EF910D05FC967F960C968F961C969F925
:1016E00062C96AF963C96BF964C96CF965C96DF9B6
:1016F00066C96EF9C1D034C467F935C468F936C417
:1017000069F937C46AF938C46BF939C46CF93AC459
:101710006DF93BC46EF9F3C52CF0F4C52DF0F5C599
:101720002EF0F6C52FF020C427F021C428F022C4E3
:1017300029F023C42AF0C9EC6EF0010A4FE1EFC58D
:101740002CF0F0C52DF0F1C52EF0F2C52FF020C41D
:1017500027F021C428F022C429F023C42AF0F7EC92
:101760006CF027C000F028C001F029C002F02AC0A8
:1017700003F038C42CF039C42DF03AC42EF03BC429
:101780002FF034C427F035C428F036C429F037C40C
:101790002AF0F8EC6CF027C004F028C005F029C04E
:1017A00006F02AC007F004C02CF005C02DF006C0DA
:1017B0002EF007C02FF000C027F001C028F002C0B3
:1017C00029F003C02AF08EEC6DF027C0EBF528C09D
:1017D000ECF529C0EDF52AC0EEF54ED0F7C52CF09A
:1017E000F8C52DF0F9C52EF0FAC52FF020C427F06A
:1017F00021C428F022C429F023C42AF0F7EC6CF0AD
:1018000027C000F028C001F029C002F02AC003F070
:1018100038C42CF039C42DF03AC42EF03BC42FF05C
:1018200034C427F035C428F036C429F037C42AF070
:10183000F8EC6CF027C004F028C005F029C006F0D1
:101840002AC007F004C02CF005C02DF006C02EF011
:1018500007C02FF000C027F001C028F002C029F017
:1018600003C02AF08EEC6DF027C0EBF528C0ECF534
:1018700029C0EDF52AC0EEF520C42CF021C42DF0CE
:1018800022C42EF023C42FF0EBC527F0ECC528F0BE
:10189000EDC529F0EEC52AF0C9EC6EF0010A08E1A9
:1018A00020C4EBF521C4ECF522C4EDF523C4EEF51C
:1018B000DC0E2C6E680E2D6E800E2E6E3D0E2F6E81
:1018C000EBC527F0ECC528F0EDC529F0EEC52AF0F0
:1018D000C9EC6EF0010A69E1DC0E2C6E680E2D6E0B
:1018E000800E2E6E3D0E2F6EEBC527F0ECC528F056
:1018F000EDC529F0EEC52AF0F7EC6CF027C000F03A
:1019000028C001F029C002F02AC003F000C02CF06A
:1019100001C02DF002C02EF003C02FF067C927F0E0
:1019200068C928F069C929F06AC92AF0E1EC6DF0AC
:1019300027C024F428C025F429C026F42AC027F49F
:10194000DC0E2C6E680E2D6E800E2E6E3D0E2F6EF0
:10195000EBC527F0ECC528F0EDC529F0EEC52AF05F
:10196000F7EC6CF027C000F028C001F029C002F0AD
:101970002AC003F000C02CF001C02DF002C02EF0F0
:1019800003C02FF06BC927F06CC928F06DC929F08E
:101990006EC92AF0E1EC6DF027C028F428C029F4C4
:1019A00029C02AF42AC02BF409D00401246B256B2A
:1019B000266B276B286B296B2A6B2B6BD0EC97F06F
:1019C000F5EC69F00201010EC16F22ECA0F00501F7
:1019D0002329236F100E235D04E2010E0401066F1C
:1019E000076B02D00501236B0401010E061901E10A
:1019F000075101E132D6050123510F0803E2010E20
:101A0000236F04D0C2EC69F00501236B120093EC44
:101A100096F00501236B08C420F409C421F40AC41C
:101A200022F40BC423F40201010E926F0401066B31
:101A3000076B2C6A2D6A800E2E6E3F0E2F6E20C40F
:101A400027F021C428F022C429F023C42AF0F7EC9F
:101A50006CF027C020F428C021F429C022F42AC049
:101A600023F405011F0509E1B7C293F2B8C294F24D
:101A7000B9C295F2BAC296F208D074C493F275C492
:101A800094F276C495F277C496F293C22CF094C285
:101A90002DF095C22EF096C22FF020C427F021C45D
:101AA00028F022C429F023C42AF0C9EC6EF0010A00
:101AB00001E05AD20CC42CF00DC42DF00EC42EF04F
:101AC0000FC42FF020C427F021C428F022C429F02D
:101AD00023C42AF0C9EC6EF0010A01E045D20201EC
:101AE000926B0301066B0501185164E12C6A2D6AA3
:101AF0002E6A3F0E2F6E20C427F021C428F022C486
:101B000029F023C42AF0F8EC6CF027C0EBF528C0CC
:101B1000ECF529C0EDF52AC0EEF52C6A2D6A2E6A87
:101B20003F0E2F6E20C427F021C428F022C429F0D4
:101B300023C42AF0F8EC6CF027C000F028C001F0B4
:101B400029C002F02AC003F06FC92CF070C92DF033
:101B500071C92EF072C92FF000C027F001C028F023
:101B600002C029F003C02AF0C9EC6EF0010A11E1AD
:101B700034C467F935C468F936C469F937C46AF9F9
:101B800038C46BF939C46CF93AC46DF93BC46EF9C9
:101B900010D05FC967F960C968F961C969F962C99C
:101BA0006AF963C96BF964C96CF965C96DF966C9ED
:101BB0006EF948D134C467F935C468F936C469F997
:101BC00037C46AF938C46BF939C46CF93AC46DF991
:101BD0003BC46EF92C6A2D6A2E6A3F0E2F6E20C40C
:101BE00027F021C428F022C429F023C42AF0F8ECFD
:101BF0006CF027C000F028C001F029C002F02AC014
:101C000003F0F3C52CF0F4C52DF0F5C52EF0F6C5A4
:101C10002FF000C027F001C028F002C029F003C057
:101C20002AF0C9EC6EF0010A66E12C6A2D6A2E6A70
:101C30003F0E2F6E20C427F021C428F022C429F0C3
:101C400023C42AF0F8EC6CF027C004F028C005F09B
:101C500029C006F02AC007F0EFC52CF0F0C52DF022
:101C6000F1C52EF0F2C52FF004C027F005C028F012
:101C700006C029F007C02AF0F7EC6CF027C000F08E
:101C800028C001F029C002F02AC003F038C42CF0AB
:101C900039C42DF03AC42EF03BC42FF034C427F0E1
:101CA00035C428F036C429F037C42AF0F8EC6CF0BB
:101CB00027C008F028C009F029C00AF02AC00BF09C
:101CC00008C02CF009C02DF00AC02EF00BC02FF078
:101CD00000C027F001C028F002C029F003C02AF09C
:101CE0008EEC6DF027C0EBF528C0ECF529C0EDF5C2
:101CF0002AC0EEF565D02C6A2D6A2E6A3F0E2F6E33
:101D000020C427F021C428F022C429F023C42AF0DB
:101D1000F8EC6CF027C004F028C005F029C006F0EC
:101D20002AC007F0F7C52CF0F8C52DF0F9C52EF044
:101D3000FAC52FF004C027F005C028F006C029F02E
:101D400007C02AF0F7EC6CF027C000F028C001F0C3
:101D500029C002F02AC003F038C42CF039C42DF099
:101D60003AC42EF03BC42FF034C427F035C428F019
:101D700036C429F037C42AF0F8EC6CF027C008F01C
:101D800028C009F029C00AF02AC00BF008C02CF0C6
:101D900009C02DF00AC02EF00BC02FF000C027F0B4
:101DA00001C028F002C029F003C02AF08EEC6DF0CB
:101DB00027C0EBF528C0ECF529C0EDF52AC0EEF5FB
:101DC0002C6A2D6A2E6A3F0E2F6E20C427F021C484
:101DD00028F022C429F023C42AF0F8EC6CF027C0C4
:101DE00000F028C001F029C002F02AC003F000C0B2
:101DF0002CF001C02DF002C02EF003C02FF0EBC577
:101E000027F0ECC528F0EDC529F0EEC52AF0C9ECA5
:101E10006EF0010A17E12C6A2D6A2E6A3F0E2F6EB2
:101E200020C427F021C428F022C429F023C42AF0BA
:101E3000F8EC6CF027C0EBF528C0ECF529C0EDF507
:101E40002AC0EEF5DC0E2C6E680E2D6E800E2E6E06
:101E50003D0E2F6EEBC527F0ECC528F0EDC529F03F
:101E6000EEC52AF0C9EC6EF0010A69E1DC0E2C6EB9
:101E7000680E2D6E800E2E6E3D0E2F6EEBC527F078
:101E8000ECC528F0EDC529F0EEC52AF0F7EC6CF0B2
:101E900027C000F028C001F029C002F02AC003F0DA
:101EA00000C02CF001C02DF002C02EF003C02FF0B6
:101EB00067C927F068C928F069C929F06AC92AF0FA
:101EC000E1EC6DF027C024F428C025F429C026F4E5
:101ED0002AC027F4DC0E2C6E680E2D6E800E2E6E3E
:101EE0003D0E2F6EEBC527F0ECC528F0EDC529F0AF
:101EF000EEC52AF0F7EC6CF027C000F028C001F026
:101F000029C002F02AC003F000C02CF001C02DF05F
:101F100002C02EF003C02FF06BC927F06CC928F067
:101F20006DC929F06EC92AF0E1EC6DF027C028F4E4
:101F300028C029F429C02AF42AC02BF409D00401AE
:101F4000246B256B266B276B286B296B2A6B2B6BFD
:101F5000D0EC97F005012329236F100E235D04E2D6
:101F6000010E0401066F076B0401010E061901E161
:101F7000075101E15BD5120013EE00F0010EF86E7F
:101F8000050163690401706B716B726B736B040103
:101F9000006B100E0401005D02E34CEF94F0020EA2
:101FA000F76E04010051002500250025F66E09009A
:101FB000F5CF59F40900F5CF58F40900F5CF5BF4DB
:101FC0000800F5CF5AF4400FF66E0900F5CF5DF426
:101FD0000900F5CF5CF40900F5CF5FF40800F5CFF8
:101FE0005EF4400FF66E0900F5CF41F40900F5CF1D
:101FF00040F40900F5CF43F40800F5CF42F4400F58
:10200000F66E0900F5CF45F40900F5CF44F4090058
:10201000F5CF47F40800F5CF46F4400FF66EF72AE7
:102020000900F5CF49F40900F5CF48F40900F5CFD0
:102030004BF40800F5CF4AF4400FF66E0900F5CFD7
:102040004DF40900F5CF4CF40900F5CF4FF408002A
:10205000F5CF4EF4D40E2C6E400E2D6E180E2E6E53
:10206000380E2F6E58C427F059C428F05AC429F0EE
:102070005BC42AF0D2EC6EF0010A01E1DED0450E1D
:102080002C6E120E2D6EBD0E2E6E3B0E2F6E58C492
:1020900027F059C428F05AC429F05BC42AF0C9ECCF
:1020A0006EF0010A01E1C9D04B0E2C6E890E2D6E27
:1020B000C90E2E6E380E2F6E5CC427F05DC428F05A
:1020C0005EC429F05FC42AF0D2EC6EF0010A01E18F
:1020D000B4D09A0E2C6E990E2D6E190E2E6E3E0EE9
:1020E0002F6E5CC427F05DC428F05EC429F05FC485
:1020F0002AF0C9EC6EF0010A01E19FD0440E2C6E6B
:102100008B0E2D6E6C0E2E6E3E0E2F6E40C427F081
:1021100041C428F042C429F043C42AF0D2EC6EF046
:10212000010A01E18AD05C0E2C6E8F0E2D6EA20E7C
:102130002E6E3F0E2F6E40C427F041C428F042C4DB
:1021400029F043C42AF0C9EC6EF0010A76E0250EAE
:102150002C6E060E2D6E010E2E6E3F0E2F6E48C495
:1021600027F049C428F04AC429F04BC42AF0D2EC25
:102170006EF0010A62E0C70E2C6E4B0E2D6E770ECC
:102180002E6E3F0E2F6E48C427F049C428F04AC473
:1021900029F04BC42AF0C9EC6EF0010A4EE05C0E47
:1021A0002C6E8F0E2D6E020E2E6E3F0E2F6E44C4BF
:1021B00027F045C428F046C429F047C42AF0D2ECE1
:1021C0006EF0010A3AE02C6A2D6AE00E2E6E3F0E88
:1021D0002F6E44C427F045C428F046C429F047C4F4
:1021E0002AF0C9EC6EF0010A28E0750E2C6E930EF1
:1021F0002D6ED80E2E6E3E0E2F6E4CC427F04DC4A1
:1022000028F04EC429F04FC42AF0D2EC6EF0010A37
:1022100014E0DF0E2C6E4F0E2D6E6D0E2E6E3F0EE7
:102220002F6E4CC427F04DC428F04EC429F04FC483
:102230002AF0C9EC6EF0010A02E10901358B0401B4
:102240000051040DF3CFE9FFF4CFEAFF800EE92639
:10225000040EEA22EECF04F0EECF05F0EECF06F04A
:10226000EFCF07F004C02CF005C02DF006C02EF013
:1022700007C02FF024C427F025C428F026C429F075
:1022800027C42AF0F7EC6CF027C000F028C001F05A
:1022900029C002F02AC003F058C42CF059C42DF014
:1022A0005AC42EF05BC42FF000C027F001C028F004
:1022B00002C029F003C02AF0E1EC6DF027C02CF435
:1022C00028C02DF429C02EF42AC02FF41CEC6AF08B
:1022D00004010051040DF3CFE9FFF4CFEAFF800EB3
:1022E000E926040EEA22EECF04F0EECF05F0EECFA1
:1022F00006F0EFCF07F02CC42CF02DC42DF02EC427
:102300002EF02FC42FF004C027F005C028F006C01F
:1023100029F007C02AF0F8EC6CF027C000F028C0C4
:1023200001F029C002F02AC003F004010051040D9D
:10233000F3CFE9FFF4CFEAFF800EE926040EEA228C
:1023400000C0EEFF01C0EEFF02C0EEFF03C0EEFFD3
:10235000100E04010025040DF3CFE9FFF4CFEAFFCE
:10236000800EE926040EEA22EECF04F0EECF05F04F
:10237000EECF06F0EFCF07F004C02CF005C02DF033
:1023800006C02EF007C02FF028C427F029C428F07B
:102390002AC429F02BC42AF0F7EC6CF027C000F017
:1023A00028C001F029C002F02AC003F05CC42CF060
:1023B0005DC42DF05EC42EF05FC42FF000C027F086
:1023C00001C028F002C029F003C02AF0E1EC6DF052
:1023D00027C02CF428C02DF429C02EF42AC02FF4D5
:1023E0001CEC6AF0100E04010025040DF3CFE9FF88
:1023F000F4CFEAFF800EE926040EEA22EECF04F0C5
:10240000EECF05F0EECF06F0EFCF07F02CC42CF0A6
:102410002DC42DF02EC42EF02FC42FF004C027F0B1
:1024200005C028F006C029F007C02AF0F8EC6CF0CF
:1024300027C000F028C001F029C002F02AC003F034
:10244000100E04010025040DF3CFE9FFF4CFEAFFDD
:10245000800EE926040EEA2200C0EEFF01C0EEFF66
:1024600002C0EEFF03C0EEFF04010051040DF3CFE4
:10247000E9FFF4CFEAFF800EE926040EEA22EECF50
:1024800000F0EECF01F0EECF02F0EFCF03F0100E30
:1024900004010025040DF3CFE9FFF4CFEAFF800E1D
:1024A000E926040EEA22EECF04F0EECF05F0EECFDF
:1024B00006F0EFCF07F004C02CF005C02DF006C0E9
:1024C0002EF007C02FF000C027F001C028F002C096
:1024D00029F003C02AF0F8EC6CF027C02CF428C0D7
:1024E0002DF429C02EF42AC02FF404010051040D4C
:1024F000F3CFE9FFF4CFEAFF800EE926040EEA22CB
:10250000EECF08F0EECF09F0EECF0AF0EFCF0BF0F0
:1025100008C02CF009C02DF00AC02EF00BC02FF01F
:1025200040C427F041C428F042C429F043C42AF033
:10253000E1EC6DF027C004F028C005F029C006F0DA
:102540002AC007F0100E04010025040DF3CFE9FFA7
:10255000F4CFEAFF800EE926040EEA22EECF10F057
:10256000EECF11F0EECF12F0EFCF13F010C02CF041
:1025700011C02DF012C02EF013C02FF044C427F06C
:1025800045C428F046C429F047C42AF0E1EC6DF0B8
:1025900027C00CF028C00DF029C00EF02AC00FF0A3
:1025A0000CC02CF00DC02DF00EC02EF00FC02FF07F
:1025B00004C027F005C028F006C029F007C02AF0A3
:1025C000F8EC6CF027C000F028C001F029C002F040
:1025D0002AC003F02CC42CF02DC42DF02EC42EF0F4
:1025E0002FC42FF000C027F001C028F002C029F04E
:1025F00003C02AF08EEC6DF027C040F428C041F4EF
:1026000029C042F42AC043F404010051040DF3CF61
:10261000E9FFF4CFEAFF800EE926040EEA22EECFAE
:1026200008F0EECF09F0EECF0AF0EFCF0BF008C0C4
:102630002CF009C02DF00AC02EF00BC02FF048C4BA
:1026400027F049C428F04AC429F04BC42AF0E1EC31
:102650006DF027C004F028C005F029C006F02AC09C
:1026600007F0100E04010025040DF3CFE9FFF4CFAD
:10267000EAFF800EE926040EEA22EECF10F0EECF3C
:1026800011F0EECF12F0EFCF13F010C02CF011C00C
:102690002DF012C02EF013C02FF04CC427F04DC403
:1026A00028F04EC429F04FC42AF0E1EC6DF027C0A9
:1026B0000CF028C00DF029C00EF02AC00FF00CC09D
:1026C0002CF00DC02DF00EC02EF00FC02FF004C066
:1026D00027F005C028F006C029F007C02AF0F8EC62
:1026E0006CF027C000F028C001F029C002F02AC019
:1026F00003F02CC42CF02DC42DF02EC42EF02FC4CA
:102700002FF000C027F001C028F002C029F003C05C
:102710002AF08EEC6DF027C048F428C049F429C097
:102720004AF42AC04BF440C42CF041C42DF042C4FA
:102730002EF043C42FF02CC427F02DC428F02EC453
:1027400029F02FC42AF0F7EC6CF027C004F028C061
:1027500005F029C006F02AC007F048C42CF049C48F
:102760002DF04AC42EF04BC42FF004C027F005C052
:1027700028F006C029F007C02AF0E1EC6DF027C070
:1027800000F028C001F029C002F02AC003F00401C3
:102790000051040DF3CFE9FFF4CFEAFF670EE926FD
:1027A000050EEA2200C0EEFF01C0EEFF02C0EEFF00
:1027B00003C0EEFF04010051040DF3CFE9FFF4CF95
:1027C000EAFF670EE926050EEA22EECF00F0EECF13
:1027D00001F0EECF02F0EFCF03F02C6A2D6A2E6AE3
:1027E0002F6A00C027F001C028F002C029F003C002
:1027F0002AF0D2EC6EF0010A0FE104010051040D41
:10280000F3CFE9FFF4CFEAFF670EE926050EEA22CF
:10281000EE6AEE6AEE6AEE6A04010051040DF3CF2F
:10282000E9FFF4CFEAFF670EE926050EEA22EECFB4
:1028300000F0EECF01F0EECF02F0EFCF03F070C466
:102840002CF071C42DF072C42EF073C42FF000C0B0
:1028500027F001C028F002C029F003C02AF0C9EC1B
:102860006EF0010A15E104010051040DF3CFE9FFF8
:10287000F4CFEAFF670EE926050EEA22EECF70F4E8
:10288000EECF71F4EECF72F4EFCF73F400C463F5C2
:102890000401002BC9EF8FF012000501226B010E1D
:1028A0000401046F056BEDD8F1EC9BF00A0E0501F5
:1028B0002225226F010E04010425046F000E05215C
:1028C000056F05011F0535E1B3C22CF0B4C22DF030
:1028D000B5C22EF0B6C22FF09BC227F09CC228F0E2
:1028E0009DC229F09EC22AF0E1EC6DF027C000F0F5
:1028F00028C001F029C002F02AC003F0AFC22CF0BA
:10290000B0C22DF0B1C22EF0B2C22FF000C027F03D
:1029100001C028F002C029F003C02AF0F8EC6CF0E6
:1029200027C010F428C011F429C012F42AC013F4EF
:1029300008D074C410F475C411F476C412F477C4CA
:1029400013F430C42CF031C42DF032C42EF033C453
:102950002FF010C427F011C428F012C429F013C4BA
:102960002AF0C9EC6EF0010A03E104010469056B69
:102970000401110E045D000E055995E3FF0E0419C4
:1029800001E1055105E1CFD80A0E0501225D226F54
:10299000010E0401046F056B3C0E0501225D70E21F
:1029A000FFDA05012229226F010E04010425046FBC
:1029B000000E0521056F05011F0535E1B3C22CF09E
:1029C000B4C22DF0B5C22EF0B6C22FF09BC227F0D4
:1029D0009CC228F09DC229F09EC22AF0E1EC6DF065
:1029E00027C000F028C001F029C002F02AC003F07F
:1029F000AFC22CF0B0C22DF0B1C22EF0B2C22FF097
:102A000000C027F001C028F002C029F003C02AF05E
:102A1000F8EC6CF027C010F428C011F429C012F4AF
:102A20002AC013F408D074C410F475C411F476C429
:102A300012F477C413F430C42CF031C42DF032C436
:102A40002EF033C42FF010C427F011C428F012C4A4
:102A500029F013C42AF0C9EC6EF0010A03E1040165
:102A60000469056B04010A0E045D000E055998E324
:102A7000FF0E041901E1055103E105012205226F52
:102A800012000401016B100E015D4CE20151040DB6
:102A9000F3CFE9FFF4CFEAFF000EE926060EEA22A3
:102AA000EECF00F0EECF01F0EECF02F0EFCF03F06B
:102AB0000151040DF3CFE9FFF4CFEAFF800EE926C0
:102AC000060EEA2200C0EEFF01C0EEFF02C0EEFFDC
:102AD00003C0EEFF100E0125040DF3CFE9FFF4CF84
:102AE000EAFF000EE926060EEA22EECF00F0EECF56
:102AF00001F0EECF02F0EFCF03F0100E0125040D30
:102B0000F3CFE9FFF4CFEAFF800EE926060EEA22B2
:102B100000C0EEFF01C0EEFF02C0EEFF03C0EEFFFB
:102B2000012BB1D712000401016B100E015D4CE2C4
:102B30000151040DF3CFE9FFF4CFEAFF800EE9263F
:102B4000060EEA22EECF00F0EECF01F0EECF02F05B
:102B5000EFCF03F00151040DF3CFE9FFF4CFEAFF0B
:102B6000000EE926060EEA2200C0EEFF01C0EEFFCD
:102B700002C0EEFF03C0EEFF100E0125040DF3CFDF
:102B8000E9FFF4CFEAFF800EE926060EEA22EECF37
:102B900000F0EECF01F0EECF02F0EFCF03F0100E19
:102BA0000125040DF3CFE9FFF4CFEAFF000EE9267B
:102BB000060EEA2200C0EEFF01C0EEFF02C0EEFFEB
:102BC00003C0EEFF012BB1D712000CC42CF00DC4D2
:102BD0002DF00EC42EF00FC42FF008C427F009C446
:102BE00028F00AC429F00BC42AF0C9EC6EF0010ADF
:102BF00001E096D005012351010A49E0030A45E0AE
:102C00000CC42CF00DC42DF00EC42EF00FC42FF008
:102C100008C427F009C428F00AC429F00BC42AF01C
:102C2000F7EC6CF027C000F028C001F029C002F0DA
:102C30002AC003F09A0E2C6E990E2D6E190E2E6E70
:102C40003F0E2F6E00C027F001C028F002C029F00F
:102C500003C02AF0F8EC6CF027C010F428C011F47F
:102C600029C012F42AC013F42C6A2D6A2E6A2F6A26
:102C700010C427F011C428F012C429F013C42AF09C
:102C8000D2EC6EF0010A09E103D0316948D047D097
:102C90000401106B116B126B136B2C6A2D6A7F0E83
:102CA0002E6E430E2F6E10C427F011C428F012C4EC
:102CB00029F013C42AF0C9EC6EF0010A07E10401FF
:102CC000106B116B7F0E126F430E136F10C427F041
:102CD00011C428F012C429F013C42AF06CEC6EF071
:102CE00029C031F50401006B070E005D18E20051A8
:102CF000EA6A240FE96E050EEA22EF50050131253C
:102D00000401016F050131510401015D03E2050178
:102D1000316902D001C431F50401002BE5D702D09E
:102D20000501316B120070C474F471C475F472C47F
:102D300076F473C477F405016351040DF3CFE9FF12
:102D4000F4CFEAFF800EE926040EEA22EECF00F06F
:102D5000EECF01F0EECF02F0EFCF03F0100E6325BF
:102D6000040DF3CFE9FFF4CFEAFF800EE926040E4D
:102D7000EA22EECF04F0EECF05F0EECF06F0EFCF73
:102D800007F004C02CF005C02DF006C02EF007C0DF
:102D90002FF000C027F001C028F002C029F003C0C6
:102DA0002AF0F8EC6CF027C0AFF228C0B0F229C0CE
:102DB000B1F22AC0B2F2AFC22CF0B0C22DF0B1C253
:102DC0002EF0B2C22FF074C427F075C428F076C478
:102DD00029F077C42AF0F7EC6CF027C0B3F228C0D2
:102DE000B4F229C0B5F22AC0B6F2B3C22CF0B4C214
:102DF0002DF0B5C22EF0B6C22FF097C227F098C2C0
:102E000028F099C229F09AC22AF0E1EC6DF027C0AF
:102E100000F028C001F029C002F02AC003F0AFC2C0
:102E20002CF0B0C22DF0B1C22EF0B2C22FF000C013
:102E300027F001C028F002C029F003C02AF0F8EC06
:102E40006CF027C0B7F228C0B8F229C0B9F22AC086
:102E5000BAF20CC42CF00DC42DF00EC42EF00FC429
:102E60002FF0B7C227F0B8C228F0B9C229F0BAC211
:102E70002AF0F7EC6CF027C0BBF228C0BCF229C0E6
:102E8000BDF22AC0BEF22C6A2D6A2E6A2F6ABBC21E
:102E900027F0BCC228F0BDC229F0BEC22AF0D2EC95
:102EA0006EF0010A05E10201BB6BBC6BBD6BBE6B32
:102EB00063C5C2F20401016B100E015D70E20151A5
:102EC000040DF3CFE9FFF4CFEAFF800EE926040EEC
:102ED000EA22EECF00F0EECF01F0EECF02F0EFCF1E
:102EE00003F00151040DF3CFE9FFF4CFEAFF000E28
:102EF000E926060EEA2200C0EEFF01C0EEFF02C086
:102F0000EEFF03C0EEFF100E0125040DF3CFE9FF25
:102F1000F4CFEAFF800EE926040EEA22EECF00F09D
:102F2000EECF01F0EECF02F0EFCF03F0100E01254F
